:020000040800F2
:1000000000000520F9020008157A0008197A000896
:100010001D7A0008217A0008257A000800000000F7
:100020000000000000000000000000000D040008B7
:10003000297A000800000000150400086D57000828
:1000400029040008290400082904000829040008DC
:1000500029040008290400082904000829040008CC
:1000600029040008290400082904000829040008BC
:1000700029040008290400082904000829040008AC
:10008000290400082904000829040008290400089C
:10009000290400082904000829040008290400088C
:1000A000290400082904000829040008290400087C
:1000B000290400086D6E00087D6E00082904000800
:1000C000290400082904000829040008290400085C
:1000D000290400082904000829040008290400084C
:1000E000290400082904000829040008290400083C
:1000F000290400082904000829040008290400082C
:10010000290400082904000829040008290400081B
:10011000290400082904000829040008290400080B
:1001200029040008290400082904000829040008FB
:1001300029040008290400082904000829040008EB
:1001400029040008290400082904000829040008DB
:1001500029040008290400082904000829040008CB
:1001600029040008290400082904000829040008BB
:1001700029040008290400082904000800000000E0
:10018000290400082904000829040008290400089B
:10019000290400082904000829040008290400088B
:1001A000290400082904000829040008290400087B
:1001B000290400082904000829040008290400086B
:1001C000290400082904000800B583B003F010FDDD
:1001D000384B394A1360394A136039490CE00A68D0
:1001E0004B6801F10C04886803E01168196004335E
:1001F00004329842F9D82146324B9942EFD32E4B24
:100200001A68314B9A4204D12C4B1A682F4B9A42F0
:1002100000D0FEE7274B2E4A13602E4A13602E4B68
:100220000AE0194651F8082B5B6802E000201060D4
:1002300004329A42FAD30B46284A9342F1D3244B14
:100240001B6813B9234B1B6803B1FEE704F03EFBA8
:10025000694601A803F04AFC214C224B1C1BA41048
:10026000002504E01E4B53F8253098470135AC4279
:10027000F8DC1D4C1D4B1C1BA410002504E01A4B80
:1002800053F8253098470135AC42F8DC00990198C5
:1002900006F052FE0546164C164B1C1BA41004E03B
:1002A000013C134B53F824309847002CF8DC2846C7
:1002B00003F0EEFBBABADECA00000020EC04002016
:1002C0002C040008440400087856341232547698FE
:1002D000F0040020D449002044040008540400081D
:1002E000540400085404000854040008540400088E
:1002F000540400085404000808B5FFF765FF00BF68
:1003000000BEFEE71EF0040F0CBFEFF30880EFF312
:1003100009807146414A10472DE9F04182B00446F8
:100320008846134B5E6B9F6B9D6A1B6B13F0020F2D
:100330000DD00F4BDB6A002B09DA4BF6AB6103F0F3
:10034000E1FC20B14FF00042094BDA620CE00948B1
:1003500003F0DEFBCDF800803B46324629462046BE
:1003600003F058FC00BEFEE702B0BDE8F08100BF1C
:1003700000ED00E0C4AA000800BEFEE71EF0040F76
:100380000CBFEFF30880EFF309807146244A104751
:100390002DE9F04182B004468846084B5E6B9F6BA6
:1003A0009D6A074803F0B4FBCDF800803B46324617
:1003B0002946204603F02EFC00BEFEE700ED00E0DB
:1003C000D4AA00081EF0040F0CBFEFF30880EFF36F
:1003D00009807146134A10472DE9F04182B0044666
:1003E0008846084B5E6B9F6B9D6A074803F090FB45
:1003F000CDF800803B4632462946204603F00AFCF1
:1004000000BEFEE700ED00E0E0AA000800BEFEE747
:1004100000BEFEE700BEFEE77047000019030008BB
:0C04200091030008D903000800BEFEE7AD
:10042C000470010800000020F00400200470010892
:10043C000000001000000010F0040020D84900203B
:08044C00000000100000001088
:1004800010B5044602F046F8064BA3FB0030800985
:1004900000F01CFC002221464FF0FF3000F0C0FBB2
:1004A000002010BDD34D621008B5032000F09AFB68
:1004B0000020FFF7E5FF07F0ABFA002008BD00BF02
:1004C000024A136801331360704700BFF404002030
:1004D000014B1868704700BFF404002010B50446B3
:1004E000504B5A6822F440325A60596842680A43B5
:1004F0005A600268536823F480735360026853683B
:10050000016943EA012353600268536823F0407392
:1005100053600268516883680B43536002689368B4
:1005200023F40063936002689168C3680B4393608F
:10053000826A3D4B9A4214D00268936823F070633C
:10054000936002689168836A0B43936002689368C2
:1005500023F04053936002689168C36A0B43936031
:1005600009E00268936823F07063936002689368FF
:1005700023F0405393602268936823F00203936052
:1005800022689368A16943EA41039360236A03B335
:10059000636A013B072B04D940F20F61234803F043
:1005A000ADFA2268536843F40063536022685368CD
:1005B00023F460435360636A013B4FF4604292FA54
:1005C000A2F2B2FA82F2934021684A6813434B6068
:1005D00004E02268536823F4006353602268D36AFE
:1005E00023F47003D3622168CA6AE369013B42EADB
:1005F0000353CB622268936823F4007393602268EC
:100600009368216B43EA412393602268936823F443
:100610008063936022689368616943EA81239360F1
:1006200010BD00BF002301400100000F30A70008EB
:10063000704700BF002800F0DD8010B50446036855
:100640006D4A6E498B4218BF934208D002F5807202
:10065000934204D04FF48771694803F04FFA6368FE
:10066000002B18BFB3F5803F0AD0B3F5003F07D089
:10067000B3F5403F04D040F20F11614803F03EFA59
:10068000A368002B18BFB3F1807F0AD0B3F1007FBD
:1006900007D0B3F1407F04D04FF48871584803F07D
:1006A0002DFA2369012B04D940F21111544803F0AB
:1006B00025FAA369012B04D94FF48971504803F03E
:1006C0001DFAA36A002B18BFB3F1807F2ED0B3F1BF
:1006D000007F2BD0B3F1407F28D0B3F1806F25D0BD
:1006E000B3F1A06F22D0B3F1C06F1FD0B3F1E06FB0
:1006F0001CD0B3F1006F19D0B3F1106F16D0B3F165
:10070000206F13D0B3F1306F10D0B3F1406F0DD024
:10071000B3F1506F0AD0B3F1706F07D0394A9342EA
:1007200004D040F21311364803F0E8F9E368002BD7
:1007300018BFB3F5006F04D04FF48A71304803F04E
:10074000DDF9E369013B0F2B04D940F215112C4868
:1007500003F0D4F9236B012B04D94FF48B71284893
:1007600003F0CCF96369022B04D940F21711244835
:1007700003F0C4F9236A012B04D94FF48C7120488B
:1007800003F0BCF9A26A1F4B9A4210D0E36A002B17
:1007900018BFB3F1805F0AD0B3F1005F07D0B3F1A7
:1007A000405F04D04FF48E71154803F0A7F9236C15
:1007B0002BB9636484F83C302046FFF739FF236C83
:1007C00013F0100F11D1226C0F4B134043F00203B2
:1007D00023642046FFF782FE00206064236C23F030
:1007E000030343F00103236400E00120002384F8A5
:1007F0003C3010BD01207047002101400020014025
:1008000030A700080100000FFDEEFFFF10B582B019
:100810000446002301938369012B04D94FF4DD7151
:10082000414803F06BF9E36A002B18BFB3F1805F16
:100830000AD0B3F1005F07D0B3F1405F04D040F2BB
:10084000BB11394803F05AF994F83C30012B5FD0C2
:10085000012384F83C3023689A6812F0010F13D109
:100860009A6842F001029A60304B1B68304AA2FB42
:1008700003239B0C03EB4303019302E0019B013B29
:100880000193019B002BF9D12268936813F0010FAB
:1008900040D0216C274B0B4043F480732364536892
:1008A00013F4806F05D0236C23F4405343F480533A
:1008B0002364236C13F4805F04D0636C23F006037D
:1008C000636401E000236364002384F83C306FF02C
:1008D00002031360184B5B6813F01F0F0AD12368E3
:1008E0009A6812F0405F17D19A6842F080429A608D
:1008F000002016E02368114A93420FD19A6812F043
:10090000405F0DD19A6842F080429A60002008E072
:10091000022006E0002004E0002002E0002000E0C9
:10092000002002B010BD00BF30A700080C0000205E
:1009300083DE1B43FEF8FFFF00230140002001403F
:1009400070B503689A6812F4806F0CD09B6813F43A
:10095000807F08D0036C43F020030364002380F8F9
:100960003C30012070BD0D460446FFF7B1FD064640
:1009700011E0B5F1FF3F0ED025B1FFF7A9FD801BB7
:10098000854208D2236C43F004032364002384F8D7
:100990003C30032070BD23681A6812F0020FE8D0C3
:1009A0006FF012021A60236C43F40073236423680F
:1009B0009A6812F0405F17D1A269BAB9DA6A12F4E4
:1009C000700F03D09B6813F4806F11D1236C23F454
:1009D00080732364236C13F4805F0BD1236C43F08A
:1009E00001032364002070BD002070BD002070BD95
:1009F000002070BD002070BD0368D86C704700BF38
:100A000030B583B005460C46002301930B686E4A4F
:100A1000934218BF122B04D940F2FB416B4803F0FC
:100A20006DF86368013B0F2B04D940F2FC41674825
:100A300003F064F8A368072B04D940F2FD41634832
:100A400003F05CF895F83C30012B00F0BA800123EC
:100A500085F83C302368092B22D92868C2689BB2EC
:100A600003EB43031E3B072101FA03F322EA0303CE
:100A7000C3602368544A934206D12A68D368A168A8
:100A800043EA0163D3601FE02968C868A2689BB28B
:100A900003EB43031E3B02FA03F30343CB6013E073
:100AA000286802699BB203EB4303072101FA03F3B1
:100AB00022EA0303036129680869A368228802EB1C
:100AC0004202934003430B616368062B16D82868E3
:100AD000426B03EB8303053B1F2101FA03F322EA78
:100AE000030343632968486B636803EB8303053B97
:100AF000228802FA03F303434B632EE00C2B16D833
:100B00002868026B03EB8303233B1F2101FA03F3E5
:100B100022EA030303632968086B636803EB83031A
:100B2000233B228802FA03F303430B6315E0286892
:100B3000C26A03EB8303413B1F2101FA03F322EA5C
:100B40000303C3622968C86A636803EB8303413BFC
:100B5000228802FA03F30343CB622A681C4B9A42B1
:100B600007D12368122B04D11A4A536843F4800337
:100B700053602A68164B9A421FD12368124A112BE0
:100B800018BF934219D1134A536843F400035360CA
:100B900022680D4B9A4210D10F4B1B680F4AA2FBE3
:100BA00003239B0C03EB83035A00019202E0019B99
:100BB000013B0193019B002BF9D1002085F83C00FB
:100BC00000E0022003B030BD1200001030A7000882
:100BD00000200140002301400C00002083DE1B4365
:100BE000006C704710B50446C31E042B03D9A42122
:100BF000084802F083FF084AD36823F4E0631B042B
:100C00001B0C240204F4E0641C43044B2343D36014
:100C100010BD00BF60A7000800ED00E00000FA056D
:100C200070B504460E4615460F2A03D9BC21184854
:100C300002F064FF0F2E03D9BD21154802F05EFFBC
:100C4000144BDA68C2F30222C2F10701042928BF5B
:100C50000421131D062B01D9033A00E000220123D1
:100C600003FA01F101393140914003FA02F2013AED
:100C70002A400A43002C06DA04F00F041201D2B213
:100C8000054B1A5570BD1201D2B2044B1A5570BDF6
:100C900060A7000800ED00E014ED00E000E400E0D3
:100CA00010B5041E03DAD021064802F027FF6209BE
:100CB00004F01F04012303FA04F4034B43F8224019
:100CC00010BD00BF60A7000800E100E00138B0F1EE
:100CD000807F0AD2064B5860F021064A82F8231022
:100CE0000020986007221A6070470120704700BFFB
:100CF00010E000E000ED00E010B50446042818BF45
:100D0000002804D040F2B311084802F0F7FE042C8A
:100D100005D1074A136843F00403136010BD044A69
:100D2000136823F00403136010BD00BF60A7000820
:100D300010E000E0704700BFC8B110B5044602687B
:100D40000C4B9A4203D0EE210B4802F0D7FE2379D8
:100D500013F0FF0F04D1002363712046FFF7EAFF71
:100D600002232371002020610123237110BD012083
:100D7000704700BF0074004094A7000838B50446CF
:100D80000D46002918BF102904D04FF4B7711C4834
:100D900002F0B4FE6379012B30D00123637102228B
:100DA000227122681168AB400B43136085B9226839
:100DB0001168136803F03803382B14BF0023012394
:100DC00013EA910315D0536843F00103536010E018
:100DD00022681168136803F46013B3F5601F14BF31
:100DE0000023012313EA914303D0536843F0020325
:100DF0005360012323710020607138BD022038BD8B
:100E000094A70008F8B504460E4615460B68002B5B
:100E100018BF242B12D00C2B10D0142B0ED01C2B4F
:100E20000CD0042B0AD02C2B08D0342B06D03C2B12
:100E300004D040F20E311C4802F060FE7368002BB3
:100E400018BF022B04D040F20F31174802F056FEB3
:100E5000002D18BF102D04D04FF44471124802F039
:100E60004DFE6379012B1CD0012060710223237198
:100E700027683A6840F6FE73AB4022EA0301336804
:100E800072681343AB400B433B6021680B68C02280
:100E900002FA05F523EA05050D6020710020607156
:100EA000F8BD0220F8BD00BF94A70008F0B583B0DC
:100EB000074614461D46002301930E46994218BF6B
:100EC000102904D040F24631134802F017FE002CDE
:100ED00018BF042C06D0082C04D040F247310E482D
:100EE00002F00CFE4FF6F0739D4204D94FF452719C
:100EF000094802F003FE3B68019326B9019B1C449C
:100F00000834019403E0019B1C4414340194019BB8
:100F10001D60002003B0F0BD94A700082DE9F04744
:100F200082B080460F46B34BB34A904218BF9842F6
:100F30002BD003F50063C31A18BF012302F500622A
:100F4000904222D00BB3AD4BC31A18BF012302F558
:100F50000062904219D0C3B1A94BC31A18BF012334
:100F600002F50062904210D07BB1A64BC31A18BFA5
:100F7000012302F50062904207D033B1A24B9842A0
:100F800003D0C321A14802F0B9FD3B881BB9C4219D
:100F90009E4802F0B3FD7B68112B18BF012B20D9AE
:100FA000022B1ED0122B1CD0994A934219D002F565
:100FB0008012934215D002F58012934211D0A2F50F
:100FC000F81293420DD002F58012934209D002F537
:100FD0008012934205D0032B03D0C5218B4802F029
:100FE0008DFDBB68022B03D9C621884802F086FD1F
:100FF0000025F9E00124AC403E682640B44240F0B0
:10100000F2807B68122B18BF022B1CD13B690F2B7F
:1010100018BF0C2B07D90D2B05D00E2B03D0D721D1
:101020007A4802F06BFDEA08083258F8220005F011
:10103000070399000F238B4020EA03003B698B4094
:10104000034348F82230D8F800304FEA450A4FF001
:10105000030909FA0AF96FEA090903EA09027B6838
:1010600003F0030303FA0AF31343C8F800307B6864
:101070005A1E112B18BF012A01D9122B1BD1FB6854
:10108000032B03D9EB21614802F038FDD8F8083072
:1010900009EA0302FB6803FA0AF31343C8F80830AD
:1010A000D8F8043023EA04047B68C3F30013AB4090
:1010B0001C43C8F80440D8F80C3009EA0309BB689F
:1010C00003FA0AF349EA0303C8F80C307B6813F00B
:1010D000805F00F08880002301934E4B5A6C42F4ED
:1010E00080425A645B6C03F480430193019BA9081E
:1010F0008A1C494B53F8220005F003039B000F2282
:101100009A4020EA02003C4A904525D002F58062D0
:10111000904523D002F58062904521D002F580628F
:1011200090451FD002F5806290451DD002F5806287
:1011300090451BD002F58062904519D002F580627F
:10114000904517D002F58062904515D002F5806277
:10115000904513D1092212E0002210E001220EE096
:1011600002220CE003220AE0042208E0052206E045
:10117000062204E0072202E0082200E00A2202FA26
:1011800003F303430231244A42F82130234B1A6807
:10119000F34302EA0301786810F4803F01D046EA85
:1011A00002011E4A1160526803EA0201786810F4D5
:1011B000003F01D046EA0201184A5160926803EAF2
:1011C0000201786810F4801F01D046EA0201134A38
:1011D0009160D2681340796811F4001F01D046EA8B
:1011E00002030E4AD36001350F2D7FF603AF02B024
:1011F000BDE8F087000402400000024000140240F5
:10120000001C02400024024000280240C4A700083D
:10121000000011100038024000380140003C01403D
:1012200038B505460C4621B940F28D11044802F04C
:1012300065FC2B691C4201D0012038BD002038BD5F
:10124000C4A7000870B5064615460C4621B940F201
:10125000AD11084802F052FC012D04D94FF4D771AA
:10126000044802F04BFC0DB1B46170BD2404B461BC
:1012700070BD00BFC4A700082DE9F04180460C46B0
:1012800017461E46069D0368204A21498B4218BF17
:1012900093420CD002F58062934208D002F580623E
:1012A000934204D041F259011A4802F027FCB6F1EA
:1012B000807F18BFB6F1007F05D026B141F25A01F8
:1012C000144802F01BFCB5F5804F18BFB5F5105F50
:1012D0000BD02B1C18BF0123B5F5005F05D023B13F
:1012E00041F25B010B4802F009FCD8F800104B6892
:1012F000094A1A40C4F3090343EA0743334345EA62
:10130000030442EA04034B60BDE8F081005800404A
:1013100000540040F4A70008009800FC70B5044693
:101320000D46FFF7D5F8064623689B6913F0100FAA
:1013300012D1002070BDB5F1FF3F0DD025B1FFF7F0
:10134000C7F8801B854207D2012384F8353000237B
:1013500084F83430032070BD23689A6912F0200F9E
:10136000E9D01022DA6123682022DA6123689A69C1
:1013700012F0010F01D10122DA612268536823F0D3
:10138000FF7323F48B3323F4FF7323F001035360C3
:101390000423A363012084F83500002384F834304B
:1013A00070BD00BF70B504460D46FFF791F80646C4
:1013B00019E029462046FFF7B1FFD8B9B5F1FF3F44
:1013C00011D025B1FFF784F8801B85420BD2A36BA7
:1013D00043F02003A363012384F83530002384F80D
:1013E0003430032070BD23689B6913F0020FE0D0F6
:1013F000002070BD012070BD2DE9F04105460E466C
:1014000090461C46FFF764F80746B8F1000F12D06B
:101410002EE0B4F1FF3F0ED024B1FFF759F8C01B06
:10142000844208D2012385F83530002385F8343012
:101430000320BDE8F0812B689B6926EA0303C3F310
:101440001003002BE5D10020BDE8F081B4F1FF3F8F
:101450000ED024B1FFF73CF8C01B844208D2012310
:1014600085F83530002385F834300320BDE8F0815D
:101470002B689B6926EA0303C3F31003002BE5D016
:101480000020BDE8F08100BF70B505460C46FFF7AF
:101490001FF8064616E021462846FFF73FFFC0B971
:1014A00024B1FFF715F8801B84420BD2AB6B43F0DD
:1014B0002003AB63012385F83530002385F83430F1
:1014C000032070BD2B689B6913F0200FE3D0002030
:1014D00070BD012070BD00BF70B504460D46FEF71B
:1014E000F7FF064631E029462046FFF717FF0028A0
:1014F00032D123689A6912F0200F14D02022DA61C9
:101500002268536823F0FF7323F48B3323F4FF73B3
:1015100023F0010353600023A363012084F8350006
:1015200084F8343070BD25B1FEF7D2FF801B8542B0
:101530000BD2A36B43F02003A363012384F835305F
:10154000002384F83430032070BD23689B6913F0B6
:10155000040FC8D0002070BD012070BD002800F02D
:10156000A88010B504460368534A54498B4218BFFB
:1015700093420CD002F58062934208D002F580625B
:10158000934204D040F22B114D4802F0B7FAA36801
:10159000B3F5806F04D34FF49671494802F0AEFA68
:1015A000E368013B012B04D940F22D11444802F0BD
:1015B000A5FA2369002B18BFB3F5004F04D04FF4F0
:1015C00097713F4802F09AFA6369FF2B04D940F201
:1015D0002F113B4802F092FAA369072B04D94FF46C
:1015E0009871374802F08AFAE369002B18BFB3F507
:1015F000002F04D040F23111314802F07FFA236A03
:10160000002B18BFB3F5003F04D04FF499712C485C
:1016100002F074FA94F8353013F0FF0F05D100236F
:1016200084F83430204603F04DFD022384F8353031
:101630002268136823F0010313602268636823F0B3
:10164000706313612268936823F400439360A36876
:101650005BB1E268012A04D1226843F4004393603D
:1016600003E0226843F404439360E368022B03D150
:1016700023684FF400625A6022685168114B0B4393
:1016800053602268216963690B43A16943EA01231E
:10169000D3602268E169236A0B43136022681368F0
:1016A00043F0010313600020A063012384F8353068
:1016B00010BD0120704700BF00580040005400409A
:1016C000F4A7000800800002704700BF38B310B5CF
:1016D00004460368134A14498B4218BF93420CD046
:1016E00002F58062934208D002F58062934204D0F2
:1016F00040F27D110D4802F001FA022384F83530E2
:101700002268136823F0010313602046FFF7DCFF13
:101710000020A06384F8350084F8340010BD012057
:10172000704700BF0058004000540040F4A7000874
:101730002DE9F04383B01D4690F83530DBB2012B24
:1017400040F0918004460F461646002D18BF002A2F
:1017500000F08B8003689B6913F4004F40F0878092
:1017600090F83430012B00F08480012380F834306D
:10177000122380F8353000238363FF2D0AD94FF4FC
:10178000005300934FF08073FF22FFF775FD4FF079
:10179000FF080AE04FF4005300934FF00073EAB2E1
:1017A000FFF76AFDA84600E04E460A992046FFF77B
:1017B000F9FD20B1A36B042B5DD1012360E0236808
:1017C00006F1010932789A62013DADB2B8F1010823
:1017D0000CBF01230023002D0CBF002303F00103E5
:1017E000FBB10A9B002280212046FFF705FE00285E
:1017F00043D1FF2D0BD9002300934FF08073FF22BC
:1018000039462046FFF738FD4FF0FF0809E0002376
:1018100000934FF00073EAB239462046FFF72CFDE3
:10182000A846002DC0D10A992046FFF72DFE034699
:1018300020B1A36B042B22D1012321E022682021B7
:10184000D16121684A6822F0FF7222F48B3222F4BF
:10185000FF7222F001024A60012284F83520002242
:1018600084F834200CE002230AE0012308E002237C
:1018700006E0022304E0032302E0032300E0032345
:10188000184603B0BDE8F0832DE9F04383B01D4650
:1018900090F83530DBB2012B40F0918004460F46C2
:1018A0001646002D18BF002A00F08B8003689B6944
:1018B00013F4004F40F0878090F83430012B00F093
:1018C0008480012380F83430222380F835300023CF
:1018D0008363FF2D0AD94FF4105300934FF08073A8
:1018E000FF22FFF7C9FC4FF0FF080AE04FF4105346
:1018F00000934FF00073EAB2FFF7BEFCA84600E089
:101900004E4604212046FFF7E7FD20B1A36B042BD0
:101910005DD1012360E006F1010923685B6A337041
:10192000013DADB2B8F101080CBF01230023002D29
:101930000CBF002303F00103FBB10A9B00228021AE
:101940002046FFF759FD002843D1FF2D0BD9002376
:1019500000934FF08073FF2239462046FFF78CFC3E
:101960004FF0FF0809E0002300934FF00073EAB244
:1019700039462046FFF780FCA846002DC0D119212A
:101980002046FFF781FD034620B1A36B042B22D133
:10199000012321E022682021D16121684A6822F0D8
:1019A000FF7222F48B3222F4FF7222F001024A60AD
:1019B000012284F83520002284F834200CE0022330
:1019C0000AE0012308E0022306E0022304E00323E7
:1019D00002E0032300E00323184603B0BDE8F083D0
:1019E0002DE9F04782B00024019490F83540E4B22C
:1019F000012C40F08C800468A46914F4004F40F07E
:101A0000888090F83440012C00F085801F46904675
:101A100089460646012380F83430022380F83530A9
:101A2000002383633268F368012B04D1C9F30901F1
:101A30003E4B0B4303E0C9F3090343F420535360C7
:101A4000FEF746FD824611E0B7F1FF3F0ED02FB101
:101A5000FEF73EFDCAEB0000874207D2012386F85D
:101A60003530002386F8343003235BE03568AB69FA
:101A700013F0200F08D1AB6913F0100F04D196F8C2
:101A80003540E4B2032CDFD1AB6913F0100F12D153
:101A90003B46002220213046FFF7AEFC03460028DB
:101AA0003BD132682021D161012286F83520002205
:101AB00086F8342036E03B46002220213046FFF7EE
:101AC0009BFC60BB33681022DA6133682022DA6144
:101AD000019B5A1C019243450ED13268536843F46E
:101AE000804353603B46002220213046FFF784FCB0
:101AF000B8B933682022DA61019B984592D8012356
:101B000086F83530002386F8343003230AE00223B8
:101B100008E0022306E0022304E0032302E003239B
:101B200000E00323184602B0BDE8F0870020000261
:101B300010B582B0002301931C4B1A6C42F0805206
:101B40001A641B6C03F080530193019B184A1368BD
:101B500043F480331360FEF7BBFC044605E0FEF758
:101B6000B7FC001BB0F57A7F1AD8114B5B6813F4F1
:101B7000803FF4D00E4A136843F400331360FEF73D
:101B8000A7FC044605E0FEF7A3FC001BB0F57A7F36
:101B900008D8074B5B6813F4003FF4D0002002E044
:101BA000032000E0032002B010BD00BF0038024057
:101BB0000070004030B583B0044603680F2B04D991
:101BC0004FF480719A4801F099FF236813F0010FD8
:101BD00000F08E806368002B18BFB3F5803F07D0FC
:101BE000B3F5A02F04D04FF48371914801F086FF24
:101BF000904B9B6803F00C03042B0AD08D4B9B6821
:101C000003F00C03082B0DD18A4B5B6813F4800F93
:101C100008D0884B1B6813F4003F69D06368002B21
:101C200066D159E2834B1A6822F480321A601A682E
:101C300022F480221A601A6822F480321A60FEF7B9
:101C400047FC054605E0FEF743FC401B642800F214
:101C50004582784B1B6813F4003FF4D1754A136832
:101C600023F4803313606368B3F5803F09D11346D2
:101C7000126822F480221A601A6842F480321A60D4
:101C800015E0B3F5A02F09D16A4B1A6842F48022FF
:101C90001A601A6842F480321A6008E0654B1A68CC
:101CA00022F480221A601A6822F480321A60636873
:101CB0007BB1FEF70DFC054605E0FEF709FC401B75
:101CC000642800F20D825B4B1B6813F4003FF4D0D4
:101CD0000EE0FEF7FDFB054605E0FEF7F9FB401BB5
:101CE000642800F2FF81534B1B6813F4003FF4D1CA
:101CF000236813F0020F6ED0E368012B04D940F281
:101D000047114B4801F0FAFE23691F2B04D94FF409
:101D1000A471474801F0F2FE464B9B6813F00C0F8C
:101D20000AD0444B9B6803F00C03082B1BD1414B9A
:101D30005B6813F4800F16D13E4B1B6813F0020F43
:101D400003D0E368012B40F0CF813A48036823F0C9
:101D5000F8012369F82292FAA2F2B2FA82F29340D1
:101D60000B43036037E0E3680BB3324A136843F078
:101D700001031360FEF7ACFB054605E0FEF7A8FB88
:101D8000401B642800F2B2812A4B1B6813F0020F3B
:101D9000F4D02848036823F0F8012369F82292FA66
:101DA000A2F2B2FA82F293400B43036013E0214A9D
:101DB000136823F001031360FEF78AFB054605E074
:101DC000FEF786FB401B642800F29281194B1B68CA
:101DD00013F0020FF4D1236813F0080F37D06369B2
:101DE000012B04D94FF4C471114801F087FE6369D7
:101DF000A3B1104A536F43F001035367FEF768FB2A
:101E0000054605E0FEF764FB401B642800F2728182
:101E1000084B5B6F13F0020FF4D018E0054A536FC4
:101E200023F001035367FEF753FB05460AE000BFAA
:101E300034A8000800380240FEF74AFB401B642823
:101E400000F25A81B54B5B6F13F0020FF4D1236897
:101E500013F0040F00F09480A368052B18BF012B2A
:101E600004D94FF4D971AE4801F048FE0023019324
:101E7000AA4B1A6C42F080521A641B6C03F0805318
:101E80000193019BA74A136843F480731360FEF724
:101E90001FFB054605E0FEF71BFB401B642800F214
:101EA0002D81A04B1B6813F4807FF4D09B4B1A6FDD
:101EB00022F001021A671A6F22F004021A671A6FE1
:101EC00022F001021A67FEF703FB054607E0FEF762
:101ED000FFFA401B41F28833984200F211818F4B88
:101EE0001B6F13F0020FF2D18C4A136F23F0010322
:101EF0001367A368012B09D11346126F22F0040265
:101F00001A671A6F42F001021A6714E0052B09D113
:101F1000824B1A6F42F004021A671A6F42F00102F4
:101F20001A6708E07D4B1A6F22F004021A671A6FD5
:101F300022F001021A67A3688BB1FEF7C9FA0546C1
:101F400007E0FEF7C5FA401B41F28833984200F2E1
:101F5000D980724B1B6F13F0020FF2D010E0FEF726
:101F6000B7FA054607E0FEF7B3FA401B41F28833A3
:101F7000984200F2C980694B1B6F13F0020FF2D137
:101F8000A369022B04D94FF4FB71654801F0B6FD3B
:101F9000A369002B00F0BA80604A926802F00C023C
:101FA000082A00F0B580022B40F08180E369002B05
:101FB00018BFB3F5800F04D040F2FF11584801F06C
:101FC0009DFD236A023B3D2B04D94FF40071544818
:101FD00001F094FD636A323BB3F5BF7F04D940F250
:101FE00001214F4801F08AFDA36A022B18BF042B80
:101FF00008D0062B06D0082B04D040F20221484816
:1020000001F07CFDE36A023B0D2B04D940F2032171
:10201000434801F073FD414A136823F08073136055
:10202000FEF756FA054604E0FEF752FA401B642814
:1020300070D83A4B1B6813F0007FF5D1216A636AB0
:1020400047F6C07292FAA2F2B2FA82F293401943B2
:10205000A36A5B085A1E4FF4403393FAA3F3B3FA12
:1020600083F302FA03F30B43E2691343E26A4FF08E
:10207000706191FAA1F1B1FA81F18A40134343F002
:102080000053264A5360136843F080731360FEF7D1
:102090001FFA044604E0FEF71BFA001B64283BD835
:1020A0001E4B1B6813F0007FF5D000203DE01B4A5B
:1020B000136823F080731360FEF70AFA044604E005
:1020C000FEF706FA001B64282ED8144B1B6813F089
:1020D000007FF5D1002028E0012026E0032024E045
:1020E000032022E0032020E001201EE003201CE06A
:1020F00003201AE0032018E0032016E0032014E078
:10210000032012E0032010E003200EE000200CE08A
:1021100001200AE0032008E0032006E00038024026
:1021200034A8000800700040032003B030BD00BF99
:1021300070B504460D460368013B0E2B04D940F2EE
:102140006221894801F0DAFC0F2D04D940F26321A5
:10215000854801F0D3FC854B1B6803F00F039D42BB
:1021600040F28F80814A136823F00F032B431360E2
:10217000136803F00F039D4240F05781236813F06A
:10218000020F1ED0A368002B18BF802B12D0902BFB
:1021900010D0A02B0ED0B02B0CD0C02B0AD0D02B3F
:1021A00008D0E02B06D0F02B04D040F279216E4805
:1021B00001F0A4FC6E498B6823F0F002A36813437E
:1021C0008B60236813F0010F00F0EB806368022B33
:1021D00004D94FF42071644801F090FC6268012A30
:1021E00005D1634B1B6813F4003F0ED11FE1022A97
:1021F00005D15F4B1B6813F0007F06D119E15C4BE2
:102200001B6813F0020F00F0168159498B6823F008
:10221000030313438B60FEF75BF905466368012BEC
:102220000FD107E0FEF754F9401B41F28833984282
:1022300000F203814E4B9B6803F00C03042BF1D199
:10224000AFE0022B17D107E0FEF742F9401B41F245
:102250008833984200F2F380454B9B6803F00C03EF
:10226000082BF1D19DE0FEF733F9401B41F2883392
:10227000984200F2E6803E4B9B6813F00C0FF2D1BF
:102280008FE0236813F0020F1ED0A368002B18BF45
:10229000802B12D0902B10D0A02B0ED0B02B0CD0B6
:1022A000C02B0AD0D02B08D0E02B06D0F02B04D0C6
:1022B0004FF432712C4801F021FC2D498B6823F03A
:1022C000F002A36813438B60236813F0010F5DD005
:1022D0006368022B04D940F2CF21234801F00EFCA1
:1022E0006268012A05D1224B1B6813F4003F0ED10E
:1022F000A9E0022A05D11E4B1B6813F0007F06D10E
:10230000A3E01B4B1B6813F0020F00F0A0801849DC
:102310008B6823F0030313438B60FEF7D9F806465E
:102320006368012B0FD107E0FEF7D2F8801B41F262
:102330008833984200F28D800D4B9B6803F00C03AC
:10234000042BF1D122E0022B1BD106E0FEF7C0F8EE
:10235000801B41F2883398427DD8054B9B6803F07F
:102360000C03082BF2D111E034A80008003C024015
:1023700000380240FEF7ACF8801B41F288339842E7
:102380006BD8384B9B6813F00C0FF3D1364A1368A7
:1023900023F00F032B431360136803F00F039D42D8
:1023A0005DD1236813F0040F1AD0E368002B18BF27
:1023B000B3F5805F0DD0B3F5A05F0AD0B3F5C05F71
:1023C00007D0B3F5E05F04D040F21E31274801F09A
:1023D00095FB24498B6823F4E052E36813438B6038
:1023E000236813F0080F1BD02369002B18BFB3F527
:1023F000805F0DD0B3F5A05F0AD0B3F5C05F07D002
:10240000B3F5E05F04D040F22531184801F076FBC7
:10241000144A936823F46043216943EAC10393603B
:102420000020FEF72DF8002070BD012070BD0120B6
:1024300070BD012070BD012070BD032070BD032060
:1024400070BD032070BD012070BD012070BD012052
:1024500070BD032070BD032070BD032070BD01203E
:1024600070BD00BF00380240003C024034A80008A4
:10247000254B9B6803F00C03042B3FD0082B01D0A5
:102480002248704710B4204B586800F03F005B684A
:1024900013F4800F10D01E4BB3FBF0F01A4B5A68A8
:1024A00047F6C0710A4091FAA1F3B3FA83F322FA16
:1024B00003F303FB00F310E0144BB3FBF0F0124BFB
:1024C0005A6847F6C07402EA040194FAA4F2B2FA18
:1024D00082F221FA02F202FB00F30B4A506800F488
:1024E00040324FF4403090FAA0F0B0FA80F022FA77
:1024F00000F001304000B3FBF0F001E00448704709
:102500005DF8044B704700BF003802400024F4001F
:1025100080BA8C0108B5FFF7ABFF084B9B6803F04E
:10252000F002F02393FAA3F3B3FA83F322FA03F34E
:10253000034AD35CD840034B186008BD0038024002
:1025400024A800080C000020F0B583B004460268FF
:10255000644B13401BB98721634801F0CFFA23680D
:1025600013F0010F16D0636B002B18BFB3F5000FEB
:1025700003D08D215C4801F0C1FA5C4B9A6822F4CB
:1025800000029A609968626B0A439A60636B1BB1A0
:10259000002702E0002700E00127236813F4002F42
:1025A0001DD0E36B002B18BFB3F5801F06D0B3F529
:1025B000001F03D09D214C4801F0A0FA4B49D1F8EF
:1025C0008C3023F44012E36B1343C1F88C30E36B7F
:1025D000B3F5801F00D101271BB1002502E00025C3
:1025E00000E00125236813F4801F1CD0236C002B0E
:1025F00018BFB3F5800F06D0B3F5000F03D0B1219B
:10260000394801F07BFA3949D1F88C3023F4400283
:10261000236C1343C1F88C30236CB3F5800F00D1C9
:10262000012703B90125236813F0807F00D001271B
:1026300013F0200F6CD0002301932C4B1A6C42F046
:1026400080521A641B6C03F080530193019B284A4B
:10265000136843F480731360FDF73AFF064605E004
:10266000FDF736FF801B642800F2F184204B1B68C5
:1026700013F4807FF4D01D4B1A6F236B534013F477
:10268000407F45D0194B196F21F440701A6F42F406
:1026900080321A671A6F22F480321A67186711F0B5
:1026A000020F10D0FDF714FF064607E0FDF710FFFC
:1026B000801B41F28833984200F2CB840B4B1B6F96
:1026C00013F0020FF2D0236B03F44072B2F5407F97
:1026D00012D10648826822F4F811064A1A400A43C9
:1026E00082600EE0F9FFFF0164A800080038024094
:1026F00000700040FFFCFF0FBB4A936823F4F813FF
:102700009360B94A116F236BC3F30B030B43136739
:10271000236813F0100F17D0A36B002B18BFB3F171
:10272000807F04D04FF48071B04801F0E7F9AE4BE0
:10273000D3F88C2022F08072C3F88C20D3F88C1050
:10274000A26B0A43C3F88C20236813F4804F16D081
:10275000636E002B18BFB3F5803F07D0B3F5003F81
:1027600004D04FF48571A14801F0C8F99E49D1F811
:10277000903023F44032636E1343C1F890302368E5
:1027800013F4004F16D0A36E002B18BFB3F5802FA3
:1027900007D0B3F5002F04D04FF48A71934801F0AD
:1027A000ADF99149D1F8903023F44022A36E134340
:1027B000C1F89030236813F4803F16D0E36E002BED
:1027C00018BFB3F5801F07D0B3F5001F04D04FF436
:1027D0008F71864801F092F98349D1F8903023F443
:1027E0004012E36E1343C1F89030236813F4003FA6
:1027F00016D0236F002B18BFB3F5800F07D0B3F5A9
:10280000000F04D04FF49471784801F077F97649BD
:10281000D1F8903023F44002236F1343C1F8903075
:10282000236813F0400F14D0636C032B18BF012BE7
:1028300006D9022B04D04FF499716C4801F05EF96F
:102840006949D1F8903023F00302636C1343C1F857
:102850009030236813F0800F16D0A36C002B18BFA4
:10286000042B08D00C2B06D0082B04D04FF49E71FB
:102870005E4801F043F95C49D1F8903023F00C0236
:10288000A36C1343C1F89030236813F4807F16D0F3
:10289000E36C002B18BF102B08D0302B06D0202B58
:1028A00004D04FF4A371514801F028F94E49D1F8F2
:1028B000903023F03002E36C1343C1F8903023686A
:1028C00013F4007F16D0236D002B18BF402B08D0C7
:1028D000C02B06D0802B04D04FF4A871434801F0E0
:1028E0000DF94149D1F8903023F0C002236D134314
:1028F000C1F89030236813F4806F19D0636D002BFA
:1029000018BFB3F5807F0AD0B3F5407F07D0B3F589
:10291000007F04D04FF4AD71344801F0EFF8324934
:10292000D1F8903023F44072636D1343C1F89030B6
:10293000236813F4006F19D0A36D002B18BFB3F5F3
:10294000806F0AD0B3F5406F07D0B3F5006F04D0A5
:102950004FF4B271254801F0D1F82349D1F89030F5
:1029600023F44062A36D1343C1F89030236813F43D
:10297000805F19D0E36D002B18BFB3F5805F0AD0DC
:10298000B3F5405F07D0B3F5005F04D04FF4B771E3
:10299000164801F0B3F81449D1F8903023F44052AE
:1029A000E36D1343C1F89030236813F4005F1FD028
:1029B000236E002B18BFB3F5804F0AD0B3F5404FFC
:1029C00007D0B3F5004F04D04FF4BC71074801F0B5
:1029D00095F80549D1F8903023F44042236E134313
:1029E000C1F8903004E000BF0038024064A800083D
:1029F000236813F4800F13D0A36FB3F1806F18BF57
:102A0000002B04D04FF4C171394801F077F83949EF
:102A1000D1F8903023F08062A36F1343C1F8903057
:102A2000236813F4001F18D0E36FB3F1006F18BFD1
:102A3000002B04D04FF4C6712D4801F05FF82D49EA
:102A4000D1F8903023F00062E36F1343C1F8903067
:102A5000E36FB3F1006F00D10125236813F0080F75
:102A600000D0012513F4802F19D0636F002B18BFFD
:102A7000B3F1807F0AD0B3F1007F07D0B3F1407F7C
:102A800004D040F2A3111A4801F038F81949D1F8DE
:102A9000903023F04072636F1343C1F89030236885
:102AA00013F4000F15D0D4F88030B3F1805F18BF55
:102AB000002B04D040F2AD110D4801F01FF80D4974
:102AC000D1F8903023F08052D4F880301343C1F80D
:102AD000903027B92368B3F1007F40F07181054A37
:102AE000136823F080631360FDF7F2FC064609E0EB
:102AF00064A8000800380240FDF7EAFC801B642847
:102B000000F2A982B44B1B6813F0006FF4D1636824
:102B1000323BB3F5BF7F04D94FF4E471AF4800F006
:102B2000EDFF236813F0010F45D0636B002B42D1FA
:102B3000A368023B052B04D94FF4E771A74800F0C6
:102B4000DDFFA548D0F8846006F440364FF44032EB
:102B500092FAA2F3B3FA83F3DE40D0F8841001F0C6
:102B600070674FF0706393FAA3F1B1FA81F127FA1D
:102B700001F1676847F6C07E9EFAAEFEBEFA8EFE91
:102B800007FA0EF792FAA2F2B2FA82F206FA02F20B
:102B90003A4393FAA3F3B3FA83F301FA03F31A4324
:102BA000A3684FF0E04191FAA1F1B1FA81F18B40B5
:102BB0001343C0F88430236813F4002F03D0E26B72
:102BC000B2F5801F06D013F4801F59D0236CB3F5E3
:102BD000800F55D1E368023B0D2B04D94FF4EF7100
:102BE0007E4800F08BFF636A013B1F2B04D94FF432
:102BF000F0717A4800F082FF7748D0F8842002F420
:102C000040324FF4403E9EFAAEF3B3FA83F322FA19
:102C100003F6D0F8841001F0E0414FF0E04393FA5E
:102C2000A3F2B2FA82F2D14047F6C07797FAA7F73B
:102C3000B7FA87F7626802FA07F79EFAAEF2B2FABD
:102C400082F206FA02F247EA0206E2684FF0706783
:102C500097FAA7F7B7FA87F7BA40324393FAA3F384
:102C6000B3FA83F301FA03F31343C0F88430D0F8C6
:102C70008C3023F01F02636A013B1343C0F88C3091
:102C8000236813F0807F43D02369032B04D940F2DB
:102C9000F311524800F032FF4F4ED6F8840000F096
:102CA00070604FF0706292FAA2F3B3FA83F3D840E7
:102CB000D6F8841001F0E04E4FF0E04797FAA7F104
:102CC000B1FA81F32EFA03F1636847F6C07E9EFAEB
:102CD000AEFEBEFA8EFE03FA0EFE4FF4403393FAB8
:102CE000A3F3B3FA83FC236903FA0CF34EEA03035C
:102CF00092FAA2F2B2FA82F200FA02F21A4397FAB8
:102D0000A7F3B3FA83F301FA03F31343C6F884304D
:102D1000236813F0007F3FD02369032B04D940F2CE
:102D200002212E4800F0EAFEA368023B052B04D9DD
:102D300040F20321294800F0E1FEE368023B0D2B3D
:102D400004D94FF40171254800F0D8FE626847F6B7
:102D5000C07393FAA3F3B3FA83F39A4023694FF451
:102D6000403191FAA1F1B1FA81F18B401343E2684D
:102D70004FF0706191FAA1F1B1FA81F18A401A43E2
:102D8000A3684FF0E04191FAA1F1B1FA81F18B40D3
:102D90001343114AC2F884300F4A136843F080632A
:102DA0001360FDF795FB064605E0FDF791FB801BE0
:102DB000642800F25281084B1B6813F0006FF4D0B6
:102DC000002D00F04C81044A136823F080531360F7
:102DD000FDF77EFB054609E00038024064A80008C4
:102DE000FDF776FB401B642800F23B819F4B1B687C
:102DF00013F0005FF4D16369323BB3F5BF7F04D9B0
:102E000040F232219A4800F079FE236813F4002F33
:102E100001D0E26B2AB113F4801F59D0236C002B30
:102E200056D1A369023B0D2B04D940F239219048B9
:102E300000F064FEA36A013B1F2B04D940F23B2142
:102E40008B4800F05BFE8948D0F8885005F4403587
:102E50004FF4403292FAA2F3B3FA83F3DD40D0F894
:102E6000881001F0E0464FF0E04393FAA3F1B1FA85
:102E700081F126FA01F1676947F6C07696FAA6F65F
:102E8000B6FA86F607FA06F692FAA2F2B2FA82F2D9
:102E900005FA02F246EA0205A2694FF0706696FA58
:102EA000A6F6B6FA86F6B2402A4393FAA3F3B3FA2B
:102EB00083F301FA03F31343C0F88830D0F88C3061
:102EC00023F4F853A26A013A43EA0223C0F88C3093
:102ED000236813F4001F45D0E36FB3F1006F41D1B5
:102EE000236A032B04D940F24E21614800F006FE0C
:102EF0005E4ED6F8880000F070604FF0706292FA73
:102F0000A2F3B3FA83F3D840D6F8881001F0E04179
:102F10004FF0E04595FAA5F3B3FA83F3D94067691A
:102F200047F6C07393FAA3F3B3FA83F307FA03FEE9
:102F3000236A4FF4403797FAA7F7B7FA87F7BB40F1
:102F40004EEA030392FAA2F2B2FA82F200FA02F215
:102F50001A4395FAA5F3B3FA83F301FA03F3134383
:102F6000C6F88830236813F0080F5BD0E369023B92
:102F7000052B04D940F25D213D4800F0BFFDE36A16
:102F8000002B18BFB3F5803F0AD0B3F5003F07D040
:102F9000B3F5403F04D040F25E21354800F0AEFD6D
:102FA000324DD5F8882002F070624FF0706191FACE
:102FB000A1F3B3FA83F322FA03F6D5F8883003F4C9
:102FC00040334FF4403090FAA0F2B2FA82F223FA82
:102FD00002F2676947F6C07393FAA3F3B3FA83F377
:102FE0009F4090FAA0F3B3FA83F302FA03F33B4352
:102FF00091FAA1F2B2FA82F206FA02F21343E269FE
:103000004FF0E04191FAA1F1B1FA81F18A40134306
:10301000C5F88830D5F88C3023F44032E36A134386
:10302000C5F88C30114A136843F080531360FDF7E4
:103030004FFA044604E0FDF74BFA001B642812D84F
:103040000A4B1B6813F0005FF5D000200CE0032052
:103050000AE0032008E0032006E0032004E000204B
:1030600002E0032000E0032003B0F0BD003802407E
:1030700064A800082DE9F04105460F4616461C4697
:10308000FDF726FA804637E0B4F1FF3F34D02CB18B
:10309000FDF71EFAC8EB000084422DD82A68536859
:1030A00023F0E00353606B68B3F5827F0BD1AB680C
:1030B000B3F5806F18BFB3F5004F04D12A681368C9
:1030C00023F040031360AB6AB3F5005F0BD12A68AD
:1030D000136823F400531B041B0C13602A68136845
:1030E00043F400531360012385F85D30002385F815
:1030F0005C300320BDE8F0812B689B683B40B34205
:10310000C2D10020BDE8F0812DE9F04182B0074630
:103110000D4614461E46FDF7DBF9804641E0B5F545
:10312000C06F08BF002C05D1137BDBB28DF80730D0
:103130009DF80730B6F1FF3F33D02EB1FDF7C8F947
:10314000C8EB000086422CD83A68536823F0E003AD
:1031500053607B68B3F5827F0BD1BB68B3F5806F9A
:1031600018BFB3F5004F04D13A68136823F0400349
:103170001360BB6AB3F5005F0BD13A68136823F4A0
:1031800000531B041B0C13603A68136843F400538C
:103190001360012387F85D30002387F85C3003203B
:1031A00005E03A6893682B40A342B8D1002002B0F2
:1031B000BDE8F08138B504460D460B4600224FF4B9
:1031C000C051FFF7A1FF28B1236E43F0200323660F
:1031D00003231AE02B46002280212046FFF74AFFF6
:1031E00028B1236E43F02003236603230DE02B4612
:1031F00000224FF4C0612046FFF786FF034620B14E
:10320000236E43F0200323660323184638BD00BF16
:10321000704700BF002800F0228110B50446036803
:10322000904A91498B4218BF934213D002F58062B5
:1032300093420FD002F5784293420BD002F5E05250
:10324000934207D002F58062934203D0CC21874895
:1032500000F054FC6368002B18BFB3F5827F03D0E5
:10326000CD21824800F04AFCA368002B18BFB3F5BB
:10327000806F06D0B3F5004F03D0CE217B4800F01D
:103280003DFCE368B3F5706F18BFB3F5606F24D0F1
:10329000B3F5506F21D0B3F5406F1ED0B3F5306F4A
:1032A0001BD0B3F5206F18D0B3F5106F15D0B3F560
:1032B000006F12D0B3F5E06F0FD0B3F5C06F0CD034
:1032C000B3F5A06F09D0B3F5806F06D0B3F5407F9A
:1032D00003D0CF21654800F011FC2369002B18BFF3
:1032E000022B03D0D021614800F008FC6369012B58
:1032F00003D9D1215D4800F001FCA369B3F5007F3B
:1033000018BF002B06D0B3F5802F03D0D221574829
:1033100000F0F4FB636B082B18BF002B03D0D32104
:10332000524800F0EBFBE369002B18BF082B0FD0CD
:10333000102B0DD0182B0BD0202B09D0282B07D009
:10334000302B05D0382B03D0D421484800F0D6FBD1
:10335000236A002B18BF802B03D0D521434800F0EF
:10336000CDFB636A002B18BF102B03D0D6213F483A
:1033700000F0C4FBA36A002B18BFB3F5005F03D0B5
:10338000D7213A4800F0BAFBE36A013B4FF6FE72E0
:10339000934203D9D821354800F0B0FB236B022BB0
:1033A00003D9D921314800F0A9FB94F85D3023B945
:1033B00084F85C302046FFF72BFF022384F85D3051
:1033C0002268136823F040031360E268B2F5E06FEF
:1033D00001D9002001E04FF48050B2F5706F18BFA2
:1033E000B2F5E06F01D00023A362236B3BB9B2F5C5
:1033F000E06F02D90223236301E0012323632168E4
:103400006268A3681A4323691A4363691343A26974
:1034100002F400721A43E3691A43236A1A43A36A47
:1034200013430B60236B022B04D12268136843F40F
:10343000006313602168638B03F00403626A134323
:10344000626B1A43E368134303434B602368E26AE9
:103450001A6100202066012384F85D3010BD012030
:10346000704700BF003800400030014098A80008B5
:10347000F0B583B004460F4616461D468368002B00
:1034800018BFB3F5004F04D04FF4CC71664800F07C
:1034900035FB94F85C30012B00F0BD80012384F8EB
:1034A0005C3094F85D30012B07D0012384F85D3047
:1034B000002384F85C300223B2E0002E18BF002FF6
:1034C00006D1012384F85D30002284F85C20A7E057
:1034D000032384F85D3000232366A763A687E6876D
:1034E0002364A4F84430A4F84630A368B3F5004F31
:1034F00004D12268136843F480431360A36AB3F5D0
:10350000005F0BD12268136823F400531B041B0CCB
:1035100013602268136843F40053136023681A6829
:1035200012F0400F03D11A6842F040021A60E368BB
:10353000B3F5E06F19D849E02B4602221146204628
:10354000FFF798FD38B1012384F85D30002384F83B
:103550005C30032364E02368A26B1288DA60A36BFB
:103560000233A363E38F013BE387E38F002BE3D1B7
:103570002FE0012B19D02B46022211462046FFF7DF
:1035800079FD38B1012384F85D30002384F85C3084
:10359000032345E02368A26B1288DA60A36B023331
:1035A000A363E38F023BE38710E02B460222114620
:1035B0002046FFF75FFD00282FD12268A36B591C1E
:1035C000A1631B781373E38F013BE387E38F002B29
:1035D000CFD1A36AB3F5005F04D12268136843F426
:1035E0008053136029462046FFF7E4FD0346B0B937
:1035F000A26832B901922268D16801919268019261
:10360000019A012284F85D20002284F85C20226E59
:1036100032B1012304E0022302E0032300E003238C
:10362000184603B0F0BD00BF98A80008704700BF5F
:1036300010B504460368234A934218BFB3F1804F84
:1036400034D0A2F57C42934230D002F5806293429E
:103650002CD002F58062934228D002F5806293421A
:1036600024D002F58062934220D002F5704293424A
:103670001CD002F57052934218D002F5806293423A
:1036800014D002F58062934210D0A2F59832934292
:103690000CD002F58062934208D002F5806293421A
:1036A00004D040F25D11084800F028FA2268D3687F
:1036B00043F00103D3602268136843F001031360F1
:1036C000002010BD00000140C8A80008704700BFDE
:1036D000704700BF704700BF704700BF10B5044679
:1036E00003681A6912F0020F17D0DA6812F0020F9D
:1036F00013D06FF002021A610123037603689B69FD
:1037000013F0030F02D0FFF7E3FF04E0FFF7DEFF43
:103710002046FFF7DFFF0023237623681A6912F0A3
:10372000040F19D0DA6812F0040F15D06FF00402FC
:103730001A610223237623689B6913F4407F03D028
:103740002046FFF7C5FF05E02046FFF7BFFF2046F4
:10375000FFF7C0FF0023237623681A6912F0080FD1
:1037600019D0DA6812F0080F15D06FF008021A614C
:10377000042323762368DB6913F0030F03D020466C
:10378000FFF7A6FF05E02046FFF7A0FF2046FFF762
:10379000A1FF0023237623681A6912F0100F19D0B5
:1037A000DA6812F0100F15D06FF010021A610823BA
:1037B00023762368DB6913F4407F03D02046FFF7AC
:1037C00087FF05E02046FFF781FF2046FFF782FFD5
:1037D0000023237623681A6912F0010F09D0DA68F2
:1037E00012F0010F05D06FF001021A61204604F0BB
:1037F00079F823681A6912F0800F09D0DA6812F09C
:10380000800F05D06FF080021A61204600F03EF96B
:1038100023681A6912F4807F09D0DA6812F0800FE9
:1038200005D06FF080021A61204600F02FF923685E
:103830001A6912F0400F09D0DA6812F0400F05D073
:103840006FF040021A612046FFF746FF23681A69AD
:1038500012F0200F09D0DA6812F0200F05D06FF0B7
:1038600020021A61204600F00FF910BD70B4026802
:10387000434B984214BF00230123B0F1804F14BF83
:103880001C4643F00104BCB93E4DA84214BF0025BC
:1038900001253D4EB04211D085B905F1804505F5B1
:1038A0008235A84214BF0025012506F50066B04206
:1038B00000D02DB1012504E0012502E0012500E042
:1038C00000251DB122F070024D682A43002C35D12D
:1038D0002C4CA04214BF002401242B4DA8422FD011
:1038E00074BB04F1804404F58234A04214BF002468
:1038F000012405F50065A84224D01CBB234CA0423E
:1039000014BF0024012405F59A35A8421CD0DCB967
:103910001F4CA04214BF0024012405F50065A842F5
:1039200014D09CB91B4CA04214BF00240124A5F55F
:103930009635A84200D05CB101240AE0012408E0D9
:10394000012406E0012404E0012402E0012400E057
:1039500000241CB122F44072CC68224302608A68C1
:10396000C2620A6882620C4A904208BF43F00103B7
:103970000BB10B6903630123436170BC704700BF47
:1039800000000140000800400004004000440140E5
:1039900000180040002000400004014000286CD0C6
:1039A00010B504460368364A934218BFB3F1804FFE
:1039B00033D0A2F57C4293422FD002F5806293422D
:1039C0002BD002F58062934227D002F580629342A9
:1039D00023D002F5806293421FD002F570429342D9
:1039E0001BD002F57052934217D002F580629342C9
:1039F00013D002F5806293420FD0A2F59832934221
:103A00000BD002F58062934207D002F580629342A8
:103A100003D0D2211B4800F071F8A368002B18BF17
:103A2000102B09D0202B07D0402B05D0602B03D0C2
:103A3000D321144800F062F82369002B18BFB3F5B6
:103A4000807F06D0B3F5007F03D0D4210D4800F06D
:103A500055F894F8393013F0FF0F02D12046FFF7E4
:103A6000E5FD022384F83930211D2068FFF7FEFEB2
:103A7000012384F83930002010BD0120704700BFB9
:103A800000000140C8A80008704700BF704700BF91
:103A9000FEE700BF08B5034800F05CF80120FFF71F
:103AA000F7FF00BFF8A8000808B50D4B1B6813B955
:103AB0000C4A0B4B1A600A4B1A68C31C23F0030311
:103AC000134409498B4206D905F09AFE0C23036082
:103AD0004FF0FF3008BD02490B60104608BD00BF23
:103AE000F8040020D849002000FC042001230360D2
:103AF000014B0B60704700BF0400002008B50A4668
:103B00000146024800F004F8FFF7C4FF4CA9000882
:103B10000FB480B582B000AF07F114033B603B687F
:103B20003A6980210A4806F073F878607B68002BB8
:103B300005DD7B681946064800F056F878607B681A
:103B400018460837BD46BDE8804004B0704700BF46
:103B50000005002080B582B000AF7860786805F07D
:103B6000AFFF03461946786800F03EF8012104488B
:103B700000F03AF8034618460837BD4680BD00BF3E
:103B800078A900082DE9F04385B004460F46435656
:103B900013BB042528462146ABBE04461FE035462C
:103BA000102E28BF1025002306E014F9011B04AADB
:103BB0001A4402F8101C0133AB42F6D304AA134492
:103BC000002203F8102CE9464FF00408404649460D
:103BD000ABBE8046761B00E00E46002EDFD1384695
:103BE00005B0BDE8F08300BF08B5FFF7CBFF08BD07
:103BF00008B500F097F8054B054A9A60D3F888207D
:103C000042F47002C3F8882008BD00BF00ED00E058
:103C100000000008F8B504460D4617461E46264823
:103C2000FFF776FF21682548FFF772FF6168244897
:103C3000FFF76EFFA1682348FFF76AFFE16822489B
:103C4000FFF766FF21692148FFF762FF616920489D
:103C5000FFF75EFFA1691F48FFF75AFFE1691E48A1
:103C6000FFF756FF1D48FFF753FF29461C48FFF793
:103C70004FFF1C4CE16A1C48FFF74AFF216B1B48B1
:103C8000FFF746FFE16B1A48FFF742FF15F0800F80
:103C900003D039461748FFF73BFF15F4004F03D018
:103CA00031461548FFF734FF1448FFF731FF0699F6
:103CB0001348FFF72DFFF8BDA8A90008B8A9000810
:103CC000C8A90008D8A90008E8A90008F8A90008B0
:103CD00008AA000818AA000828AA000838AA00089C
:103CE00044AA000800ED00E054AA000864AA0008F5
:103CF00074AA000884AA000894AA0008A4AA0008CC
:103D0000ACAA000883691A888A4207D10268033A7C
:103D1000012A05D8023383610120704700207047D3
:103D20000020704710B40F4AD2F8883043F4700373
:103D3000C2F888300C4B196841F00101196000206D
:103D400098601C680949214019600949596019683F
:103D500021F480211960D8604FF0006393605DF812
:103D6000044B704700ED00E000380240FFFFF6FE14
:103D700010300024224B9B6803F00C03042B07D067
:103D8000082B09D0002B2DD11E4A1F4B1A602CE0A6
:103D90001E4A1D4B1A6028E0194B5A685B6803F0F5
:103DA0003F0312F4800F09D0184AB2FBF3F2144B10
:103DB0005B68C3F3881303FB02F208E0114AB2FB0D
:103DC000F3F30F4A5168C1F3881101FB03F20C4B66
:103DD0005B68C3F3014301335B00B2FBF3F30A4AB0
:103DE000136002E0074A084B1A60054B9B68C3F357
:103DF0000313074AD15C044A1368CB401360704731
:103E0000003802400024F4000C00002080BA8C012D
:103E1000F0AA00082DE9F84305468946164698465B
:103E2000BDF82070044607E03B464246494620461E
:103E300000F026FB013424B2AB199C42F4DBBDE850
:103E4000F88300BF00B583B0064BB3F90030064AD3
:103E5000B2F9002000900021084600F0C5FB03B035
:103E60005DF804FB360C0020300C00202DE9F04FEB
:103E700089B00D4604911E460593BDF94840BDF931
:103E80004CB0BDF850700097994204DD049605953A
:103E9000034610461A46059B5B4505DDCDF814B078
:103EA0009B46134622461C46049B059EB34204DDF6
:103EB00004960593034610461A46049B5B4518D1A9
:103EC000904205DC01DB024602E01346024618463A
:103ED000944205DB844201DC144601E0204614468E
:103EE000001B421C009B12B20499204600F022FBEA
:103EF0007CE01FFA82FA87B2C7EB0A039BB20293F7
:103F0000059883B2BDF81080C8EB030212B2964642
:103F1000A4B2C7EB04091FFA89F91FFA8BF2C8EBA8
:103F200002080FFA88F8CAEB0404A1B20191D21A70
:103F300012B20392584502D0013B1BB200E0059B30
:103F4000049C00252E46CDF818A09A46CDF81CB04A
:103F5000F3461AE096FBFBF23A4412B295FBF8F0F6
:103F6000384400B2029B1E4436B24D442DB2824208
:103F700002DC034610461A46121A0132009B12B2A6
:103F8000214600F0D7FA013424B25445E2DDDDF8D1
:103F900018A0DDF81CB0059BE51ABDF8043015FB30
:103FA00003F52DB2049BE61A16FB09F636B21BE0A8
:103FB000039B95FBF3F2524412B296FBF8F038449F
:103FC00000B2019B1D442DB24E4436B2824202DC47
:103FD000034610461A46121A0132009B12B22146BD
:103FE00000F0A8FA013424B2A345E1DA09B0BDE833
:103FF000F08F00BF2DE9F04784B090461E46BDF912
:104000003070BDF8345080B289B2CB19013B8219AF
:10401000013A9BB292B200F0D7F9184B012299886D
:104020001868FDF70FF9164BD3F80090B3F804A009
:10403000002251464846FDF705F9002411E038F802
:10404000143003EA0502120A8DF804202B408DF883
:1040500005300123022201A90A48FFF709FA0134B9
:1040600024B207FB06F39C42E9DB01225146484695
:10407000FDF7E8F804B0BDE8F08700BF90AB00089A
:1040800098AB0008880B002008B90120FFE7014B1E
:1040900018707047350C0020024B1880024B1980B5
:1040A000704700BFD20C0020D00C0020014B1870CC
:1040B000704700BF340C002070B50646104B00223C
:1040C00099881868FDF7BEF80E4B00229988186889
:1040D000FDF7B8F80C4B1C689D8800222946204645
:1040E000FDF7B0F809490E8001231A460848FFF78A
:1040F000BFF9012229462046FDF7A4F870BD00BF94
:1041000090AB000888AB000898AB0008D40C0020E6
:10411000880B002070B50646104B0122998818685C
:10412000FDF790F80E4B002299881868FDF78AF881
:104130000C4B1C689D88002229462046FDF782F81A
:1041400009490E8001231A460848FFF791F9012218
:1041500029462046FDF776F870BD00BF90AB0008F9
:1041600088AB000898AB0008D40C0020880B002016
:1041700038B5934B1C689D88012229462046FDF7DF
:1041800061F8052000F038FD002229462046FDF7A1
:1041900059F8142000F030FD012229462046FDF791
:1041A00051F8962000F028FD864B00229988186867
:1041B000FDF748F8EF20FFF77FFF0320FFF7AAFF86
:1041C0008020FFF7A7FF0220FFF7A4FFCF20FFF713
:1041D00073FF0020FFF79EFFC120FFF79BFF3020F9
:1041E000FFF798FFED20FFF767FF6420FFF792FFCE
:1041F0000320FFF78FFF1220FFF78CFF8120FFF7CE
:1042000089FFE820FFF758FF8520FFF783FF002094
:10421000FFF780FF7820FFF77DFFCB20FFF74CFFF3
:104220003920FFF777FF2C20FFF774FF0020FFF7FE
:1042300071FF3420FFF76EFF0220FFF76BFFF720BE
:10424000FFF73AFF2020FFF765FFEA20FFF734FF72
:104250000020FFF75FFF0020FFF75CFFC020FFF7A3
:104260002BFF2320FFF756FFC120FFF725FF10206B
:10427000FFF750FFC520FFF71FFF3E20FFF74AFF63
:104280002820FFF747FFC720FFF716FF8620FFF71C
:1042900041FF3620FFF710FF4820FFF73BFF3A2091
:1042A000FFF70AFF5520FFF735FFB120FFF704FFA6
:1042B0000020FFF72FFF1820FFF72CFFB620FFF795
:1042C000FBFE0820FFF726FF8220FFF723FF2720B1
:1042D000FFF720FFF220FFF7EFFE0020FFF71AFFA5
:1042E0002620FFF7E9FE0120FFF714FFE020FFF78B
:1042F000E3FE0F20FFF70EFF3120FFF70BFF2B200F
:10430000FFF708FF0C20FFF705FF0E20FFF702FF65
:104310000820FFF7FFFE4E20FFF7FCFEF120FFF71D
:10432000F9FE3720FFF7F6FE0720FFF7F3FE102017
:10433000FFF7F0FE0320FFF7EDFE0E20FFF7EAFE89
:104340000920FFF7E7FE0020FFF7E4FEE120FFF77A
:10435000B3FE0020FFF7DEFE0E20FFF7DBFE142089
:10436000FFF7D8FE0320FFF7D5FE1120FFF7D2FE9E
:104370000720FFF7CFFE3120FFF7CCFEC120FFF76B
:10438000C9FE4820FFF7C6FE0820FFF7C3FE0F2036
:10439000FFF7C0FE0C20FFF7BDFE3120FFF7BAFE8D
:1043A0003620FFF7B7FE0F20FFF7B4FE1120FFF70E
:1043B00083FE782000F020FC2920FFF77DFE38BD29
:1043C00018AB000898AB0008F8B507460D4616462E
:1043D0001C462A20FFF770FE380AFFF79BFEF8B252
:1043E000FFF798FE300AFFF795FEF0B2FFF792FE56
:1043F0002B20FFF761FE280AFFF78CFE2846FFF707
:1044000089FE200AFFF786FE2046FFF783FE2C2058
:10441000FFF752FEF8BD00BFF0B599B00446134B4C
:10442000012299881868FCF70DFF114B1D689E88C2
:10443000002231462846FCF705FF0E4B1C800E4C2F
:104440000127179716930D4B1593542204F1100171
:10445000684605F0DBF994E80F0003F0BFFA3A462E
:1044600031462846FCF7EEFE19B0F0BD90AB0008CF
:1044700098AB0008D40C0020880B0020D80C00203A
:104480002DE9F04198B01E46234BB3F9003083422A
:104490003FDD1446214BB3F900308B4239DD8A18D9
:1044A000013A9A4201DB5C1A24B280B289B20B193C
:1044B000013B9BB20246FFF787FF194B0122998807
:1044C0001868FCF7BFFE174B1F68B3F80480002282
:1044D00041463846FCF7B6FE12E0134B1E80134CE3
:1044E000012217921693124B1593542204F11001D6
:1044F000684605F08BF994E80F0003F06FFA2C463C
:10450000631E1DB2002CE8D1012241463846FCF75B
:1045100099FE18B0BDE8F081300C0020360C002068
:1045200090AB000898AB0008D40C0020880B00204A
:10453000D80C00202DE9F04198B01E46234BB3F96A
:10454000003083423FDD1446214AB2F900208A42FE
:1045500039DD0219013A9A4201DB1C1A24B280B2F9
:1045600089B20219013A0B4692B2FFF72DFF194B9F
:10457000012299881868FCF765FE174B1F68B3F88D
:104580000480002241463846FCF75CFE12E0134BE3
:104590001E80134C012217921693124B159354222E
:1045A00004F11001684605F031F994E80F0003F0BA
:1045B00015FA2C46631E1DB2002CE8D1012241469B
:1045C0003846FCF73FFE18B0BDE8F081300C002003
:1045D000360C002090AB000898AB0008D40C0020EB
:1045E000880B0020D80C00202DE9F04798B01F461A
:1045F000BDF880602C4BB3F90030834250DD90460B
:104600002A4AB2F900208A424ADD00EB0804013C44
:104610009C4202DB1B1A0FFA83F8CB19013B934231
:1046200001DB571A3FB280B289B2CB19013B00EBD4
:104630000802013A9BB292B2FFF7C6FE1C4B012260
:1046400099881868FCF7FEFD1A4BD3F80090B3F870
:1046500004A0002251464846FCF7F4FD19E0164A32
:104660001680164C012317931692154B159354225E
:1046700004F11001684605F0C9F894E80F0003F052
:10468000ADF9013D2DB200E04546002DE7DC013FCC
:104690003FB2002FF8DC012251464846FCF7D2FD1C
:1046A00018B0BDE8F08700BF300C0020360C0020A9
:1046B00090AB000898AB0008D40C0020880B0020B9
:1046C000D80C002010B504463720FFF7F5FC200A6F
:1046D000FFF720FDE0B2FFF71DFD10BD43181344A6
:1046E000B3F5A07F19D170B514460D4606463320A8
:1046F000FFF7E2FC300AFFF70DFDF0B2FFF70AFD0D
:10470000280AFFF707FDE8B2FFF704FD200AFFF7CC
:1047100001FDE0B2FFF7FEFC70BD704710B5044626
:104720003620FFF7C9FC04F0030003282ED8DFE889
:1047300000F0020D18234820FFF7ECFCF022144B88
:104740001A804FF4A072134B1A8010BD2820FFF777
:10475000E1FC4FF4A0720E4B1A80F0220D4B1A8030
:1047600010BD8820FFF7D6FCF022094B1A804FF4C9
:10477000A072084B1A8010BDE820FFF7CBFC4FF465
:10478000A072034B1A80F022024B1A8010BD00BFAA
:10479000300C0020360C002030B587B00C4A136B6B
:1047A00043F0100313634FF4005501950123029366
:1047B000022204920393074C01A92046FCF7AEFBAA
:1047C000002229462046FCF73DFD07B030BD00BF62
:1047D00000380240001002400A4B1B680A4AA2FB44
:1047E00003239B09013BB3F1807F09D2074A536041
:1047F000F021074B83F823100023936007231360F5
:10480000704700BF0C000020D34D621010E000E0A4
:1048100000ED00E0034B1B681BB1024A1368013B2B
:1048200013607047EC0C002030B595B00024019463
:10483000234B1A6C42F080521A641B6C03F08053B5
:104840000193019B02941F4B1A6842F440421A6084
:104850001B6803F440430293029B012308934FF427
:10486000803309934FF480030F931A2310934FF46E
:10487000D873119302251295082313930E9508A857
:10488000FDF798F9FDF754F90F2303930495059468
:104890004FF4A05306934FF480530793062103A8C7
:1048A000FDF746FCFDF736FE074BA3FB0030800901
:1048B000FCF70CFA0420FCF71FFA15B030BD00BF5E
:1048C0000038024000700040D34D621010B5BFF3B5
:1048D0004F8FBFF36F8F1D4B0021C3F850125A69E1
:1048E00042F400325A61BFF34F8FBFF36F8FC3F8AA
:1048F0008410BFF34F8FD3F88040C4F34E3000E0F4
:104900001846C4F3C90200E01A4643F6E07303EA0E
:10491000401343EA82730D49C1F86032531E002AE6
:10492000F2D1431E0028EBD1BFF34F8F4B6943F404
:1049300080334B61BFF34F8FBFF36F8FFBF7B4FD35
:10494000FFF772FFFFF716FA10BD00BF00ED00E0A1
:1049500010B586B00022684B1A80684B1A80684BED
:104960001A706421674B1980674B1A70674B1A7075
:104970000092674B596C41F480715964596C01F491
:104980008071009100990192596C41F40071596451
:10499000596C01F40071019101990292596C41F432
:1049A00080615964596C01F480610291029903920B
:1049B000196B41F001011963196B01F001010391B9
:1049C00003990492196B41F002011963196B01F00C
:1049D0000201049104990592196B41F004011963D5
:1049E000196B01F0040105910599596A41F4807130
:1049F0005962596A21F4807159624648A3F58C3393
:104A000003604FF48033436082600261012383615D
:104A100002624262C2628262C260C3610263426138
:104A2000FBF708FE18B1394A1378013313703A487E
:104A30003A4B03604FF4803343600023836003618B
:104A40000122826103624362C3628362C360C26106
:104A500003634361FBF7EEFD18B12C4A1378013371
:104A600013702F482F4B03604FF4803343600023B3
:104A7000836003610122826103624362C3628362D5
:104A8000C360C26103634361FBF7D4FD18B11F4AE1
:104A9000137801331370244909230B6001234B6001
:104AA0008B600020C860214A032414605360936027
:104AB000D0601F4A0224146053609360D060154890
:104AC000FBF79EFF18B1114A137801331370174991
:104AD0001148FBF795FF18B10C4A13780133137096
:104AE00013490F48FBF78CFF18B1084A13780133BC
:104AF000137006B010BD00BF140A00202C0B00205C
:104B0000F10B0020380C0020810B0020800B0020CE
:104B1000003802409C0A0020E40A002000210140E5
:104B2000780C002000220140180A0020C00C002050
:104B3000700B002008B564211848FBF701FF6421C1
:104B40001748FBF7FDFE64211648FBF7F9FE18BB7A
:104B50001248FCF745F810F4007F1DD01048FCF710
:104B60003FF810F4007F17D00E48FCF739F810F426
:104B7000007F11D00948FBF73FFF80B20A4B188035
:104B80000748FBF739FF80B2084B18800548FBF750
:104B900033FF80B2064B188008BD00BF9C0A00207E
:104BA000E40A0020780C0020140A00202C0B0020BE
:104BB000EE0B002008B50C48FBF728FE18B10B4A95
:104BC0001378013313700A48FBF720FE18B1074A27
:104BD0001378013313700748FBF718FE18B1034A26
:104BE00013780133137008BD9C0A0020800B00204D
:104BF000E40A0020780C0020034B1860024B1B686D
:104C0000002BFBD1704700BF300B00202DE9F04F87
:104C100087B0802301934FF00208CDF81080012562
:104C2000029500240594039401A9B948FCF776F98C
:104C30004FF0400ACDF804A0CDF8108002950594FD
:104C4000039401A9B248FCF769F94FF400530193AA
:104C50000494112702970594039401A9AD48FCF729
:104C60005DF922464FF40051AA48FCF7EBFA019592
:104C7000CDF8108002940395059401A9A648FCF78D
:104C80004DF9CDF80480CDF8108002940395059479
:104C900001A9A148FCF742F94FF400730193CDF844
:104CA000108002940395059401A99948FCF736F900
:104CB0004FF0040BCDF804B04FF00309CDF8089085
:104CC00003940DEB0B019548FCF728F90826019693
:104CD000CDF8089003940DEB0B019048FCF71EF9FA
:104CE00030230193CDF8089003940DEB0B018B4812
:104CF000FCF714F9CDF804B00295049403940DEB7D
:104D00000B018348FCF70AF92A4659468048FCF70C
:104D100099FA802301930295049403940DEB0B01FF
:104D20007E48FCF7FBF8224680217C48FCF78AFA93
:104D3000CDF804800295049403940DEB0B017548A3
:104D4000FCF7ECF8224641467248FCF77BFACDF8B6
:104D500004A00295049403940DEB0B016F48FCF73B
:104D6000DDF82A4651466D48FCF76CFA019502952C
:104D7000049403940DEB0B016848FCF7CFF822462E
:104D800029466648FCF75EFACDF804A00295049423
:104D900003940DEB0B016048FCF7C0F82A4651461E
:104DA0005D48FCF74FFA01960297049403940DEBCB
:104DB0000B015948FCF7B2F8224631465648FCF739
:104DC00041FA4FF4004301930295049403940DEBD0
:104DD0000B014F48FCF7A2F82A464FF400414C481B
:104DE000FCF730FA4FF400530193029504940394B6
:104DF0000DEB0B014648FCF791F82A464FF40051A1
:104E00004348FCF71FFA202301930295049403946E
:104E10000DEB0B014048FCF781F82A4620213E4863
:104E2000FCF710FA102701970295049403940DEBF8
:104E30000B013948FCF772F82A4639463648FCF728
:104E400001FA4FF4006701970295049403940DEB67
:104E50000B013348FCF762F82A4639463048FCF724
:104E6000F1F94FF4804701970295049403940DEBF8
:104E70000B012948FCF752F82A4639462648FCF728
:104E8000E1F94FF480530193CDF808900494039412
:104E90000DEB0B012248FCF741F822464FF48051FC
:104EA0001F48FCF7CFF9CDF80480CDF808900494A2
:104EB00003940DEB0B011648FCF730F84FF48068B3
:104EC000CDF804800295049403940DEB0B01144873
:104ED000FCF724F82A4641461148FCF7B3F901973C
:104EE0000295049403940DEB0B010D48FCF716F8A2
:104EF0002A4639460A48FCF7A5F920230193029473
:104F0000049403950DEB0B010548FCF707F809E045
:104F1000000402400008024000100240000002406D
:104F2000000C0240CDF804A00294049403950DEB0C
:104F30000B015F48FBF7F2FF01960294049403957E
:104F40000DEB0B015A48FBF7E9FF80230193029414
:104F5000049403950DEB0B015548FBF7DFFF4FF46D
:104F6000005301930295049403940DEB0B015148F7
:104F7000FBF7D4FF22464FF400514E48FCF762F98C
:104F80004FF48079CDF804900494029503950DEBCD
:104F90000B014948FBF7C2FF224649464648FCF749
:104FA00051F94FF4004301930494029503940DEBDF
:104FB0000B014048FBF7B2FF2A464FF400413D4841
:104FC000FCF740F9802301930494029403940DEBC1
:104FD0000B013848FBF7A2FFCDF804B0049402950A
:104FE00003940DEB0B013548FBF798FF2A46594611
:104FF0003248FCF727F9CDF8048004940295039415
:105000000DEB0B012B48FBF789FF2A464146294847
:10501000FCF718F9CDF804900494029503940DEB75
:105020000B012348FBF77AFF224649462048FCF74C
:1050300009F901960494029503940DEB0B011F48A6
:10504000FBF76CFF224631461C48FCF7FBF8CDF815
:1050500004900494029503940DEB0B011548FBF7A3
:105060005DFF224631461348FCF7ECF8CDF804B05A
:105070000494029503940DEB0B010E48FBF74EFFD1
:10508000224659460B48FCF7DDF8CDF8049004940D
:10509000029503940DEB0B010948FBF73FFF2A46ED
:1050A00049460748FCF7CEF807B0BDE8F08F00BFCF
:1050B000000C0240001002400000024000080240C4
:1050C00000040240F0B587B00E4B9A880192022787
:1050D00004971226029601250395042405940DEBEE
:1050E00004011868FBF71AFF074B9A88019204978E
:1050F0000296039505940DEB04011868FBF70EFF6B
:1051000007B0F0BDF0AB000838AB000800B585B0C3
:105110008DF80C008DF80D1064230093022303AA70
:10512000E0210348FCF704FB05B05DF804FB00BF79
:10513000F40B0020F8B51E4603FB0121CC01B4FBA3
:10514000F3F4A4F50074D201B2FBF3F703FB1727C5
:10515000C5B2E1B22846FFF7D9FF681CC4F30721A6
:10516000C0B2FFF7D3FFC4F3014101EB8701A81CD4
:10517000C9B2C0B2FFF7CAFFE81CC7F38711C0B2BB
:10518000FFF7C4FF281DC7F38731C0B2FFF7BEFF8A
:10519000681DC7F38751C0B2FFF7B8FFA81DF1B271
:1051A000C0B2FFF7B3FFE81DC6F30721C0B2FFF797
:1051B000ADFF05F10800C6F30741C0B2FFF7A6FF37
:1051C00005F10900C6F30561C0B2FFF79FFFF8BD06
:1051D00030B587B08DF80F0000238DF817300B4CD9
:1051E0006425009501230DF10F02E0212046FCF714
:1051F0009FFA009501230DF11702E0212046FCF7EC
:1052000043FB9DF8170007B030BD00BFF40B002032
:1052100070B50E4900EB40028B188D5C5E789C786F
:1052200094B10146FF2C04D131462846FFF76EFFAA
:1052300070BD2846FFF7CCFF20EA0400C1B234401D
:1052400021432846FFF762FF70BD00BF1800002011
:1052500010B51021E620FFF759FFE521F120FFF7F7
:1052600055FF002403E02046FFF7D2FF0134B4F5D8
:10527000AF7FF8DB0121DA20FFF7AAFF00F004007E
:10528000C0B206E00121DA20FFF7A2FF00F004001F
:10529000C0B20028F6D101213120FFF799FF00F0BC
:1052A0007F013120FFF732FF0221F620FFF72EFFAA
:1052B0006521F120FFF72AFF0121DA20FFF788FF9F
:1052C00000F0150005E00121DA20FFF781FF00F072
:1052D00015000028F7D10121EB20FFF779FF0146E7
:1052E0002D20FFF713FF0121EC20FFF771FF01468E
:1052F0002E20FFF70BFF01212F20FFF769FF044647
:105300000121ED20FFF764FF24F0030100F003000A
:105310000143C9B22F20FFF7F9FE01213120FFF729
:1053200057FF60F07F01C9B23120FFF7EFFE002187
:10533000E620FFF7EBFEC1211F20FFF7E7FE40F25A
:10534000BF2340F2B922C9213520FFF7F3FEC02167
:105350001F20FFF7DBFE10BD2DE9F0414400124B8A
:105360009C421ED9114B9C421BD8114BD3E90067BC
:10537000002522462B463046394604F0B5F88046D3
:1053800022462B463046394604F0AEF801E052087A
:105390006408084B9C42FAD8234641463520FFF763
:1053A000C9FEBDE8F08100BF3F4B4C008093DC1488
:1053B00010000020A086010010B4BFF34F8FBFF390
:1053C0006F8F1B4B0021C3F850125A6942F4003210
:1053D0005A61BFF34F8FBFF36F8FC3F88410BFF3D1
:1053E0004F8FD3F88040C4F34E3000E01846C4F32A
:1053F000C90200E01A4643F6E07303EA401343EAA9
:1054000082730B49C1F86032531E002AF2D1431E49
:105410000028EBD1BFF34F8F4B6943F480334B61CE
:10542000BFF34F8FBFF36F8F5DF8044B704700BF22
:1054300000ED00E0022956DC30B4002347E00129EA
:1054400019D0022929D0002940D11418C4F50074BC
:10545000A3420ADDC2F50074A34206DA224C04EB33
:1054600083044FF07E55256030E01F4C04EB83042D
:10547000002525602AE0934209DD1418A34206DACC
:10548000194C04EB83044FF07E5525601EE0164C4A
:1054900004EB83040025256018E01418C4F500759A
:1054A000AB4203DDC2F50075AB4203DB934208DD7E
:1054B000A34206DA0C4C04EB83044FF07E552560C2
:1054C00004E0094C04EB8304002525600133B3F5A7
:1054D000007FB4DB044B03F5806100220A6003F215
:1054E000FC731A6030BC7047F80C0020F0B4002444
:1054F00029E0E200871897ED007A6300224EB51884
:1055000095ED006A67EE066A151D054495ED007A73
:1055100001339B001E44D6ED007A27EE277A36EE43
:10552000C77A1A4E324482ED007A95ED007A67EE22
:10553000877A97ED007A26EE076A77EE867A33440B
:10554000C3ED007A0134FF2CD3DD002316E04A00BE
:10555000002B03DA00EB830400252560B3F5007F00
:1055600003DB00EB83040025256000EB83059C181A
:10557000064A02EB840212682A600133B3F5007F09
:10558000E5DBF0BC704700BFF80C0020A83D002010
:1055900088B000220092294B196B41F00101196378
:1055A000196B01F00101009100990192196B41F012
:1055B00002011963196B01F0020101910199029234
:1055C000196B41F004011963196B01F00401029198
:1055D00002990392196B41F008011963196B01F0EC
:1055E0000801039103990492196B41F010011963AA
:1055F000196B01F01001049104990592196B41F4A3
:1056000000111963196B01F40011059105990692B7
:10561000196B41F480011963196B01F48001069143
:10562000069907921A6C42F480021A641B6C03F408
:1056300080030793079B08B0704700BF0038024003
:10564000024A136801331360704700BFE809002065
:105650000023064A1360064A13607F21054A116041
:10566000054A13606422054B1A607047F814002045
:10567000F40C002020250020FC140020CC49002040
:105680002F4B1B78002B5AD110B52E4B99881868D8
:10569000FBF7C6FD44002C4B99881868FBF7C0FD4A
:1056A00020442A4B18602A4B1B68984242D00BB901
:1056B000012813D0012B01D1032808D0032B01D1DD
:1056C000022806D0022B06D138B1002006E0184689
:1056D00004E0012002E0002000E001201D4B1860E2
:1056E0001D4B99881868FBF79BFDB8B9194B1B68CF
:1056F00023B11A4A13880133138003E0174A138831
:10570000013B1380154B1B885B08154A1188B3FBBE
:10571000F1F201FB1233134A13800BE00D4B1B68AF
:1057200023B1114A13680133136003E00E4A136872
:10573000013B1360054B1A68054B1A6010BD70479A
:10574000C209002010AB000860AB0008F40C002078
:10575000F81400202C3D002020AB00089C090020FC
:1057600038040020C8090020D049002008B50B49A2
:10577000D1E90023013243F10003C1E90023FFF71F
:1057800049F8FFF77DFFFAF79BFE054B1B681BB13D
:10579000034A1368013B136008BD00BF8805002061
:1057A000300B0020034B1868002800DA013040104D
:1057B000704700BFD0490020002308E000EB8301C0
:1057C0000B4A02EB830212680A6001339BB2094A5A
:1057D0001288B3EB420FF1DB05E000EB83020021FE
:1057E000116001339BB2B3F5007FF6D3704700BF61
:1057F000AC450020680400202DE9F04F83B08246BC
:1058000089463B4B1A6810460192B3F804B0002257
:105810005946FBF717FD374B1F68B3F80480002289
:1058200041463846FBF70EFD334B1D689E8800222B
:1058300031462846FBF706FD012231462846FBF794
:1058400001FD002415E0C4F107024AFA02F202F059
:10585000010241463846FBF7F5FC00223146284656
:10586000FBF7F0FC012231462846FBF7EBFC013444
:10587000E4B2072CE7D901225946019C2046FBF7E8
:10588000E1FC002259462046FBF7DCFC01224146A0
:105890003846FBF7D7FC002231462846FBF7D2FCFE
:1058A000012231462846FBF7CDFC002415E0C4F167
:1058B000070249FA02F202F0010241463846FBF7BC
:1058C000C1FC002231462846FBF7BCFC01223146D0
:1058D0002846FBF7B7FC0134E4B2072CE7D90122D4
:1058E00059460198FBF7AEFC03B0BDE8F08F00BF4E
:1058F000C8AB0008E8AB000830AB000808B50228C8
:105900004ED0032800F09580002840F0DA806D4BDF
:10591000012299881868FBF795FC6B4B0022998847
:105920001868FBF78FFC694B002299881868FBF711
:1059300089FC674B012299881868FBF783FC654B4B
:10594000002299881868FBF77DFC634B0122998837
:105950001868FBF777FC614B012299881868FBF700
:1059600071FC5F4B002299881868FBF76BFC5D4B5C
:10597000002299881868FBF765FC5B4B0022998828
:105980001868FBF75FFC594B012299881868FBF7F0
:1059900059FC574B002299881868FBF753FC08BD47
:1059A000484B012299881868FBF74CFC464B0022B3
:1059B00099881868FBF746FC444B002299881868C0
:1059C000FBF740FC424B012299881868FBF73AFC30
:1059D000404B002299881868FBF734FC3E4B0122AB
:1059E00099881868FBF72EFC3C4B012299881868AF
:1059F000FBF728FC3A4B002299881868FBF722FC39
:105A0000384B012299881868FBF71CFC364B0122A1
:105A100099881868FBF716FC344B0122998818689E
:105A2000FBF710FC324B002299881868FBF70AFC40
:105A300008BD244B002299881868FBF703FC224B11
:105A4000012299881868FBF7FDFB204B00229988FA
:105A50001868FBF7F7FB1E4B012299881868FBF7C3
:105A6000F1FB1C4B002299881868FBF7EBFB1A4BE3
:105A7000012299881868FBF7E5FB184B01229988E9
:105A80001868FBF7DFFB164B002299881868FBF7B4
:105A9000D9FB144B012299881868FBF7D3FB124BF2
:105AA000012299881868FBF7CDFB104B01229988D9
:105AB0001868FBF7C7FB0E4B002299881868FBF7A4
:105AC000C1FB08BDA8AB000850AB0008F8AB00084C
:105AD00008AB000878AB000880AB000868AB000892
:105AE00070AB0008B8AB000828AB000840AB00085A
:105AF00048AB000810B582B01D4BD3ED007A9FED86
:105B00001D7A67EE877AB7EE007A77EE877A17EE1E
:105B1000900A03F06DF941EC100B02F0C5FC002275
:105B2000154B51EC100B03F0B7F903F065FC04467C
:105B3000124B1A6890420CDD90B2221A96304FF444
:105B400078430093032312B29C2100B2FEF762F95E
:105B50000AE080B2121A963000230093032312B297
:105B60009C2100B2FEF756F9044B1C6002B010BD38
:105B7000B809002000247449000024409409002042
:105B800008B59FED147A002308E000EB8302D2ED04
:105B9000007A67EEA77A37EE277A01338B42F4DB7F
:105BA00007EE901AF8EEE77AC7EE276AF5EEC06ABC
:105BB000F1EE10FA0BDBB1EEE60AB4EE400AF1EEBC
:105BC00010FA06D0B0EE660A02F0F6FC08BD9FEDB2
:105BD000010A08BD00000000934B1B68012B40F038
:105BE00015812DE970432DED028B82B08F4B1B6820
:105BF0000BB18F4E00E08F4E4FF480728E498F486C
:105C000002F098FB0124DFED8E6A9FED8E7A14E09E
:105C1000894B03EB8403D3ED007AB4EEE77AF1EE1F
:105C200010FA01D5B0EE677AF4EEE76AF1EE10FAF9
:105C300001DDF0EE676A0134E4B2FF2CE8D1824B5B
:105C400093ED008AB4EEC87AF1EE10FA16DD17EE85
:105C5000100A03F0CDF86EA3D3E9002303F01CF97A
:105C60008046894618EE100A03F0C2F842464B46B9
:105C700002F060FF03F0E8FB734B1860724D286878
:105C800003F0B6F841EC100B02F00EFC286803F0AC
:105C9000AFF861A3D3E9002303F0FEF803F0D4FBCF
:105CA00007EE900A2860694B93ED007AF4EEC77A0C
:105CB000F1EE10FA01DD85ED007A634B93ED007A89
:105CC000634BD3ED007AB4EEE77AF1EE10FA02D529
:105CD0005D4BC3ED007A5F4B1878782302460021B4
:105CE000FEF772FB782537E0534B03EB850393ED0A
:105CF000007AF7EE007A77EE277A17EE900A03F033
:105D000077F841EC100B02F0CFFB45A3D3E9002359
:105D100051EC100B03F0EAF9804689464A4B1868AB
:105D200003F066F802460B464046494603F0DEF9AA
:105D30000022494B03F0B0F803F086FB07EE900A0F
:105D4000FCEEE77ACDED017A9DF8043036F81300C9
:105D5000FEF762FB013DEDB2002DC5D13D4B187839
:105D6000EF2302467821FEF72FFB37E0324B03EB9F
:105D7000840393ED007AF7EE007A77EE277A17EE38
:105D8000900A03F035F841EC100B02F08DFB24A3D0
:105D9000D3E9002351EC100B03F0A8F980468946A3
:105DA000294B186803F024F802460B464046494642
:105DB00003F09CF90022284B03F06EF803F044FB3B
:105DC00007EE900AFCEEE77ACDED017A9DF80430FB
:105DD00036F81300FEF720FB013CE4B2872CC5D84F
:105DE0001C4A13780133DBB21370772B02D90022DF
:105DF000184B1A70174B1878FEF764FC00220A4BF8
:105E00001A6002B0BDEC028BBDE87083704700BF22
:105E10009A9999999999B93FAE47E17A14AEEF3FB3
:105E2000EF39FAFE422EE63FBC0900208005002033
:105E3000F8B0000844CB0008900500202825002079
:105E40000000C84200000000A409002074040020E3
:105E500070040020D80900200000594010B400232D
:105E600004E001EB8302002414600133B3F5007FEA
:105E7000F7DBC300C818044A0260043319440A60FF
:105E80005DF8044B704700BF6666663F964B1B7813
:105E900013F0FF0F00F0268110B586B0934B1B68FE
:105EA000012B78D1924B186800283DD101230022A4
:105EB0004FF4807101A802F0E3F98E4901A802F0C5
:105EC000BFF98D4B1B6893B98C4B1B78012B0AD102
:105ED0000DE09A008749114409688948024411601D
:105EE00001339BB200E00023B3F5007FF1D3854B73
:105EF00019688048FFF7FAFA7F4B1B68012B16D10F
:105F00007E4B1B78012B0AD111E09A00794911448C
:105F100009687B480244116001339BB200E0002312
:105F2000B3F5007FF1D302E07249FFF797FF012339
:105F30001A464FF4807101A802F0A2F96D4901A838
:105F400002F07EF9704B1B78022B18D14FF480724F
:105F50006E49684802F0EEF900230EE059006B4AE2
:105F600002EB83021068634A02EBC3042060013134
:105F700002EB8102106001339BB2FF2BEED94FF48C
:105F800000715C48FFF7FCFD614B83ED000A0022C5
:105F9000564B1A609EE05F4B1B68012B4BD1544B54
:105FA000186888B9012300224FF4807101A802F01B
:105FB00067F9594C214601A802F042F9514B196882
:105FC0002046FFF793FA02E05349FFF747FF01230A
:105FD0001A464FF4807101A802F052F94E4901A807
:105FE00002F02EF9484B1B78022B18D14FF4807227
:105FF0004649494802F09EF900230EE05900434A01
:1060000002EB83021068444A02EBC30420600131B2
:1060100002EB8102106001339BB2FF2BEED94FF4EB
:1060200000713D48FFF7ACFD394B83ED000A0022BB
:10603000384B1A604EE0394B1B68012B4AD12C4B70
:10604000186888B9012300224FF4807101A802F07A
:1060500017F9334C214601A802F0F2F8294B1968D0
:106060002046FFF743FA02E02D49FFF7F7FE012330
:106070001A464FF4807101A802F002F9284901A8DC
:1060800002F0DEF8204B1B78022B18D14FF48072FF
:106090001E49234802F04EF900230EE059001B4A26
:1060A00002EB830210681E4A02EBC3042060013138
:1060B00002EB8102106001339BB2FF2BEED94FF44B
:1060C00000711748FFF75CFD114B83ED000A0022B9
:1060D000124B1A600022044B1A700122114B1A60F5
:1060E00006B010BD704700BF810B0020980900204A
:1060F000E40900202C2D00208005002084050020CC
:1061000028250020DC090020AC0900202C350020C7
:10611000B8090020C409002000150020F009002063
:10612000201D0020BC09002010B5FFF73BFB134BDE
:106130001860134B1B68984216D01A1A114B1C6832
:1061400011490B6804FB02330B60104A934201DCD7
:1061500001320A600C4B1A680D4B9A4202DD1A4656
:10616000094B1A60064B1860074B1868094B1B68EF
:10617000984201D0FFF7F0F810BD00BFA43D002009
:10618000282D0020800400206C0400209F2526007C
:10619000C0496E0AEC09002008B57B4B1B880A2B0E
:1061A00000F2F180DFE813F0BF009A000B0011004D
:1061B00017001E0025002B00310037006900734ACC
:1061C000734B1A60FFF7B0FF08BD724A704B1A603C
:1061D000FFF7AAFF08BD42F210726D4B1A60FFF77D
:1061E000A3FF08BD4FF47A72694B1A60FFF79CFF5A
:1061F00008BD6422664B1A60FFF796FF08BD0A22AD
:10620000634B1A60FFF790FF08BD0122604B1A60D4
:10621000FFF78AFF08BDFFF7C5FA5F4B18605F4BB9
:106220001B68984200F0AF801A1A5D490B8813442E
:106230001BB20B80002B01DC00220A80584BB3F903
:106240000030C72B02DD6422554B1A80544BB3F942
:106250000020544BB3F900309A4202DB5A1E5049D9
:106260000A804E4A10604E4AB2F9000002464E497A
:106270000978181AFFF7DEF808BDFFF793FA464BC6
:106280001860464B1B6898427DD01A1A45490B8806
:1062900013441BB20B80002B01DC00220A80414B0F
:1062A000B3F90030C72B02DD64223E4B1A803D4B10
:1062B000B3F900203A4BB3F900309A4202DC5A1C81
:1062C00038490A80354A1060364AB2F900001A4649
:1062D00035490978C01AFFF7ADF808BDFFF762FA33
:1062E0002D4B18602D4B1B6898424CD01B1A2E4A20
:1062F00011780B442D4981FB0301A1EBE37101EB04
:106300004101591AC9B21170254BB3F90030254A21
:10631000B2F900001A46C01AFFF78CF81E4B1A6833
:106320001E4B1A6008BDFFF73DFA1B4B18601B4B54
:106330001B68984227D01B1A07EE903AF8EEE77ACE
:106340001B4B93ED007A67EE877A1A4B93ED007A38
:1063500077EE877AC3ED007A174B93ED007AF4EE6F
:10636000C77AF1EE10FA02DD124B83ED007A114B81
:10637000D3ED007AF5EEC07AF1EE10FA01D80022E2
:106380001A60064B186008BDC809002040420F0083
:1063900080040020A0860100A43D0020282D0020BC
:1063A000E009002066040020AC0900205655555530
:1063B00034040020780400205404002010B582B07A
:1063C0000C4611462E380B2875D8DFE800F006740D
:1063D0006A101A242E38424C5660019313230093FE
:1063E0000F233A4A09B220B2FDF704FE6BE0019395
:1063F000132300930F23364A09B220B2FDF7FAFDAA
:1064000061E00193132300930F23324A09B220B2B3
:10641000FDF7F0FD57E00193132300930F232E4A5D
:1064200009B220B2FDF7E6FD4DE00193132300937E
:106430000F232A4A09B220B2FDF7DCFD43E00193A5
:10644000132300930F23264A09B220B2FDF7D2FD91
:1064500039E00193132300930F23224A09B220B29B
:10646000FDF7C8FD2FE00193132300930F231E4A6D
:1064700009B220B2FDF7BEFD25E00193132300937E
:106480000F231A4A09B220B2FDF7B4FD1BE00193B5
:10649000132300930F23164A09B220B2FDF7AAFD79
:1064A00011E00193132300930F23124A09B220B283
:1064B000FDF7A0FD07E00023009313230F2209B28C
:1064C00020B2FDF7A7FC02B010BD00BFC0BA0008A3
:1064D00008E3000870C3000808C9000884BF00086A
:1064E00044CC000844E50008F4B70008ACC5000837
:1064F000F8B10008ACDF000810B582B00C461146B8
:106500002D38512800F2A380DFE800F08DA1A1838F
:1065100029333D47515B656F79A1A1A1A1A1A1A13B
:10652000A1A1A1A1A1A1A1A1A1A1A1A1A1A1A1A15B
:10653000A1A1A1A1A1A1A1A1A1A1A1A1A1A1A1A14B
:10654000A1A1A1A1A1A1A1A1A1A1A1A1A1A1A1A13B
:10655000A1A1A1A1A1A1A1A1A1A1A1A1A1970193E3
:106560000923009308233F4A09B220B2FDF742FDF8
:1065700075E001930923009308233B4A09B220B236
:10658000FDF738FD6BE00193092300930823374A98
:1065900009B220B2FDF72EFD61E0019309230093BB
:1065A0000823334A09B220B2FDF724FD57E00193D6
:1065B0000923009308232F4A09B220B2FDF71AFDE0
:1065C0004DE001930923009308232B4A09B220B21E
:1065D000FDF710FD43E00193092300930823274AA8
:1065E00009B220B2FDF706FD39E0019309230093BB
:1065F0000823234A09B220B2FDF7FCFC2FE00193E7
:106600000923009308231F4A09B220B2FDF7F2FCC8
:1066100025E001930923009308231B4A09B220B205
:10662000FDF7E8FC1BE00193092300930823174AB8
:1066300009B220B2FDF7DEFC11E0019309230093BB
:106640000823134A09B220B2FDF7D4FC07E0002367
:1066500000930923082209B220B2FDF7DBFB02B048
:1066600010BD00BFE0C2000878D00008C0C100081B
:1066700078E2000800D30008F4BE000868B0000803
:1066800050C20008E8E10008E8C7000830BA000876
:1066900078C8000800000000F0B585B001229D4BCD
:1066A0001A70054690B34FF6FF7401940C270097BB
:1066B0002823994A5A219620FDF79CFC02947223C4
:1066C0000193882600967C23324677217E20FDF7B1
:1066D000CDFB019400972F23904A31469620FDF779
:1066E00089FC23466C22BE212E20FFF767FE23463D
:1066F0006C22FE212E20FFF761FE01940A230093F5
:106700009B23874AA2218E20FDF774FC854C864B83
:106710001A688649204603F035F994F90000844B45
:1067200093F9003098420AD14DB9824B1B88824AB6
:106730001288934210D0022B01D0022A0CD17D4B3B
:106740001B88022B02D14FF4784301E04FF6FF7310
:106750006C228E21FFF732FE724B93F90100744BCD
:1067600093F9013098420DD1744B1B7853B94DB950
:10677000704B1B88704A1288934210D0022B01D0B4
:10678000022A0CD16B4B1B88022B02D14FF47843A9
:1067900001E04FF6FF736C229E21FFF70FFE614B65
:1067A00093F90200624B93F9023098420AD14DB935
:1067B000604B1B88604A1288934210D0022B01D094
:1067C000022A0CD15B4B1B88022B02D14FF4784379
:1067D00001E04FF6FF736C22AE21FFF7EFFD514B46
:1067E00093F90300524B93F9033098420AD14DB903
:1067F000504B1B88504A1288934210D0032B01D073
:10680000032A0CD14B4B1B88032B02D14FF4784346
:1068100001E04FF6FF736C22CE21FFF7CFFD414B15
:1068200093F90400424B93F9043098420AD14DB9D0
:10683000404B1B88404A1288934210D0042B01D051
:10684000042A0CD13B4B1B88042B02D14FF4784314
:1068500001E04FF6FF736C22DE21FFF7AFFD314BF5
:1068600093F90500324B93F9053098420AD14DB99E
:10687000304B1B88304A1288934210D0052B01D030
:10688000052A0CD12B4B1B88052B02D14FF47843E2
:1068900001E04FF6FF736C22EE21FFF78FFD214BD5
:1068A00093F90600224B93F9063098420AD14DB96C
:1068B000204B1B88204A1288934211D0062B01D00E
:1068C000062A0DD11B4B1B88062B02D14FF47843AF
:1068D00001E04FF6FF736C224FF48771FFF76EFDF6
:1068E000104B93F90700124B93F9073098420AD1E5
:1068F0004DB9104B1B88104A1288934227D0072BA2
:1069000001D0072A23D10B4B1B88072B18D14FF43A
:10691000784317E0C209002034B4000800AC000836
:1069200090D30008F40900206C04002080E70008E0
:106930003C040020C809002030040020001D002075
:106940004FF6FF736C224FF48F71FFF737FD9E4BAC
:1069500093F908009D4B93F9083098420AD14DB93C
:106960009B4B1B889B4A1288934211D0082B01D065
:10697000082A0DD1964B1B88082B02D14FF478437F
:1069800001E04FF6FF736C224FF49771FFF716FD8D
:10699000914B1A68914B1A608B498C4803F018F898
:1069A0008F4B1A788F4B1B789A4212D18E4BB3F9CA
:1069B00000208E4BB3F900309A420AD14DB9844B76
:1069C0001B88844A128893422AD0092B01D0092AB5
:1069D00028D1854BB3F9003003EB8303DA008449F7
:1069E000794802F0CFFF002412E0774B185704EBF0
:1069F000C401CD3189B2764B1B88092B02D14FF4EB
:106A0000784301E04FF6FF738922FFF775FD0134EB
:106A1000032CEADD744B1A88744B1A80012602E0BD
:106A2000002600E000266E4B1A786E4B1B789A42C7
:106A300012D1704BB3F900206F4BB3F900309A427A
:106A40000AD14DB9624B1B88624A1288934229D001
:106A50000A2B01D00A2A25D1664BB3F9003003EB8B
:106A60008303DA006549584802F08CFF002412E0E5
:106A7000554B185704EBC401FA3189B2544B1B88AB
:106A80000A2B02D14FF4784301E04FF6FF738922BD
:106A9000FFF732FD0134032CEADD564B1A88564BC2
:106AA0001A800126564B93ED007A564BD3ED007AAF
:106AB000B4EE677AF1EE10FA08D13DB9444B1B8869
:106AC000444A128893422FD003B16ABB3E48342314
:106AD000037033234370322383703123C370B2EECB
:106AE000047A67EE877AFDEEE77A17EE902A40493E
:106AF00002F048FF002411E0334B185704EBC401A7
:106B0000FA3189B2324B1B8813B94FF4784301E054
:106B10004FF6FF730A22FFF7EFFC0134032CEBDD85
:106B2000384B1A68364B1A60002E00F0A9802C4BA7
:106B30001B78012B25D013B1022B65D0A0E00021DA
:106B40000091F02303227920FDF764F9264BB3F975
:106B50000030002B00DA0133C3F34F01254BB3F9AA
:106B60000030002B00DA0133C1EB630378314FF6BC
:106B7000FF7200921BB2032209B27920FDF74AF995
:106B80007EE000210091F02303227920FDF742F9F5
:106B9000184BB3F90030002B00DA0133C3F34F0177
:106BA000114BB3F90030002B00DA0133A1EB630382
:106BB000C1F178014FF6FF7200921BB2032209B2B5
:106BC0007920FDF727F95BE0F40900203C04002060
:106BD000C8090020300400206C040020EC090020CB
:106BE000AC0900207C040020E00900204C040020B7
:106BF00088E7000866040020640400208CE7000891
:106C0000500400207804002000210091F02303228A
:106C10007920FDF7FFF8524BB3F90030002B00DA72
:106C20000133C3F34F014F4BB3F90030002B00DAAF
:106C30000133C1EB630378314FF6FF7200921BB250
:106C4000032209B27920FDF7E5F8464BB3F900308D
:106C5000002B00DA0133C3F34F01414BB3F900308D
:106C6000002B00DA0133A1EB6303C1F178014FF689
:106C7000FF7200921BB2032209B27920FDF7CAF815
:106C8000394B1B78394A127893420AD14DB9384AA8
:106C90001288384909888A4245D0012A01D0012941
:106CA00041D1012B16D013B1022B26D037E0304B47
:106CB0001B88012B02D14FF4784301E04FF6FF739C
:106CC0000193092300931C232B4A5B21C420FDF769
:106CD00091F924E0264B1B88012B02D14FF4784315
:106CE00001E04FF6FF730193092300931C23234A0D
:106CF0005B21C420FDF77EF911E01D4B1B88012BA1
:106D000002D14FF4784301E04FF6FF73019309235A
:106D100000931C231A4A5B21C420FDF76BF9124B28
:106D20001A78124B1A70174B186802F061F80AA310
:106D3000D3E9002302F0B0F80022002302F014FB94
:106D400018B90B4B1A880B4B1A8000220E4B1A7085
:106D500005B0F0BDAFF30080AE47E17A14AEEF3F6F
:106D6000E009002066040020AC0900207C0400201B
:106D7000C80900203004002080CE000808D1000897
:106D8000FCBC000878040020C20900202DE9F04175
:106D900082B02D4B1B682D4AA2FB03231B0E013B27
:106DA0002B4F3B60002500952A4E326C42F00202C8
:106DB0003264326C02F002020092009A264A916814
:106DC00041F002019160916841F004019160234C0F
:106DD000234A2260A56040F21A48C4F80C80636020
:106DE00025612046FCF7DAFD2046FCF721FC012254
:106DF00029461D20F9F714FF1D20F9F751FF0195D1
:106E0000336C43F004033364336C03F004030193E5
:106E1000019B144C144B2360A560C4F80C803B68A4
:106E2000636025612046FCF7B9FD2046FCF700FCB5
:106E3000042202211E20F9F7F3FE1E20F9F730FF8D
:106E400002B0BDE8F08100BF0C00002029D94266E5
:106E5000D409002000380240002004E03C0C00204F
:106E600000040040340B00200008004008B5024830
:106E7000FCF734FC08BD00BF3C0C002008B5FFF750
:106E800005F80248FCF72AFC08BD00BF340B0020BF
:106E900000B583B000230193234B1A6C42F00052DB
:106EA0001A641B6C03F000530193019B1F48204B95
:106EB0000360F9F741FF08B1FEF7C2FB1D4900224C
:106EC0000A604A601948F9F79DFF08B1FEF7B8FB60
:106ED000102218491548F9F795FF08B1FEF7B0FBE5
:106EE0008823002211461148F9F7E0FF08B1FEF7A8
:106EF000A7FB8823002210210C48F9F7D7FF08B11F
:106F0000FEF79EFB00210948F9F738FF08B1FEF7AC
:106F100097FB10210548F9F731FF08B1FEF790FB08
:106F200003B05DF804FB00BF00380240903D002034
:106F300000740040B00900202DE9F043A5B0FEF731
:106F40003BFAF9F7B1FAFEF723FBFDF75FFE00F01D
:106F5000CDFC4FF40043039300251D9503A8FBF7D8
:106F6000F3FA744C744B23602046FAF7AFFB01230D
:106F7000E3602561E561256240F20F33A360FE23E3
:106F800063616E4B63602046FAF7E8FA10B16C4813
:106F9000FCF7E0FD012005E064231A46E021654886
:106FA000FAF71EFD0028F7D1FEF752F9654B186875
:106FB000FEF7D2F9FDF710FCFDF7EEFB01224FF4CE
:106FC00000516148FAF73EF9604BB3F90030604A6E
:106FD000B2F900001A465F490978C01AFEF72AFA8A
:106FE000FFF756FFFEF734FBFDF7C2F80120FDF76F
:106FF00095FB0020FCF726FF0320FDF745F8012054
:10700000FDF754F800214FF6FF70FDF745F8C82250
:1070100078210020FDF762FBFDF79AFC01244E4B1E
:107020001C70FDF7C7FDFFF7B1FE2046FFF734FBEC
:10703000C8210846FEF7E0FBFFF7AEF80020FFF797
:107040002BFBFEF7C9FDFEF755FD444B99881868E8
:10705000FAF7E6F810B14FF4784300E01F230093ED
:1070600003231A4600214FF49B70FCF7D3FE3C4BE0
:1070700099881868FAF7D4F810B14FF4784300E013
:107080001F23009303231A4604214FF49B70FCF73F
:10709000C1FE344B1C689D8829462046FAF7C0F88B
:1070A00010B14FF4784300E01F23009303231A46E6
:1070B00008214FF49B70FCF7ADFE2B4B1E689F8898
:1070C00039463046FAF7ACF810B14FF4784300E097
:1070D0001F23009303231A460C214FF49B70FCF7E7
:1070E00099FE224BD3F80080B3F80490204B998886
:1070F0001868FAF795F8024649464046FAF7A2F8AA
:1071000029462046FAF78CF870B939463046FAF726
:1071100087F848B90122174B1A600220FEF7EEFBF0
:107120000022154B1A6087E70020124B1860FEF70B
:10713000E5FB81E7F40B0020005800403227914026
:1071400094E700086C04002000100240E0090020D1
:1071500066040020AC090020F10B0020B0AB000851
:10716000D0AB0008D8AB0008C0AB000858AB000893
:1071700000AB000880050020E409002008B5C0F33A
:107180000B03002211460248F9F790FE08BD00BF2C
:10719000903D002008B5C0F30B03002210210248E7
:1071A000F9F784FE08BD00BF903D002000000000FC
:1071B000954B1B78002B00F05E832DE9F041934B3B
:1071C0001B88642B05D101224FF400519048FAF737
:1071D00039F8FDF7AFFC8F4B1B68012B00F0E780FF
:1071E000022B00F0F781002B40F0FE828A4B1B68D7
:1071F0003BBB864B1D886E00884B1B889BB2884A20
:107200001068181A01F0E2FD0022864B01F044FEDE
:10721000854C04EBC50502F017F92860751C834BFB
:107220001B889BB2824A1068181A01F0CFFD002219
:107230007C4B01F031FE04EB850402F005F920607F
:1072400026E0724B1D886E00DFF8EC81B8F8000074
:1072500080B2784B1F68C01B01F0B8FD0022714B53
:1072600001F01AFE704C04EBC50502F0EDF8286041
:10727000751CB8F8000080B2C01B01F0A7FD002209
:10728000684B01F009FE04EB850402F0DDF8206094
:10729000694B1B889BB2694A1288934203D9664B9B
:1072A0001A88664B1A80614B1B889BB2634A12880E
:1072B000934203D95D4B1A88604B1A80534B19884F
:1072C0004B005F4A02EBC102D2ED007A5D4A92EDBB
:1072D000007AF4EEC77AF1EE10FA01DDC2ED007A21
:1072E0005A1C574B03EB8203D3ED006A554B93EDC9
:1072F000007AF4EEC76AF1EE10FA01DDC3ED006A20
:10730000DFED515A67EEA57A504B93ED007A67EEA8
:10731000877A9FED4F6A77EE867AFDEEE77A17EE71
:10732000900A4C4BC3ED007A66EEA56A27EE267AEA
:1073300037EE067AFDEEC77A17EE903A464AC2ED6E
:10734000007A354A1268012A0BD1444A12689042E9
:1073500001DD424A1060414A1268934201DD3F4A12
:10736000136080B2FFF70AFF3B4B1888FFF712FF4C
:10737000264B1A883A4B1B88C3F1FF018A42C0F2A0
:107380003382C3F58073D31A58005400264901EBA9
:10739000C2021568334A02EBC3031D60431C601C24
:1073A00001EB8001096802EB830211601CE21A4BB9
:1073B0001B68002B58D1154B1D886E00174B1B887E
:1073C0009BB2174A1068181A01F000FD0022154BF5
:1073D00001F062FD1A4C04EBC50502F035F8286097
:1073E000751C124B1B889BB2114A1068181A01F0C9
:1073F000EDFC00220B4B01F04FFD04EB850402F085
:1074000023F8206057E000BFF10B0020380C00206B
:10741000001002409009002080050020EE0B0020A3
:10742000600400200000303F2C2D00202C0B002099
:107430005C04002058040020140A0020C009002029
:1074400000150020D00900200000804578040020AD
:1074500000000045A0090020A8090020CC09002058
:1074600068040020AC450020704B1D886E00DFF8DA
:10747000CC81B8F8000080B26D4B1F68C01B01F0D2
:10748000A5FC00226B4B01F007FD6B4C04EBC5051E
:1074900001F0DAFF2860751CB8F8000080B2C01B4C
:1074A00001F094FC0022634B01F0F6FC04EB850430
:1074B00001F0CAFF2060614B1B889BB2604A1288B2
:1074C000934203D95D4B1A885D4B1A805D4B1B8834
:1074D0009BB25B4A1288934203D95A4B1A88584B85
:1074E0001A80524B19884B00574A02EBC102D2ED69
:1074F000007A564A92ED007AF4EEC77AF1EE10FA6D
:1075000001DDC2ED007A5A1C4F4B03EB8203D3ED31
:10751000006A4E4B93ED007AF4EEC76AF1EE10FA72
:1075200001DDC3ED006ADFED4A5A67EEA57A494BEB
:1075300093ED007A67EE877A9FED476A77EE867A59
:10754000FDEEE77A17EE900A444BC3ED007A66EE43
:10755000A56A27EE267A37EE067AFDEEC77A17EE91
:10756000903A3F4AC2ED007A3E4A1268012A0BD196
:107570003D4A1268904201DD3B4A10603A4A126867
:10758000934201DD384A136080B2FFF7F7FD344BB8
:107590001888FFF7FFFD254B1A88344B1B88C3F171
:1075A000FF018A42C0F22081C3F58073D31A5800CC
:1075B0005400214901EBC20215682D4A02EBC303B6
:1075C0001D60431C601C01EB8001096802EB830213
:1075D000116009E1234B1B68002B51D1134B1D880F
:1075E0006E00244B1B889BB2234A1068181A01F0C6
:1075F000EDFB00220F4B01F04FFC134C04EBC505D3
:1076000001F022FF2860751C0E4B1B889BB21B4AA1
:107610001068181A01F0DAFB0022064B01F03CFC5E
:1076200004EB850401F010FF206050E0380C0020CE
:10763000580400200000303F00150020140A0020EC
:10764000C00900202C0B0020201D0020D0090020A4
:10765000000080457804002000000045A0090020BB
:10766000A809002080050020CC0900206804002023
:10767000AC450020EE0B0020600400205C040020DC
:107680007F4B1D886E00DFF80882B8F8000080B2DA
:107690007C4B1F68C01B01F099FB00227A4B01F064
:1076A000FBFB7A4C04EBC50501F0CEFE2860751C8F
:1076B000B8F8000080B2C01B01F088FB0022724BBA
:1076C00001F0EAFB04EB850401F0BEFE2060704B84
:1076D0001B889BB26F4A1288934203D96C4B1A885D
:1076E0006C4B1A806C4B1B889BB26A4A128893427F
:1076F00003D9694B1A88674B1A80614B19884B0074
:10770000664A02EBC102D2ED007A654A92ED007A38
:10771000F4EEC77AF1EE10FA01DDC2ED007A5A1CE0
:107720005E4B03EB8203D3ED006A5D4B93ED007A71
:10773000F4EEC76AF1EE10FA01DDC3ED006ADFED89
:10774000595A67EEA57A584B93ED007A67EE877A1F
:107750009FED566A77EE867AFDEEE77A17EE900A8D
:10776000534BC3ED007A66EEA56A27EE267A37EE14
:10777000067AFDEEC77A17EE903A4E4AC2ED007ACD
:107780004D4A1268012A0BD14C4A1268904201DD21
:107790004A4A1060494A1268934201DD474A136021
:1077A00080B2FFF7EBFC434B1888FFF7F3FC344B38
:1077B0001A88434B1B88C3F1FF018A4214DBC3F5CF
:1077C0008073D31A58005400304901EBC202156887
:1077D0003C4A02EBC3031D60431C601C01EB8001AB
:1077E000096802EB830211602D4C206801F000FB58
:1077F00021A3D3E9002301F04FFB01F025FE206017
:107800001F4A138801339BB21380FF2B2FD900220C
:107810004FF400512C48F9F715FD01222B4B1A703B
:10782000274B1A88164B1A80294B1B68012B0BD04B
:10783000022B13D0DBB90123264A1360244A1360BC
:107840002548FDF7B9FF12E00122244B1A600222FD
:107850001F4B1A600D48FDF7AFFF08E00122204BD7
:107860001A6000221A4B1A600C48FDF7A5FFFDF7BD
:10787000A1F9BDE8F08170471EA7E8482EFFEF3F51
:10788000380C0020580400200000303F201D00204C
:10789000140A0020C00900202C0B00202C2D0020F1
:1078A000D009002000008045780400200000004539
:1078B000A0090020A809002080050020CC09002094
:1078C00068040020AC45002000100240810B00201D
:1078D000900900209809002000150020C40900200C
:1078E000F009002008B5FFF763FC08BD2DE9F0435F
:1078F00087B0334C2046FBF78BFC00250095314BBD
:107900005A6C42F480525A645B6C03F480530093C7
:10791000009B2D4B9A8801920226049602964FF006
:107920000508CDF81480039501A91868F9F7F6FA4F
:10793000264B9A880192049602960395CDF81480FE
:1079400001A91868F9F7EAFA214B9A88019204967E
:10795000029501270397CDF8148001A91868F9F75B
:10796000DDFA1C4BB3F80490CDF80490049602970E
:1079700003950595D3F8008001A94046F9F7CEFAA2
:107980003A4649464046F9F75DFC134B2360A56033
:107990004FF4827363604FF4E063E36026616761D4
:1079A0004FF40073A361E5612562A5626562072358
:1079B000E3622046FBF72EFC07B0BDE8F08300BF72
:1079C000880B00200038024088AB0008A0AB0008FC
:1079D000E0AB000898AB00080030014084B008B567
:1079E0000DF1080E8EE80F001C9A138806491B0A39
:1079F0000B7013884B70012302220448FBF738FDFB
:107A0000BDE8084004B07047040A0020880B00203D
:107A1000704700BF704700BFFEE700BFFEE700BF32
:107A2000FEE700BFFEE700BFFEE700BF2DE9F04F15
:107A300049084F1C0024264662E0A6423FD24FEA86
:107A4000C50C00EB0C09D9F800A04FEAC40E00EBFE
:107A50000E08D8F800B0C9F800B0C8F800A00CF1C2
:107A6000040C8444DCF800800EF1040E8644DEF839
:107A70000090CCF80090CEF8008006EB070C4FEA9F
:107A8000CC0C00EB0C09D9F800A004EB070E4FEA70
:107A9000CE0E00EB0E08D8F800B0C9F800B0C8F858
:107AA00000A00CF1040C8444DCF800800EF1040EFC
:107AB0008644DEF80090CCF80090CEF800800135C6
:107AC000ED0000EB050CDCF800800C44E40000EB5A
:107AD000040EDEF80090CCF80090CEF8008004355B
:107AE0000544D5F800E004340444D4F800C0C5F8D7
:107AF00000C0C4F800E01C8803EB42030236B6B2B3
:107B00003546A1F1020E764597D9BDE8F08F00BF4A
:107B10002DE9F04F2DED048B87B004910292039371
:107B20004FEA9109CDF800904FF00008C246059148
:107B3000CB46164608EB0B020BEB02030BEB0301E3
:107B40004FEAC80400EB0409D9ED006A0434044488
:107B5000D4ED004AD20000EB020C9CED004A043246
:107B6000024492ED006ADB0000EB030E9EED007A0A
:107B7000043303440193D3ED005AC900471897ED2D
:107B8000005A04310144D1ED007A36EE872A74EEB2
:107B9000052A74EEA50A36EE271A4FEA0A1573195C
:107BA00093ED003A04353544D5ED003A76EEC76AD8
:107BB00034EE455A74EEE55A76EE677A32EE227A62
:107BC00089ED007A30EE817A84ED007A76EEA71A9C
:107BD00035EEC50A72EE624A30EEC12A36EEE77A19
:107BE00035EE256A4FEACA043519D5ED005A04343A
:107BF000344494ED004A0AEB4A04E4003519D5ED0B
:107C0000006A04343444D4ED007A61EEA50A60EED3
:107C1000252A23EE241A23EE025A67EE265A66EE30
:107C2000266A20EE040A21EE844A23EE822A63EEBD
:107C3000A44A26EE276A67EE277A30EE803A32EEC3
:107C4000C44A71EE023A35EE645A35EE867A76EE23
:107C5000E77ACCED003A82ED005A8EED003A019BB6
:107C600083ED004A87ED007AC1ED007A039B9A44C8
:107C700008F10108009B013B00937FF45BAFD946FC
:107C8000DDF814B0039B9B009BB20193049B9B08FF
:107C900004930393B2E04FEA9906002300939A46B7
:107CA0000AEB4A034FEACA02029C21461144D1ED75
:107CB000008A0432224492ED008A4FEA0A12A11887
:107CC00091ED000A04322244D2ED000ADB00E218F2
:107CD00092ED001A04332344D3ED001A019B9A4419
:107CE000009DAA19B318F118EC0000EB040898EDF8
:107CF000004A0434044494ED006AD20000EB020C04
:107D0000DCED005A04320244D2ED007ADB0000EBD5
:107D1000030E9EED005A0433034493ED007AC9002C
:107D20004718D7ED004A04310144D1ED006A34EE22
:107D3000453A35EEE42A76EE472A77EEE63A34EE17
:107D4000055A75EEA45A36EE077A77EEA67A73EEE8
:107D5000234A32EEC24A35EE659A77EE679A73EEA1
:107D6000636A32EE226A75EE255AC8ED005A77EE44
:107D7000277AC4ED007A28EEA45A68EE845A20EEE1
:107D8000093A60EE293A21EE267A61EE067A28EE6B
:107D9000044A68EE244A60EEA99A20EE899A21EE00
:107DA000866A61EEA66A35EE044A75EEE44A73EE21
:107DB000299A33EEC99A37EE066A77EEE66ACCED79
:107DC000009A82ED009A8EED004AC3ED004A87EDDD
:107DD000006AC1ED006A4D44AB4582D8009B013377
:107DE0001A460093731E9A427FF65AAF019B9B007E
:107DF0009BB20193039B9B080393B146039B042B07
:107E00003FF649AF049B90ED004A90ED016AD0ED3A
:107E1000026AD0ED034AD0ED045A90ED057AD0ED18
:107E2000067A90ED075A34EE253A74EE655A36EE2E
:107E3000074A36EE477A76EEA73A34EE856A76EE52
:107E4000E77A74EEC56A33EE232A74EE062A73EEDF
:107E5000633A34EE466A75EEA64A37EE675A75EE17
:107E6000E66A77EE277A80ED002AC0ED012AC0EDA0
:107E7000023A80ED036AC0ED044A80ED055AC0ED78
:107E8000066AC0ED077A2030013BBCD107B0BDECDB
:107E9000048BBDE8F08F00BF2DE9F04F2DED068B70
:107EA00087B00491029203934FEA9109CDF80090B4
:107EB0004FF00008C2460591CB46164608EB0B0270
:107EC0000BEB02030BEB03014FEAC80400EB0409C0
:107ED000D9ED006A04340444D4ED004ADB0000EB21
:107EE000030E9EED007A04330344019393ED005A90
:107EF000D20000EB020C9CED004A0432024492EDE9
:107F0000006AC9004718D7ED005A04310144D1ED89
:107F1000007A36EE872A74EE252A74EE850A36EE4C
:107F2000271A4FEA0A15731993ED003A04353544C0
:107F3000D5ED003A76EEC76A74EE655A34EEC55A4E
:107F400076EE677A32EE227A89ED007A30EE817A27
:107F500084ED007A76EEE71A35EE858A72EE624A93
:107F600030EEC12A36EEA77A35EE656A4FEACA04CA
:107F70003519D5ED005A0434344494ED004A0AEB27
:107F80004A04E4003519D5ED006A04343444D4EDD4
:107F9000007A61EEA50A68EE252A23EE241A23EE64
:107FA000025A67EE265A66EE266A28EE048A21EE09
:107FB000844A23EE822A63EEA44A26EE276A67EEFD
:107FC000277A30EEC83A32EE844A71EE423A35EE04
:107FD000245A35EEC67A76EEA77ACCED003A82EDD9
:107FE000005A8EED003A019B83ED004A87ED007A3E
:107FF000C1ED007A039B9A4408F10108009B013B04
:1080000000937FF45BAFD946DDF814B0039B9B006F
:108010009BB20193049B9B0804930393B2E04FEA45
:108020009906002300939A460AEB4A034FEACA02D4
:10803000029C2146114491ED009A04322244D2ED73
:10804000008A4FEA0A12A11891ED008A04322244F4
:10805000D2ED000ADB00E21892ED001A043323444B
:10806000D3ED001A019B9A44009DAA19B318F11888
:10807000EC0000EB040898ED004A0434044494ED4D
:10808000006AD20000EB020CDCED005A043202441C
:10809000D2ED007ADB0000EB030E9EED005A0433B4
:1080A000034493ED007AC9004718D7ED004A043124
:1080B0000144D1ED006A34EE453A75EEE42A36EE1D
:1080C000472A77EEE63A34EE055A75EEA45A36EEB4
:1080D000077A77EEA67A73EE634A32EE824A75EE3D
:1080E000659A37EE67AA73EE236A32EE626A75EE1E
:1080F000255AC8ED005A77EE277AC4ED007A29EEAA
:10810000245A69EE045A28EE293A68EE0A3A21EE1A
:10811000267A61EE067A28EE844A68EEA44A20EEBA
:108120008AAA60EEA99A21EE866A61EEA66A35EE09
:10813000444A75EEA44A33EE4AAA73EEA99A37EE82
:10814000466A77EEA66A8CED00AAC2ED009A8EED23
:10815000004AC3ED004A87ED006AC1ED006A4D4454
:10816000AB4582D8009B01331A460093731E9A4296
:108170007FF65AAF019B9B009BB20193039B9B0828
:108180000393B146039B042B3FF649AF049B90ED4C
:10819000004A90ED016AD0ED026AD0ED034AD0EDBD
:1081A000045A90ED057AD0ED067A90ED075A34EE38
:1081B000253A74EE655A36EE074A36EE477A76EE81
:1081C000A73A34EE856A76EEE77A74EEC56A33EE46
:1081D000232A74EE062A73EE633A34EE466A75EE8D
:1081E000E64A37EE275A75EEA66A77EE677A22EEF0
:1081F000003A22EE804A63EE805A26EE006A64EE70
:10820000804A25EE005A26EE807A67EE807A80ED6D
:10821000003A80ED014AC0ED025A80ED036AC0EDDC
:10822000044A80ED055A80ED067AC0ED077A2030C9
:10823000013BACD107B0BDEC068BBDE8F08F00BFB1
:1082400038B504460D468378012B08D190ED040A19
:108250008389426801882846FFF71EFE05E083896E
:10826000426801882846FFF753FCE378012B05D1CB
:10827000A368E28921882846FFF7D8FB38BD00BFF4
:1082800010B40180254C44608270C370B1F5807FCA
:108290001FD004D8102930D0402924D038E0B1F5BF
:1082A000806F0CD0B1F5805F32D101238381C3810F
:1082B0001B4B83604FF06653036100202AE00423C8
:1082C0008381C381174B83604FF06A5303610020A1
:1082D00020E010238381C381134B83604FF06E53E2
:1082E0000361002016E040238381C3810F4B83602C
:1082F0004FF07253036100200CE04FF480738381D0
:10830000C3810B4B83604FF076530361002001E083
:108310004FF0FF305DF8044B704700BFB0EF00082E
:10832000B0E70008B6E70008CEE700082EE800082E
:10833000AEE900082DE9F04104460D4617469608BF
:1083400082E0D4ED007A94ED010A67EEA77A20EE80
:10835000000A77EE807AF5EEC07AF1EE10FA0DDBC6
:10836000B1EEE70AB4EE400AF1EE10FA03D0B0EE37
:10837000670A00F021F985ED000A01E000232B6077
:10838000D4ED027A94ED030A67EEA77A20EE000A94
:1083900077EE807AF5EEC07AF1EE10FA0DDBB1EEF1
:1083A000E70AB4EE400AF1EE10FA03D0B0EE670A25
:1083B00000F002F985ED010A01E000236B60D4EDC5
:1083C000047A94ED050A67EEA77A20EE000A77EEAC
:1083D000807AF5EEC07AF1EE10FA0DDBB1EEE70A25
:1083E000B4EE400AF1EE10FA03D0B0EE670A00F0E6
:1083F000E3F885ED020A01E00023AB60D4ED067AD4
:1084000004F1200894ED070A67EEA77A20EE000A2F
:1084100077EE807A05F11004F5EEC07AF1EE10FAED
:108420000DDBB1EEE70AB4EE400AF1EE10FA03D02C
:10843000B0EE670A00F0C0F885ED030A01E0002302
:10844000EB60013E25464446002E7FF47AAF07F0EC
:10845000030724E026460836D4ED007A94ED010A9D
:1084600067EEA77A20EE000A77EE807A2C1DF5EEF3
:10847000C07AF1EE10FA0DDBB1EEE70AB4EE400A75
:10848000F1EE10FA03D0B0EE670A00F095F885ED32
:10849000000A01E000232B60013F25463446002FEF
:1084A000D8D1BDE8F08100BF2DE9F0432DED028B5E
:1084B0008BB055EC104B00F0D7F83A4BB0EE408A39
:1084C000F0EE608A93F90060731C0DD022462B46B3
:1084D0002046294600F07AFF30B9002200232046CA
:1084E000294600F069FF40B1B0EE480AF0EE680A94
:1084F0000BB0BDEC028BBDE8F0832B4B0890CDE9AF
:108500000245CDE904450193DEB9284F4FF060469E
:108510002046294600220023CDE9066700F024FF0B
:10852000002837D002230093684600F0F3FAC8B160
:10853000089BE3B99DED060B0BB0BDEC028BBDE8CB
:10854000F083DFF870904FF00008204629460022A3
:108550000023CDE9068900F007FF68B102239E429F
:108560000093E1D101F04CF922230360E0E701F030
:1085700047F9089B0360DDE70123022E00930BD12E
:1085800001F03EF921230360094800F0C5FA8DEDA2
:10859000060BCDE701230093684600F0BBFA0028E4
:1085A000F2D1EDE784040020B06F0108FFFFEFC7B0
:1085B000C4A900080000F0FF10B52DED028B8AB0B1
:1085C000B0EE408A00F054FA244B93F90040631C4B
:1085D00009D0B4EE488AF1EE10FA04D6B5EEC08A9E
:1085E000F1EE10FA03D40AB0BDEC028B10BD0123EA
:1085F0001B4A009318EE100A00230192089300F022
:10860000F7FB0022CDE90401CDE902010023BCB152
:108610001046194600F06AFD022CCDE9060111D181
:1086200001F0EEF821230360089B8BB9DDE9060118
:1086300000F00AFF00EE100A0AB0BDEC028B10BD7C
:10864000CDE90623684600F065FA0028ECD1E7E79B
:1086500001F0D6F8089B0360E8E700BF840400201F
:10866000B46F0108000000002DE9F04F51EC100B31
:10867000B1F5801F85B00B4659DA10EE102A21F0B3
:108680000044224300F0F8800029C0F280810022DB
:10869000DD4BDE4C00F000FC0B46A3426FF03502D0
:1086A0004ADCC3F3130505F5152404F6647404F4D9
:1086B000801686F07F541B1584F44014A3F2FF3318
:1086C00044EA05019C180022D14B00F031FAAB1CA2
:1086D000C3F31303022B04EB165482468B464FF070
:1086E000000232DC002300F03FFE002800F0CF80C3
:1086F000002C00F05881204600F068FBACA3D3E9C1
:10870000002306460F4600F0C7FBABA3D3E90023C6
:1087100004460D463046394600F0BEFB02460B4685
:108720002046294600F006FA41EC100B0AE0B74C4F
:10873000A3424FF00002B4DD02460B4600F0FAF906
:1087400041EC100B05B0BDE8F08F4FF0804300F016
:10875000F1F902460B465046594600F0C7FC064662
:1087600020460F4600F032FB3246CDE900013B4681
:1087700030463946CDE9026700F08EFB02460B46D3
:108780008046894600F088FB8DA3D3E90023064686
:108790000F4600F081FB8CA3D3E9002300F0CAF957
:1087A00032463B4600F078FB89A3D3E9002300F072
:1087B000C1F932463B4600F06FFB87A3D3E90023A3
:1087C00000F0B8F942464B4600F066FB84A3D3E9BB
:1087D0000023804689463046394600F05DFB82A37F
:1087E000D3E9002300F0A6F932463B4600F054FBE3
:1087F0007FA3D3E9002300F09DF932463B4600F009
:108800004BFB0B4602464946404600F093F9A5F55E
:10881000C223C5F5D725A3F27A4351351D43002D58
:10882000804689465CDD00227A4B5046594600F06E
:1088300033FB52465B4600F02FFB06460F46002CEA
:108840006ED132463B464046494600F073F9DDE9B9
:10885000022300F021FB02460B463046394600F069
:1088600067F902460B465046594600F061F941EC63
:10887000100B05B0BDE8F08F0022002300206649F0
:1088800000F034FC41EC100B05B0BDE8F08F5AA3AA
:10889000D3E900235046594600F0FEFA02460B4643
:1088A00000205C4900F044F9524606460F465B46FC
:1088B0005046594600F0F0FA02460B46304639461B
:1088C00000F0EAFA06460F46002C40F0A780024668
:1088D0000B465046594600F02BF941EC100B31E79E
:1088E000002C00F0AF8032A3D3E90023DDE90001C2
:1088F00000F0D2FA42464B4604460D4650465946D1
:1089000000F016F9DDE9022300F0C6FA2AA3D3E944
:10891000002306460F46DDE9000100F0BDFA21E024
:1089200023A3D3E90023DDE9000100F0B5FA3246C4
:108930003B4604460D464046494600F0FBF8DDE95B
:10894000022300F0A9FA1CA3D3E90023804689463C
:10895000DDE9000100F0A0FA02460B464046494618
:1089600000F0E8F802460B463046394600F0E0F8E1
:1089700052465B4600F0DCF802460B46204629468C
:1089800000F0D6F841EC100B05B0BDE8F08F10EE0A
:10899000102A0B4600F0CCF80022002300F0A6FBC2
:1089A00041EC100BCEE69FED160BCBE6AFF300804B
:1089B0000000E0FE422EE63F763C7935EF39EA3D95
:1089C00044523EDF12F1C23FDE03CB966446C73FFE
:1089D000599322942449D23F935555555555E53F17
:1089E0009FC678D0099AC33FAF788E1DC571CC3F22
:1089F00004FA97999999D93F555555555555D53FED
:108A0000000000000000000000005043FFFFEF7F67
:108A10000000F03F0000E03F000050C3204600F09F
:108A2000D5F90FA3D3E900238046894600F034FA34
:108A30000DA3D3E9002304460D464046494600F005
:108A40002BFA8FE702460B465046594600F070F865
:108A5000DDE9022300F020FA03E700BFAFF3008056
:108A60000000E0FE422EE63F763C7935EF39EA3DE4
:108A700010EE103A23F00042B2F1FF4F70B430D242
:108A80006AB3002B3DDBB2F5000F4FEAE3502CD365
:108A9000A0F17F02C3F31603D10743F4000348BFDC
:108AA0005B00002456105B00254619214FF08072B0
:108AB000A818984202DC1B1A8518144401394FEAA1
:108AC00043034FEA5202F3D113B104F001031C44F3
:108AD000641004F17C5404EBC65300EE103A70BCF1
:108AE0007047A0EE000A70BC704713F4000201D07A
:108AF0000CE00A465B001C0202F10101F9D5801A64
:108B0000C6E770EE407A87EEA70AE8E74FF0FF323B
:108B1000F5E700BF002070479FED010B704700BFD5
:108B2000000000000000F87F81F0004102E000BF7B
:108B300083F0004330B54FEA41044FEA430594EA1D
:108B4000050F08BF90EA020F1FBF54EA000C55EA58
:108B5000020C7FEA645C7FEA655C00F0E2804FEA29
:108B60005454D4EB5555B8BF6D420CDD2C4480EA0B
:108B7000020281EA030382EA000083EA010180EA3B
:108B8000020281EA0303362D88BF30BD11F0004F89
:108B90004FEA01314FF4801C4CEA113102D04042BF
:108BA00061EB410113F0004F4FEA03334CEA1333FA
:108BB00002D0524263EB430394EA050F00F0A78012
:108BC000A4F10104D5F1200E0DDB02FA0EFC22FA0D
:108BD00005F2801841F1000103FA0EF2801843FA01
:108BE00005F359410EE0A5F120050EF1200E012AF2
:108BF00003FA0EFC28BF4CF0020C43FA05F3C01830
:108C000051EBE37101F0004507D54FF0000EDCF1A8
:108C1000000C7EEB00006EEB0101B1F5801F1BD351
:108C2000B1F5001F0CD349085FEA30004FEA3C0C55
:108C300004F101044FEA445212F5800F80F09A804B
:108C4000BCF1004F08BF5FEA500C50F1000041EB4F
:108C5000045141EA050130BD5FEA4C0C404141EB53
:108C6000010111F4801FA4F10104E9D191F0000F7A
:108C700004BF01460020B1FA81F308BF2033A3F1FD
:108C80000B03B3F120020CDA0C3208DD02F1140CF4
:108C9000C2F10C0201FA0CF021FA02F10CE002F12F
:108CA0001402D8BFC2F1200C01FA02F120FA0CFC28
:108CB000DCBF41EA0C019040E41AA2BF01EB045171
:108CC000294330BD6FEA04041F3C1CDA0C340EDC6F
:108CD00004F11404C4F1200220FA04F001FA02F3B2
:108CE00040EA030021FA04F345EA030130BDC4F170
:108CF0000C04C4F1200220FA02F001FA04F340EA65
:108D00000300294630BD21FA04F0294630BD94F015
:108D1000000F83F4801306BF81F480110134013DFC
:108D20004EE77FEA645C18BF7FEA655C29D094EA6D
:108D3000050F08BF90EA020F05D054EA000C04BFEB
:108D40001946104630BD91EA030F1EBF00210020D6
:108D500030BD5FEA545C05D14000494128BF41F075
:108D6000004130BD14F580043CBF01F5801130BDD9
:108D700001F0004545F0FE4141F470014FF0000064
:108D800030BD7FEA645C1ABF194610467FEA655C15
:108D90001CBF0B46024650EA013406BF52EA0335B7
:108DA00091EA030F41F4002130BD00BF90F0000FA5
:108DB00004BF0021704730B54FF4806404F13204E1
:108DC0004FF000054FF0000150E700BF90F0000F9A
:108DD00004BF0021704730B54FF4806404F13204C1
:108DE00010F0004548BF40424FF000013EE700BF91
:108DF00042004FEAE2014FEA31014FEA02701FBF21
:108E000012F07F4393F07F4F81F06051704792F0F2
:108E1000000F14BF93F07F4F704730B54FF460746C
:108E200001F0004521F0004120E700BF50EA0102B7
:108E300008BF704730B54FF000050AE050EA010264
:108E400008BF704730B511F0004502D5404261EBD4
:108E500041014FF4806404F132045FEA915C3FF415
:108E6000DCAE4FF003025FEADC0C18BF03325FEAAE
:108E7000DC0C18BF033202EBDC02C2F1200300FA63
:108E800003FC20FA02F001FA03FE40EA0E0021FA88
:108E900002F11444C1E600BF70B54FF0FF0C4CF472
:108EA000E06C1CEA11541DBF1CEA135594EA0C0F28
:108EB00095EA0C0F00F0DEF82C4481EA030621EA63
:108EC0004C5123EA4C5350EA013518BF52EA03359E
:108ED00041F4801143F4801338D0A0FB02CE4FF050
:108EE0000005E1FB02E506F00042E0FB03E54FF080
:108EF0000006E1FB03569CF0000F18BF4EF0010E78
:108F0000A4F1FF04B6F5007F64F5407404D25FEA73
:108F10004E0E6D4146EB060642EAC62141EA555126
:108F20004FEAC52040EA5E504FEACE2EB4F1FD0C68
:108F300088BFBCF5E06F1ED8BEF1004F08BF5FEAE6
:108F4000500E50F1000041EB045170BD06F0004698
:108F500046EA010140EA020081EA0301B4EB5C0445
:108F6000C2BFD4EB0C0541EA045170BD41F480113D
:108F70004FF0000E013C00F3AB8014F1360FDEBF62
:108F8000002001F0004170BDC4F10004203C35DA3E
:108F90000C341BDC04F11404C4F1200500FA05F3C1
:108FA00020FA04F001FA05F240EA020001F0004262
:108FB00021F0004110EBD37021FA04F642EB0601D8
:108FC0005EEA430E08BF20EAD37070BDC4F10C0402
:108FD000C4F1200500FA04F320FA05F001FA04F2C6
:108FE00040EA020001F0004110EBD37041F10001B2
:108FF0005EEA430E08BF20EAD37070BDC4F12005BD
:1090000000FA05F24EEA020E20FA04F301FA05F224
:1090100043EA020321FA04F001F0004121FA04F2CC
:1090200020EA020000EBD3705EEA430E08BF20EA9C
:10903000D37070BD94F0000F0FD101F000464000D6
:1090400041EB010111F4801F08BF013CF7D041EA58
:10905000060195F0000F18BF704703F0004652005C
:1090600043EB030313F4801F08BF013DF7D043EA2D
:109070000603704794EA0C0F0CEA135518BF95EAE3
:109080000C0F0CD050EA410618BF52EA4306D1D16A
:1090900081EA030101F000414FF0000070BD50EA89
:1090A000410606BF1046194652EA430619D094EA13
:1090B0000C0F02D150EA013613D195EA0C0F05D1FD
:1090C00052EA03361CBF104619460AD181EA030151
:1090D00001F0004141F0FE4141F470014FF0000009
:1090E00070BD41F0FE4141F4780170BD70B54FF0A4
:1090F000FF0C4CF4E06C1CEA11541DBF1CEA135524
:1091000094EA0C0F95EA0C0F00F0A7F8A4EB050405
:1091100081EA030E52EA03354FEA013100F08880FC
:109120004FEA03334FF0805545EA131343EA1263C5
:109130004FEA022245EA111545EA10654FEA00267A
:109140000EF000419D4208BF964244F1FD0404F533
:10915000407402D25B084FEA3202B61A65EB03058F
:109160005B084FEA32024FF480104FF4002CB6EB4C
:10917000020E75EB030E22BFB61A754640EA0C00CC
:109180005B084FEA3202B6EB020E75EB030E22BF0C
:10919000B61A754640EA5C005B084FEA3202B6EB4D
:1091A000020E75EB030E22BFB61A754640EA9C000C
:1091B0005B084FEA3202B6EB020E75EB030E22BFDC
:1091C000B61A754640EADC0055EA060E18D04FEA9A
:1091D000051545EA16754FEA06164FEAC30343EA3A
:1091E00052734FEAC2025FEA1C1CC0D111F4801F07
:1091F0000BD141EA00014FF000004FF0004CB6E700
:1092000011F4801F04BF01430020B4F1FD0C88BF9E
:10921000BCF5E06F3FF6AFAEB5EB030C04BFB6EBA9
:10922000020C5FEA500C50F1000041EB045170BD9C
:109230000EF0004E4EEA113114EB5C04C2BFD4EBC9
:109240000C0541EA045170BD41F480114FF0000E4D
:10925000013C90E645EA060E8DE60CEA135594EAC9
:109260000C0F08BF95EA0C0F3FF43BAF94EA0C0FCC
:109270000AD150EA01347FF434AF95EA0C0F7FF441
:1092800025AF104619462CE795EA0C0F06D152EA95
:1092900003353FF4FDAE1046194622E750EA410679
:1092A00018BF52EA43067FF4C5AE50EA41047FF48A
:1092B0000DAF52EA43057FF4EBAE12E74FF0FF3CEF
:1092C00006E000BF4FF0010C02E000BF4FF0010CC0
:1092D0004DF804CD4FEA410C7FEA6C5C4FEA430C39
:1092E00018BF7FEA6C5C1BD001B050EA410C0CBF88
:1092F00052EA430C91EA030F02BF90EA020F0020EA
:10930000704710F1000F91EA030F58BF994208BF50
:1093100090422CBFD8176FEAE37040F0010070470D
:109320004FEA410C7FEA6C5C02D150EA013C07D164
:109330004FEA430C7FEA6C5CD6D152EA033CD3D0AF
:109340005DF8040B704700BF8446104662468C46A9
:109350001946634600E000BF01B5FFF7B7FF0028DC
:1093600048BF10F1000F01BD4DF808EDFFF7F4FF05
:109370000CBF012000205DF808FB00BF4DF808ED90
:10938000FFF7EAFF34BF012000205DF808FB00BFB3
:109390004DF808EDFFF7E0FF94BF012000205DF8D5
:1093A00008FB00BF4DF808EDFFF7CEFF94BF01208A
:1093B00000205DF808FB00BF4DF808EDFFF7C4FF83
:1093C00034BF012000205DF808FB00BF4FEA410CCC
:1093D0007FEA6C5C02D150EA013C0AD14FEA430CAF
:1093E0007FEA6C5C02D152EA033C02D14FF00000EC
:1093F00070474FF0010070474FEA410212F500122A
:1094000015D211D56FF47873B3EB625212D94FEACB
:10941000C12343F0004343EA505311F0004F23FAB5
:1094200002F018BF404270474FF00000704750EA0A
:10943000013005D111F0004008BF6FF000407047C7
:109440004FF00000704700BF4FEA4102B2F1E04325
:1094500024BFB3F5001CDCF1FE5C0DD901F0004C1B
:109460004FEAC0024CEA5070B2F1004F40EB83006B
:1094700008BF20F00100704711F0804F21D113F197
:109480003872BCBF01F00040704741F480114FEAD0
:109490005252C2F11802C2F1200C10FA0CF320FA59
:1094A00002F018BF40F001004FEAC1234FEAD32376
:1094B00003FA0CFC40EA0C0023FA02F34FEA4303E0
:1094C000CCE77FEA625307D150EA01331EBF4FF069
:1094D000FE4040F44000704701F0004040F0FE4084
:1094E00040F40000704700BF53B94AB9002908BFD3
:1094F00000281CBF4FF0FF314FF0FF3000F07EB965
:10950000ADF1080C6DE904CE00F006F8DDF804E0DA
:10951000DDE9022304B070472DE9F0478C460E4682
:109520000446089D002B50D18A4217466CD9B2FAE6
:1095300082FEBEF1000F0BD0CEF1200420FA04F41D
:1095400001FA0EF644EA060C02FA0EF700FA0EF4DF
:109550004FEA1749220CBCFBF9F01FFA87F809FB08
:1095600010C642EA064600FB08F3B34209D9F619D1
:1095700000F1FF3280F02281B34240F21F810238B5
:109580003E44F61AA2B2B6FBF9F309FB136642EAAF
:10959000064403FB08F8A04509D9E41903F1FF329A
:1095A00080F00A81A04540F20781023B3C44C8EBB1
:1095B000040443EA00400021002D62D024FA0EF496
:1095C00000232C606B60BDE8F0878B4207D9002D2B
:1095D00055D0002185E841000846BDE8F087B3FA80
:1095E00083F1002940F09080B34202D3824200F21E
:1095F000F880841A66EB03060120B446002D40D0A3
:1096000085E81010BDE8F08712B90127B7FBF2F723
:10961000B7FA87FEBEF1000F35D1F31B4FEA1748AA
:109620001FFA87FC0121B3FBF8F0220C08FB10366F
:1096300042EA06460CFB00F3B34207D9F61900F1E3
:10964000FF3202D2B34200F2CE801046F61AA2B226
:10965000B6FBF8F308FB136642EA06440CFB03FC76
:10966000A44507D9E41903F1FF3202D2A44500F260
:10967000B5801346CCEB040443EA00409CE729463E
:109680002846BDE8F087CEF1200106FA0EF307FA6E
:109690000EF720FA01F94FEA1748CE4049EA0309CC
:1096A000B6FBF8FA4FEA194408FB1A661FFA87FC62
:1096B00044EA06430AFB0CF29A4200FA0EF40AD975
:1096C000DB190AF1FF3180F087809A4240F28480F2
:1096D000AAF1020A3B449B1A1FFA89F9B3FBF8F17D
:1096E00008FB113349EA034301FB0CF69E4207D9FC
:1096F000DB1901F1FF326BD29E4269D902393B443A
:109700009B1B41EA0A418EE7C1F1200E22FA0EF4BA
:109710008B40234320FA0EF706FA01F44FEA134C6C
:1097200026FA0EF63C43B6FBFCF9270C0CFB196637
:109730001FFA83F847EA064609FB08F7B74202FA20
:1097400001F200FA01FA08D9F61809F1FF3041D206
:10975000B7423FD9A9F102091E44F61BA0B2B6FBDD
:10976000FCF40CFB146640EA064704FB08F8B84515
:1097700007D9FF1804F1FF3028D2B84526D9023C9A
:109780001F4444EA0940C8EB0707A0FB02894F4584
:1097900044464E4614D329D065B3BAEB040367EBB5
:1097A000060707FA0EFECB40CF404EEA030385E8DA
:1097B00088000021BDE8F0871346F8E61046E0E691
:1097C000B8EB020469EB03060138E5E70446D8E785
:1097D000114695E78146C0E78A467CE7023B3C4458
:1097E00048E708460AE702383E442FE7C245E7D378
:1097F0003E46D1E72946BDE8F08700BF704700BF6D
:10980000014B1868704700BF88040020844641EA75
:10981000000313F003036DD1403A41D351F8043BE8
:1098200040F8043B51F8043B40F8043B51F8043B3A
:1098300040F8043B51F8043B40F8043B51F8043B2A
:1098400040F8043B51F8043B40F8043B51F8043B1A
:1098500040F8043B51F8043B40F8043B51F8043B0A
:1098600040F8043B51F8043B40F8043B51F8043BFA
:1098700040F8043B51F8043B40F8043B51F8043BEA
:1098800040F8043B51F8043B40F8043B51F8043BDA
:1098900040F8043B51F8043B40F8043B403ABDD249
:1098A000303211D351F8043B40F8043B51F8043BEB
:1098B00040F8043B51F8043B40F8043B51F8043BAA
:1098C00040F8043B103AEDD20C3205D351F8043B7A
:1098D00040F8043B043AF9D2043208D0D2071CBF46
:1098E00011F8013B00F8013B01D30B88038060466F
:1098F000704700BF082A13D38B078DD010F00303E5
:109900008AD0C3F10403D21ADB071CBF11F8013B54
:1099100000F8013B80D331F8023B20F8023B7BE7A3
:10992000043AD9D3013A11F8013B00F8013BF9D2CE
:109930000B7803704B7843708B7883706046704768
:109940000CB4F0B59DB022AC029154F8042B0691F2
:1099500023466FF000454FF402774FF6FF7602A9D9
:109960000194ADF8147004950795ADF8166000F0F9
:1099700045FA029B00221A701DB0BDE8F04002B00B
:10998000704700BF0EB4F0B59CB021AB0F4953F83F
:10999000042B019305466FF00044086802954FF4CC
:1099A00002774FF6FF7602A90695ADF8147004947D
:1099B0000794ADF8166000F021FA029B00221A709D
:1099C0001CB0BDE8F04003B0704700BF8804002021
:1099D00080EA0102844612F0030F4FD111F0030F09
:1099E00032D14DF8044D11F0040F51F8043B0BD067
:1099F000A3F101329A4312F0803F04BF4CF8043BBC
:109A000051F8043B16D100BF51F8044BA3F10132C9
:109A10009A4312F0803FA4F101320BD14CF8043B81
:109A2000A24312F0803F04BF51F8043B4CF8044BB2
:109A3000EAD023460CF8013B13F0FF0F4FEA332323
:109A4000F8D15DF8044B704711F0010F06D011F802
:109A5000012B0CF8012B002A08BF704711F0020FF0
:109A6000BFD031F8022B12F0FF0F16BF2CF8022BDB
:109A70008CF8002012F47F4FB3D1704711F8012BFE
:109A80000CF8012B002AF9D1704700BF000000003C
:109A900000000000000000000000000000000000C6
:109AA00000000000000000000000000000000000B6
:109AB00000000000000000000000000000000000A6
:109AC00090F800F06DE9024520F007016FF0000CFE
:109AD00010F0070491F820F040F049804FF00004A6
:109AE0006FF00700D1E9002391F840F000F1080081
:109AF00082FA4CF2A4FA8CF283FA4CF3A2FA8CF3B9
:109B00004BBBD1E9022382FA4CF200F10800A4FA1F
:109B10008CF283FA4CF3A2FA8CF3E3B9D1E9042373
:109B200082FA4CF200F10800A4FA8CF283FA4CF3AA
:109B3000A2FA8CF37BB9D1E9062301F1200182FA64
:109B40004CF200F10800A4FA8CF283FA4CF3A2FA6A
:109B50008CF3002BC6D0002A04BF04301A4612BA78
:109B6000B2FA82F2FDE8024500EBD2007047D1E97B
:109B7000002304F00305C4F100004FEAC50514F00A
:109B8000040F91F840F00CFA05F562EA05021CBFDB
:109B900063EA050362464FF00004A9E770B5002AA6
:109BA0009AB005462FDB14461A464FF40273009113
:109BB0000491ADF80C3011D0013C4FF6FF761E9B9E
:109BC000029469460594ADF80E6000F017F9421C46
:109BD00012DB009B00221A701AB070BD1E9B02940B
:109BE0004FF6FF7669460594ADF80E6000F006F971
:109BF000431C04DB1AB070BD8B232B60E9E78B2379
:109C00002B601AB070BD8B2303604FF0FF30F1E77B
:109C100010B582B0054C0093246813460A460146ED
:109C20002046FFF7BBFF02B010BD00BF8804002034
:109C30002DE9F84F8E689E420C461F46904629D863
:109C40008B8913F4906F35D04D692268096905EB53
:109C50004505C1EB020A814605EBD5750AF1010005
:109C60006D103844A8422A4684BF05462A465B0543
:109C700023D51146484600F0BDFC834690B35246BA
:109C80002169FFF7C3FDA38923F4906343F08003A8
:109C9000A38117E008681E461D462A46414600F08B
:109CA000FFFBA36822689E1B1544A6602560002068
:109CB000BDE8F88F35460868EFE7484600F0F8FC45
:109CC000834658B1CAEB05030BEB0A0065613E46BB
:109CD000C4F810B02060A3603D46DEE72169484625
:109CE00000F042FC0C23C9F80030A38943F0400384
:109CF000A3814FF0FF30BDE8F88F00BF2DE9F04F92
:109D0000936883B09046002B72D083464FF00009D1
:109D1000166808688B680D464C46002C45D09C425E
:109D20001F469A4646D3AB8913F4906F2DD06F69C6
:109D3000296907EB4707C1EB000A07EBD777601CDF
:109D40007F105044B8423A4684BF07463A465B0506
:109D500033D51146584600F04DFC002837D0524606
:109D600029690190FFF752FDAA89019B22F49062B4
:109D700042F08002AA81CAEB070203EB0A006F617E
:109D80002B612860AA602746A2465246494600F049
:109D900087FBD8F80820AB682868DB1B5044141BED
:109DA000AB602860C8F8084014B3D6F80090746817
:109DB0000836B2E72746A246E7E7584600F078FCA7
:109DC00003460028D7D12969584600F0CDFB0C2363
:109DD000CBF80030AB89002243F040034FF0FF3056
:109DE000AB81C8F80820C8F8042003B0BDE8F08FA4
:109DF0000020C8F8040003B0BDE8F08F2DE9F04F53
:109E000014468A899DB0150688460393814603D57A
:109E10000B69002B00F0EC8030238DF82A3023787A
:109E20007C4DDFF8F4A10021202209918DF8292032
:109E3000002B00F08580252B264603D117E0252B2B
:109E400000F0888016F8013F002BF8D1B6EB040B28
:109E500076D022465B4641464846FFF7E9FE013090
:109E60006ED0099B32785B440993002A68D00023A6
:109E70004FF0FF31721C0493079306938DF8533013
:109E80001A930591012604E0049906FA03F30B43A3
:109E9000049314465F482178052200F0B1FA621C51
:109EA000431B0028F0D1049BD80644BF20228DF824
:109EB00053201907217844BF2B228DF853202A29DB
:109EC0006AD0A1F13002092A0BD8079B14F8011FB0
:109ED00003EB830302EB4303A1F13002092AF5D916
:109EE00007932E2941D003224B4800F089FA48B14C
:109EF0000499CAEB0000402202FA00F041EA000394
:109F000001340493217845488DF828100622013445
:109F100000F076FA002861D0414BFBB103AB00930F
:109F20004246404B04A94846AFF3008007467A1CDE
:109F300006D0099B3B4409932378002B7FF47BAF29
:109F4000B8F80C305B0654BF09984FF0FF301DB0D5
:109F5000BDE8F08FB6EB040B89D07AE7039B07339B
:109F600023F0070308330393E3E761782A291DD020
:109F7000A1F130020023092A04F101040593B2D8AB
:109F800014F8011F03EB830302EB4303A1F130023A
:109F9000092AF5D90593A6E7039A11680432002926
:109FA000039215DB0791617801349AE7039B1A68E5
:109FB0000592002A03F104030393B8BF4FF0FF3268
:109FC00004F10203AEBFA178A17805921C468AE78E
:109FD000494243F0020307910493E4E703AB009383
:109FE0004246104B04A9484600F0B6F807469EE7E3
:109FF000402100F0FFFAC8F80000C8F8100018B1BE
:10A000004023C8F8143007E70C23C9F800304FF09C
:10A01000FF309CE7C06F0108C86F0108CC6F0108D2
:10A0200000000000319C00082DE9F0470C469146E5
:10A030000969A268DDF820808A42B8BF0A46C9F8DB
:10A04000002094F8431006461F4611B10132C9F8AA
:10A050000020236899065DD5D9F800200232C9F89E
:10A060000020236813F0060F19461DD1E1688A1AF3
:10A07000002AD8BF194617DD04F1190A002505E0AA
:10A08000E368D9F800209B1AAB420CDD012352464D
:10A0900039463046C047013005F10105F0D14FF097
:10A0A000FF30BDE8F087216894F84330003318BFD3
:10A0B00001238A060AD5E1185A1C302081F8430092
:10A0C000224494F8451082F84310023304F143020D
:10A0D00039463046C0470130E1D0236803F006031B
:10A0E000042B29D0A36822699342C8BF4FF000090E
:10A0F0002FDD9B1A99441A34002501E04D4528D0E4
:10A100000123224639463046C047013005F101059A
:10A11000F4D1C4E713F0060F08D1E168D9F80020A4
:10A120008A1A002AD8BF1946A6DCBDE794F8433046
:10A13000003318BF0123C9E7D9F80000E168A3681C
:10A140002269091A934221EAE179D2DCB9F1000FC0
:10A15000D1D10020BDE8F0872DE9F0430C46097EFF
:10A1600085B06E29064617460C98984604F1430CB4
:10A170005AD01AD8632900F0128100F2D680002943
:10A180005CD0582940F0F58084F8451022680368B7
:10A19000DFF864E2150603F104011ED4550653BF2F
:10A1A0001B6801601B88016019E0732900F0CF80F3
:10A1B0007ED86F2900F0E480702940F0DA802268B0
:10A1C00042F020022260782384F845300368DFF8EB
:10A1D0002CE2150603F10401E0D51B680160D007ED
:10A1E00044BF42F020022260002B40F090802268A1
:10A1F00022F0200222601021002284F843206068AF
:10A20000A0600028C0F28880226822F00402226048
:10A21000002B62D1002840F08180654608296AD071
:10A22000C5EB0C0323610CE023681A0640F1D580CE
:10A2300003686269191D01601B681A600023654686
:10A240002361CDF800803B4603AA21463046FFF744
:10A25000EBFE013021D02A46236939463046C047FB
:10A2600001301AD02368039813F0020FE36819D065
:10A270001A1A002A16DD04F11909002504E0E36822
:10A2800003981A1AAA420DDD01234A463946304680
:10A29000C047013005F10105F1D14FF0FF3005B0A5
:10A2A000BDE8F0839842B8BF184605B0BDE8F0831A
:10A2B000752965D078295CD1226884E76168A1603E
:10A2C0002D200029C3F1000384F8430021DB22F094
:10A2D0000402DFF824E122600A216546B3FBF1F2B3
:10A2E00001FB123013461EF8002005F8012D002B4B
:10A2F000F4D1082994D12368D90791D562682369DC
:10A300009A428DDC302305F8013C013D88E710219D
:10A3100072E7DFF8E4E00A21002BDED19EF800307E
:10A3200084F8423004F1420578E7642901D06929B4
:10A330001FD122680368150603F104013AD51B6892
:10A340000160002BBADBDFF8B0E00A2157E70368B1
:10A350006268191D01601D680021284600F050F850
:10A36000002846D0401B60602061002384F8433001
:10A3700067E7012384F84210236104F14205F4E702
:10A3800023681A061ED503681A1D1B680260227E08
:10A39000DFF864E06F2A14BF0A2108212CE7036864
:10A3A0001A68191D0123016004F1420584F8422056
:10A3B0002361DAE7550653BF1B680160B3F900302B
:10A3C0000160BEE713F0400F036803F1040215BFFC
:10A3D00002601B681B880260D9E713F0400F036816
:10A3E000626903F1040101601B6814BF1A801A60DE
:10A3F00024E76068B8E700BFD46F0108E86F010880
:10A4000001F0FF01102A2BDB10F0070F08D010F825
:10A41000013B013A8B422DD010F0070F42B3F6D129
:10A42000F0B441EA012141EA014122F007047FF042
:10A4300000070023F0E80256083C85EA010586EA99
:10A44000010685FA47F5A3FA87F586FA47F6A5FAD5
:10A4500087F68EB9EED1F0BC01F0FF0102F00702E1
:10A4600032B110F8013B013A83EA010313B1F8D18C
:10A470000020704701387047002D06BF354603386D
:10A48000073815F0010F07D1013015F4807F02BFA6
:10A49000013015F4C03F0130F0BC0138704700BFF7
:10A4A0008842F0B50DD98B1898420AD28118002A3B
:10A4B00051D09A1A13F8014D01F8014D9342F9D188
:10A4C000F0BD0F2A48D941EA00039B0746D100F1AD
:10A4D000100401F11003154653F8106C44F8106C89
:10A4E00053F80C6C44F80C6C53F8086C44F8086C86
:10A4F000103D53F8046C44F8046C0F2D03F1100365
:10A5000004F11004E8D8A2F1100323F00F0302F0C5
:10A510000F0E1033BEF1030F1944034421D91E1F3F
:10A520000D467446043C55F8047B46F8047F032C22
:10A53000F8D8AEF1040424F0030404342344214485
:10A5400002F0030262B1013B0A4411F8014B03F827
:10A55000014F8A42F9D1F0BD0346F3E70346F2E723
:10A56000F0BD7246EEE700BF30B481B151F8043C53
:10A570000439002BB8BFC9181D4B1A682AB18A428A
:10A580000AD908680C18A24225D04A60196030BC6C
:10A5900070478B4203D81A465368002BF9D11468D0
:10A5A00015198D420CD007D808680C189C4218D099
:10A5B0004B6030BC516070470C23036030BC704767
:10A5C00009680C44111999421460E0D10ACB0C447B
:10A5D00053601460DBE7146852684A6020440860E6
:10A5E000D4E71C685B684B60204408605160CEE78C
:10A5F000080A002070B5CD1C25F0030508350C2D88
:10A6000038BF0C25002D06463BDBA94239D8274927
:10A610000A6852B113685B1B04D436E023685B1BE5
:10A620001AD522465468002CF8D149681F4C0029DD
:10A6300036D02946304600F05FF8431C21D0C41CB8
:10A6400024F00304A04205D0211A304600F054F84B
:10A65000013016D0256004E00B2B0DD923601C447B
:10A66000256004F10B0020F00700231DC31A02D05F
:10A670005A42E25070BD70BD94420ED06368536080
:10A68000EFE70C233360002070BD0B2B03D8536819
:10A6900014460B60E5E71446E0E713461446F8E776
:10A6A000304600F029F86060C3E700BF080A0020C8
:10A6B000F9B1F8B506461546B2B10C4600F02EF8D1
:10A6C000854201D82046F8BD29463046FFF792FF63
:10A6D000074668B12A462146FFF798F830462146DA
:10A6E000FFF742FF3846F8BDFFF73EFF2846F8BDAA
:10A6F000F8BD1146FFF77EBF38B5074C002305466D
:10A7000008462360F9F7D0F9431C00D038BD236810
:10A71000002BFBD02B6038BD100A002051F8040C30
:10A720000028BEBF091851F8043CC018043870470F
:10A730002E2E2F73797374656D2F7372632F73745C
:10A740006D333266372D68616C2F73746D333266EA
:10A750003778785F68616C5F6164632E6300000026
:10A760002E2E2F73797374656D2F7372632F73742C
:10A770006D333266372D68616C2F73746D333266BA
:10A780003778785F68616C5F636F727465782E6389
:10A79000000000002E2E2F73797374656D2F737275
:10A7A000632F73746D333266372D68616C2F737449
:10A7B0006D3332663778785F68616C5F6461632EF1
:10A7C000630000002E2E2F73797374656D2F7372E2
:10A7D000632F73746D333266372D68616C2F737419
:10A7E0006D3332663778785F68616C5F6770696F68
:10A7F0002E6300002E2E2F73797374656D2F737284
:10A80000632F73746D333266372D68616C2F7374E8
:10A810006D3332663778785F68616C5F6932632EBA
:10A8200063000000000000000102030401020304B1
:10A83000060708092E2E2F73797374656D2F7372B6
:10A84000632F73746D333266372D68616C2F7374A8
:10A850006D3332663778785F68616C5F7263632E40
:10A86000630000002E2E2F73797374656D2F737241
:10A87000632F73746D333266372D68616C2F737478
:10A880006D3332663778785F68616C5F7263635FDF
:10A8900065782E63000000002E2E2F737973746587
:10A8A0006D2F7372632F73746D333266372D686149
:10A8B0006C2F73746D3332663778785F68616C5FC4
:10A8C0007370692E630000002E2E2F7379737465E8
:10A8D0006D2F7372632F73746D333266372D686119
:10A8E0006C2F73746D3332663778785F68616C5F94
:10A8F00074696D2E6300000061626F727428292CE8
:10A900002065786974696E672E2E2E002C2066757E
:10A910006E6374696F6E3A200000000061737365A6
:10A920007274696F6E2022257322206661696C65DE
:10A93000643A2066696C6520222573222C206C699C
:10A940006E65202564257325730A000061737365A5
:10A9500072745F706172616D2829206661696C652F
:10A96000643A2066696C6520222573222C206C696C
:10A970006E652025640A00000A0000006D61696EA2
:10A9800028617267633D25642C20617267763D5BA8
:10A99000000000002C20000022257322000000008F
:10A9A0005D293B0A00000000537461636B206672EE
:10A9B000616D653A0A000000205230203D202025BC
:10A9C0003038580A00000000205231203D20202558
:10A9D0003038580A00000000205232203D20202547
:10A9E0003038580A00000000205233203D20202536
:10A9F0003038580A0000000020523132203D202516
:10AA00003038580A00000000204C52203D202025FC
:10AA10003038580A00000000205043203D202025F7
:10AA20003038580A0000000020505352203D2025A5
:10AA30003038580A000000004653522F4641523A1F
:10AA40000A0000002043465352203D202025303884
:10AA5000580A00002048465352203D202025303817
:10AA6000580A00002044465352203D20202530380B
:10AA7000580A00002041465352203D2020253038FE
:10AA8000580A0000204D4D464152203D20253038C7
:10AA9000580A00002042464152203D2020253038EF
:10AAA000580A00004D6973630A000000204C522FC1
:10AAB0004558435F52455455524E3D202530385835
:10AAC0000A0000005B486172644661756C745D0A3F
:10AAD000000000005B4275734661756C745D0A008E
:10AAE0005B55736167654661756C745D0A000000B3
:10AAF000000000000000000001020304060708092E
:10AB000000100240800000000010024040000000E1
:10AB1000001002400200000000040240400000005B
:10AB2000000402400002000000080240080000008B
:10AB30000004024000200000000402400008000061
:10AB40000010024000040000000C02400001000060
:10AB5000001002400400000000100240002000002D
:10AB60000010024001000000000402400400000048
:10AB700000000240800000000008024002000000C7
:10AB800000000240400000000004024008000000F5
:10AB9000000402408000000000000240008000002D
:10ABA00000040240200000000010024008000000E5
:10ABB000000C0240200000000010024010000000C5
:10ABC000000C024080000000001002402000000045
:10ABD000000C024040000000000C02400800000091
:10ABE0000004024010000000000402400080000049
:10ABF00000040240000400000000024001000000C8
:10AC000000000000EF7BFFFFFFFFFFFFFFFFFFFFE4
:10AC1000FFFFFFFFFFFFFFFFFFFFFFFFFFFFFFFF44
:10AC2000FFFFFFFFFFFFFFFFFFFFFFFFFFFFFFFF34
:10AC3000FFFFFFFFFFFFFFFFFFFFFFFFFFFFFFFF24
:10AC4000FFFFFFFFFFFFFFFFFFFFFFFFFFFFFFFF14
:10AC5000FFFFFFFFFFFFFFFFEF7B00000000000092
:10AC6000FFFFFFFFFFFFFFFFFFFFFFFFFFFFFFFFF4
:10AC7000FFFFFFFFFFFFFFFFFFFFFFFFFFFFFFFFE4
:10AC8000FFFFFFFFFFFFFFFFFFFFFFFFFFFFFFFFD4
:10AC9000FFFFFFFFFFFFFFFFFFFFFFFFFFFFFFFFC4
:10ACA000FFFFFFFFFFFFFFFFFFFFFFFFFFFFFFFFB4
:10ACB000FFFFFFFFFFFFFFFFFFFF0000EF7BFFFF36
:10ACC00030FE000000000000000000003C5514FFB2
:10ACD00000500A001FA730FE00000A001FA7FFFF58
:10ACE000FFFFFFFF00C400000000000000000000A4
:10ACF0000000180414FF00500000000000000000D5
:10AD000000003F86F8FF0080000000000000000007
:10AD100000003C55FFFFFFFFEF7BFFFFFFFF30FE12
:10AD2000000000000000000000003C5514FF00502F
:10AD30000A001FA730FE00000A001FA7FFFFFFFF49
:10AD4000FFFF00C400000000000000000000000041
:10AD5000180414FF00500000000000000000000074
:10AD60003F86F8FF008000000000000000000000A7
:10AD70000A001FA7FFFFFFFFFFFFFFFF30FE0000DD
:10AD80000A001FA7FFFFFFFFFFFF14FF00500A008C
:10AD90001FA730FE00000A001FA7FFFFFFFFFFFFF5
:10ADA000FFFFFFFF14FF00500A001FA7FFFFFFFF78
:10ADB00014FF005000003F86FFFFFFFFFFFFFFFF73
:10ADC000F8FF008000003C55FFFF14FF005000001A
:10ADD0003F86FFFFFFFFFFFFFFFF30FE0000000088
:10ADE000000000001000FFC714FF00500A001FA75A
:10ADF00030FE00000A001FA7FFFFFFFFFFFFFFFF5D
:10AE0000FFFF14FF00500A001FA7FFFFFFFF14FF02
:10AE1000005000000000000000000A001FA7F8FF1B
:10AE20000080000000000000000000001000FFC7CC
:10AE3000FFFFFFFFFFFFFFFF30FE000000000000EC
:10AE400000001000FFC714FF00500A001FA730FECB
:10AE500000000A001FA7FFFFFFFFFFFFFFFFFFFF2C
:10AE600014FF00500A001FA7FFFFFFFF14FF005050
:10AE700000000000000000000A001FA7F8FF00808B
:10AE80000000000000000000B402FFE7FFFFFFFF2A
:10AE9000FFFFFFFFFFFF30FE00000A001FA7FFFFBC
:10AEA000FFFFFFFF14FF00500A001FA730FE000045
:10AEB0000A001FA7FFFFFFFFFFFFFFFFFFFF14FFB9
:10AEC00000500A001FA7FFFFFFFF14FF0050000003
:10AED0003F86FFFFFFFFFFFFFFFFF8FF008000003E
:10AEE0003C5530FE000000003C55FFFFFFFFFFFF18
:10AEF000FFFFFFFF30FE00000A001FA7FFFFFFFF5C
:10AF0000FFFF14FF00500A001FA730FE00000000E2
:10AF10000000000000001804FFFFFFFF14FF0050B6
:10AF20000A001FA7FFFFFFFF14FF005000000000F2
:10AF30000000000000003C55F8FF008000003C5578
:10AF4000FCFFA0A200000A001FA7FFFFFFFFEF7B8E
:10AF5000FFFF30FE00000A001FA7FFFFFFFFFFFFFB
:10AF600014FF00500A001FA730FE00000000000080
:10AF7000000000001804FFFFFFFF14FF00500A004C
:10AF80001FA7FFFFFFFF14FF00500000000000009C
:10AF9000000000003C55F8FF008000003C55FFFF1A
:10AFA00014FF00500000B402FFFFEF7B0000FFFF22
:10AFB000FFFFFFFFFFFFFFFFFFFFFFFFFFFFFFFFA1
:10AFC000FFFFFFFFFFFFFFFFFFFFFFFFFFFFFFFF91
:10AFD000FFFFFFFFFFFFFFFFFFFFFFFFFFFFFFFF81
:10AFE000FFFFFFFFFFFFFFFFFFFFFFFFFFFFFFFF71
:10AFF000FFFFFFFFFFFFFFFFFFFFFFFFFFFFFFFF61
:10B00000FFFFFFFFFFFFFFFF000000000000EF7BDE
:10B01000FFFFFFFFFFFFFFFFFFFFFFFFFFFFFFFF40
:10B02000FFFFFFFFFFFFFFFFFFFFFFFFFFFFFFFF30
:10B03000FFFFFFFFFFFFFFFFFFFFFFFFFFFFFFFF20
:10B04000FFFFFFFFFFFFFFFFFFFFFFFFFFFFFFFF10
:10B05000FFFFFFFFFFFFFFFFFFFFFFFFFFFFFFFF00
:10B06000FFFFEF7B000000003C55FFFFFFFFFFFFED
:10B07000FFFFFFFFFFFF2AE53C55FFFFFFFFFFFF3C
:10B08000FFFFFFFFFFFF2AE50000000000000000B7
:10B090003C55FFFF30FE0000000000000000B4023D
:10B0A000FFE7F8FF00800000000000000A001FA773
:10B0B000FFFF2AE50000000000000000B402FFE7E7
:10B0C000F8FF008000000000000000003C55FFFF7A
:10B0D00014FF00500000000000000A001FA7FFFF3F
:10B0E0002AE500000000000000001000FFC7FFFF7D
:10B0F00000C4000000000000070009000A000B0067
:10B100000C000D000D000E000E100F180F20102067
:10B1100010281128113011301138114012481250E6
:10B12000125812601260126812681270127812803F
:10B1300012881290129012901298139813A013A0D4
:10B1400012A011A811B012B012B011B811B830C0CD
:10B1500030B850C08FC08FC08FC08FC0AEC8CDC8B0
:10B16000CDC80CC92CD14AD969D187D186D1C5D9CE
:10B17000C3D9E2D902DA21E241E260E260E2A0E270
:10B18000A0EAA0E2C0E2E0EAE0EA00EB20EB40F354
:10B1900060F380EB80EB80F3C0F3E0F300F420F485
:10B1A00020F440F460FC80FCC0FCC0FCE0FCE0FC4F
:10B1B00000FD40FD60FD80FD60F580F5C0F5E0F527
:10B1C00000FE20F640F620F640F660F6A1FEA1FE55
:10B1D000A2F6C3FEE4FEE5F606F728FF29FF2AFFE4
:10B1E0002BF74EFF90FF92FF93FF95F797F7B8FF6D
:10B1F000B9F7BAF7DCFFDEFF000000000000000036
:10B200000C00FFB7FFFFFFFFFFFFFBFFC091000037
:10B210000000000000000000000000009B3CFFFF59
:10B22000FFFFFFFFFFFFFFFFFFFFFFFFD2FE003822
:10B2300000000000000000009B3CFFFFFFFFFFFF3D
:10B24000FFFFFFFFFFFFFFFFFFFFFFFFACFD000061
:10B25000000000000C00FFB7FFFFFFFFFBFFC091E5
:10B2600000000700DF96FFFFFFFFFFFF20B3000095
:10B2700000003603FFFFFFFFFFFF20B300000000C8
:10B280000000D201FFDFFFFFFFFFACFD0000000068
:10B290003603FFFFFFFFFBFFC0910000000000002E
:10B2A0000700DF96FFFFFFFFACFD00000000360344
:10B2B000FFFFFFFFFFFF20B30000000000000C00B5
:10B2C000FFB7FFFFFFFFACFD000000000C00FFB761
:10B2D000FFFFFFFFFBFFC09100000700DF96FFFFAD
:10B2E000FFFFFFFF20B30000000000009B3CFFFFBA
:10B2F000FFFFFFFFFFFFFFFFFFFFFFFFFFFFFFFF5E
:10B30000D2FE003800000000000000009B3CFFFF60
:10B31000FFFFFFFFFFFFFFFFFFFFFFFFFFFF20B368
:10B320000000000000000000000000000C00FFB75B
:10B33000FFFFFFFFFFFFFFFFFFFFACFD000000006E
:10B3400000000000000000000000000000000000FD
:10B35000BF65FFFFFFFFFBFFC09100000000000082
:10B360000000000000000000000000003603FFFFA6
:10B37000FFFFFFFFACFD0000000000000000000028
:10B3800000000000000000000700DF96FFFFFFFF45
:10B39000FBFFC09100000000000000000000000062
:10B3A0000000000000003603FFFFFFFFFFFFACFDC1
:10B3B000000000000000000000000000000000008D
:10B3C00000000700DF96FFFFFFFFFBFFC0910000BA
:10B3D000000000000000000000000000000000006D
:10B3E0003603FFFFFFFFFFFF87DC000000000000C7
:10B3F0000000000000000000000000000700DF96D1
:10B40000FFFFFFFFF6FF00600000000000000000EB
:10B410000000000000000000000000000000070025
:10B42000DF9687DC00000000000000000000000044
:10B430000000000000000000EF7BFFFFFFFFFFFFA8
:10B44000FFFFFFFFFFFFFFFFFFFFFFFFFFFFFFFF0C
:10B45000FFFFFFFFFFFFFFFFFFFFFFFFFFFFFFFFFC
:10B46000FFFFFFFFFFFFFFFFFFFFFFFFFFFFFFFFEC
:10B47000FFFFFFFFFFFFFFFFFFFFFFFFFFFFEF7B70
:10B48000000000000000FFFFFFFFFFFFFFFFFFFFC6
:10B49000FFFFFFFFFFFFFFFFFFFFFFFFFFFFFFFFBC
:10B4A000FFFFFFFFFFFFFFFFFFFFFFFFFFFFFFFFAC
:10B4B000FFFFFFFFFFFFFFFFFFFFFFFFFFFFFFFF9C
:10B4C000FFFFFFFFFFFFFFFFFFFFFFFFFFFFFFFF8C
:10B4D000FFFF0000EF7BFFFFACFD000000000C0051
:10B4E000FFB7F6FF006000000000BF65FFFFFFFF31
:10B4F00020B3000000000000D201FFDFFFFFF6FFD5
:10B5000000600000000000000000D201FFDFFFFF2C
:10B51000D2FE003800000000000000000000BF65FF
:10B52000FFFFEF7BFFFFFFFFACFD00000000070007
:10B53000DF96D2FE003800000000BF65FBFFC0911F
:10B5400000000000000000000000D201FFDFF6FF55
:10B55000006000000000000000000000D201FFDFDA
:10B56000D2FE003800000000000000000000BF65AF
:10B57000FFFFFFFFFFFFFFFFACFD0000000000002A
:10B580009B3CACFD0700C0390000BF65ACFD00006E
:10B590000000BF65FFFFACFD00000000BF65F6FFC7
:10B5A000006000009B3CFFFFACFD00000700DF9641
:10B5B000D2FE00380000BF65FFFFFFFFFFFFFFFF67
:10B5C000FFFFFFFFFFFFFFFFACFD0000CC01C061EC
:10B5D000360320B30C0020630000BF6587DC000049
:10B5E0000C00FFB7FFFFFBFFC09100009B3CF6FF84
:10B5F000006000009B3CFFFFF6FF00600000BF659D
:10B60000D2FE003800000000000000000700DF96B6
:10B61000FFFFFFFFFFFFFFFFACFD0000D201209303
:10B620000700C039360320B30000BF6587DC000087
:10B630000C00FFB7FFFFFBFFC09100009B3CF6FF33
:10B64000006000009B3CFFFFF6FF00600000BF654C
:10B65000D2FE003800000000000000000700DF9666
:10B66000FFFFFFFFFFFFFFFFACFD0000D20187B42B
:10B67000000000009B3C20B30000BF65ACFD000053
:10B680000000BF65FFFFACFD00000000BF65F6FFD6
:10B69000006000009B3CFFFFACFD00000000BF65A8
:10B6A000D2FE00380000BF65FFFFFFFFFFFFFFFF76
:10B6B000FFFFFFFFFFFFFFFFACFD0000D201D2DE66
:10B6C00000380000BF6520B30000BF65FBFFC091DC
:10B6D00000000000000000000000D201FFDFF6FFC4
:10B6E000006000000000000000000000D201FFDF49
:10B6F000D2FE0038000000000000000000009B3C6B
:10B70000FFFFFFFFEF7BFFFFACFD0000D201F6DF84
:10B7100000600C00FFB720B30000BF65FFFFFFFF14
:10B7200020B3000000000000D201FFDFFFFFF6FFA2
:10B7300000600000000000000000D201FFDFFFFFFA
:10B74000D2FE0038000000000000000000009B3C1A
:10B75000FFFFEF7B0000FFFFFFFFFFFFFFFFFFFF8B
:10B76000FFFFFFFFFFFFFFFFFFFFFFFFFFFFFFFFE9
:10B77000FFFFFFFFFFFFFFFFFFFFFFFFFFFFFFFFD9
:10B78000FFFFFFFFFFFFFFFFFFFFFFFFFFFFFFFFC9
:10B79000FFFFFFFFFFFFFFFFFFFFFFFFFFFFFFFFB9
:10B7A000FFFF000000000000EF7BFFFFFFFFFFFF37
:10B7B000FFFFFFFFFFFFFFFFFFFFFFFFFFFFFFFF99
:10B7C000FFFFFFFFFFFFFFFFFFFFFFFFFFFFFFFF89
:10B7D000FFFFFFFFFFFFFFFFFFFFFFFFFFFFFFFF79
:10B7E000FFFFFFFFFFFFFFFFFFFFFFFFFFFFEF7BFD
:10B7F0000000000000003603FFFFFFFFFFFFFFFF18
:10B80000FFFFFFFFFFFFFFFFFFFFFFFFFFFFFBFF4C
:10B81000C09100003603FFFFFFFFFFFFFFFFFFFFA8
:10B82000FFFFFFFFFFFFFFFFFFFFFFFFFBFFC091D9
:10B8300000003603FFFFFFFFFFFFFFFFFFFFFFFFDB
:10B84000FFFFFFFFFFFFFFFFFFFFD2FE00380000FA
:10B8500000000000000000000000000000000000E8
:10B860009B3CFFFFFFFFFFFF20B300000000000034
:10B870000000000000000000000000000C00FFB706
:10B88000FFFFFFFFD2FE00380000000000000000B4
:10B89000000000000000000000009B3CFFFFFFFFD5
:10B8A000FFFF20B3000000000000000000000000C7
:10B8B0000000000000000C00FFB7FFFFFFFFD2FEFA
:10B8C0000038000000000000000000000000000040
:10B8D000000000009B3CFFFFFFFFFFFF20B30000C4
:10B8E0000000000000000000000000000000000058
:10B8F000D201FFDFFFFFFFFFD2FE00380000000093
:10B900000000000000000000000000000000BF6513
:10B91000FFFFFFFFFFFF20B300000000000000005A
:10B9200000000000000000000000D201FFDFFFFF68
:10B93000FFFFD2FE00380000000000000000000001
:10B940000000000000000000BF65FFFFFFFFFFFFD9
:10B9500020B3000000000000000000000000000014
:10B9600000000000D201FFDFFFFFFFFFD2FE003822
:10B9700000000000000000000000000000000000C7
:10B980000000BF65FFFFFFFFFFFF20B300000000C6
:10B990000000000000000000000000000000D201D4
:10B9A000FFDFFFFFFFFFD2FE0038000000000000B5
:10B9B000000000000000000000000000BF65FFFF65
:10B9C000FFFFFFFF20B300000000000000000000A8
:10B9D0000000000000000000D201FFDFFFFFFFFFBA
:10B9E000D2FE00380000000000000000000000004F
:10B9F000000000000000BF65FFFFFFFFFFFF20B356
:10BA00000000000000000000000000000000000036
:10BA100000000000000000009B3CD2FE0038000047
:10BA20000000000000000000000000000000000016
:10BA30000000000000000000000000000000000006
:10BA400000000000000000000000000000000000F6
:10BA500000000000000000000000000000000000E6
:10BA600000000000000000000000000000000000D6
:10BA7000000000001FA7FFFFFFFF14FF00500000A1
:10BA8000000000001FA7FFFFFFFF14FF0050000091
:10BA900000000000000000000000000000000000A6
:10BAA0000000000000000000000000000000000096
:10BAB0000000000000000000000000000000000086
:10BAC0000000000000000000000000000000000076
:10BAD0000000000000000000000000000000000066
:10BAE0000000000000000000000000000000000056
:10BAF0000000000000000000000000000000000046
:10BB00000000000000000000000000000000000035
:10BB10000000000000000000000000000000000025
:10BB20000000000000000000000000000000000015
:10BB30000000000000000000000000000000000005
:10BB400000000000000000000000000000000000F5
:10BB500000000000000000000000000000000000E5
:10BB600000000000000000000000000000000000D5
:10BB700000000000000000000000000000000000C5
:10BB800000000000000000000000000000000000B5
:10BB900000000000000000000000000000000000A5
:10BBA0000000000000000000000000000000000095
:10BBB0000000000000000000000000000000000085
:10BBC0000000000000000000000000000000000075
:10BBD0000000000000000000000000000000000065
:10BBE0000000000000000000000000000000000055
:10BBF0000000000000000000000000000000000045
:10BC00000000000000000000000000000000000034
:10BC10000000000000000000000000000000000024
:10BC20000000000000000000000000000000000014
:10BC30000000000000000000000000000000000004
:10BC400000000000000000000000000000000000F4
:10BC500000000000000000000000000000000000E4
:10BC600000000000000000000000000000000000D4
:10BC700000000000000000000000000000000000C4
:10BC80000000000000000000000000000000BF6590
:10BC9000FFFFFBFFC091000000000000000000005B
:10BCA00000000000000000000000D201FFDFFFFFE5
:10BCB000FFFFD2FE0038000000000000000000007E
:10BCC0000000000000000000D201FFDFFFFFFFFFC7
:10BCD000D2FE00380000000000000000000000005C
:10BCE00000000000000000009B3CFFFFFBFFC09134
:10BCF0000000000000000000000000000000000044
:10BD000000000000000000000700DF96FFFFFBFFBF
:10BD1000C09100000000D201FFDFFFFFFFFF20B352
:10BD200000003603FFFFFFFFFBFFC0910000000093
:10BD30000000000000000000000000000000000003
:10BD4000D201FFDFFFFFFFFF87DC00000000D20110
:10BD5000FFDFFFFFFFFF87DC00009B3CFFFFFFFFD3
:10BD6000FBFFC09100000000000000000000000088
:10BD70000000000000000000BF65FFFFFFFFFFFFA5
:10BD8000D2FE00380000D201FFDFFFFFFFFFD2FE2E
:10BD90000038BF65FFFFFFFFFBFFC0910000000000
:10BDA00000000000000000000000000000000C0087
:10BDB000FFB7FFFF2CB3FFB7FBFFC0910000D2011C
:10BDC000FFDFFBFFDFDEF6FF0C60FFB7DBFEFFDF10
:10BDD000FBFFC09100000000000000000000000018
:10BDE0000000000000003603FFFFF6FF0760DF964B
:10BDF000FFFF87DC0000D201FFDFF6FF9B94FFFF0F
:10BE000092B4FFDF92DCFFB7FBFFC091000000009F
:10BE10000000000000000000000000000000BF65FE
:10BE2000FFFFD2FE00389B3CFFFFD2FE0038D2015C
:10BE3000FFDFF6FF3663FFFFFFFFFFFF2CB3FFB707
:10BE4000FBFFC091000000000000000000000000A7
:10BE500000000000D201FFDFFFFFFFFFFFFFFFFF39
:10BE6000FFFFFBFFC091D201FFDFF6FF0C60FFB7C1
:10BE7000FFFFFBFFCC91FFB7FBFFC091000000006C
:10BE80000000000000000000000000009B3CFFFFDD
:10BE9000FFFFFFFFFFFFFFFFFFFFFFFF87DCD20178
:10BEA000FFDFF6FF0760DF96FFFFD2FE0C38FFB71B
:10BEB000FBFFC09100000000000000000000000037
:10BEC00000000000DF96FFFFD2FE003800000700F0
:10BED000DF96FFFFF6FFD261FFDFF6FF0060BF6570
:10BEE000FFFFACFD0C00FFB7FBFFC091000000009E
:10BEF0000000000000000A001FA7FFFFFFFFFFFF78
:10BF000000C400000A001FA7FFFFFFFFFFFFFFFFA5
:10BF1000FCFFA0A21804FFFFFFFF00C40000000008
:10BF2000000000003C55FFFFF8FF3CA5FFFFFFFFAE
:10BF300000C400003C55FFFFFFFFFFFFFFFFFFFFB6
:10BF4000FCFFA0A23C55FFFFFCFFA0A20A001FA718
:10BF5000FFFF2AE51804FFFFFCFFA0A20A001FA7AD
:10BF6000FFFF2AE50A001FA7FFFFFFFFFFFFFFFFFC
:10BF7000FCFFA0A200000A001FA7FFFFFFFFFFFFBA
:10BF800000C40000000000000000000000000000ED
:10BF900000000000BF65FFFFFFFFFFFF87DC000020
:10BFA0000000000000000000000000000000000091
:10BFB0003603FFFFFFFFFFFFFFFF87DC00000000ED
:10BFC0000000000000000000000000000C00FFB7AF
:10BFD000FFFFFFFFFFFFFFFF87DC00000000000006
:10BFE00000000000000000000000BF65FFFFFFFF31
:10BFF000FFFFFFFFFFFF87DC0000000000000000E4
:10C000000000000000003603FFFFFFFFFFFFFFFFFF
:10C01000FFFFFFFF87DC00000000000000000000C1
:10C0200000000C00FFB7FFFFFFFFFFFFFFFFFFFF58
:10C03000FFFF87DC00000000000000000000070098
:10C04000DF96FFFFFFFFFFFF92B4FFDFFFFFFFFF61
:10C0500087DC000000000000000000009B3CFFFFA8
:10C06000FFFFFFFFACFDD201FFDFFFFFFFFF87DC1B
:10C070000000000000000000D201FFDFFFFFFFFF13
:10C08000F6FF0060D201FFDFFFFFFFFF87DC00004B
:10C09000000000000700DF96FFFFFFFFFBFFC091DD
:10C0A0000000D201FFDFFFFFFFFF87DC0000000080
:10C0B00000009B3CFFFFFFFFFFFF87DC000000004C
:10C0C000D201FFDFFFFFFFFF87DC00000000D2018D
:10C0D000FFDFFFFFFFFFD2FE003800000000D201AB
:10C0E000FFDFFFFFFFFF87DC000000009B3CFFFF3E
:10C0F000FFFFFFFFFFFFFFFFFFFFFFFFFFFFFFFF50
:10C10000FFFFFFFFFFFFFBFFC0919B3CFFFFFFFF17
:10C11000FFFFFFFFFFFFFFFFFFFFFFFFFFFFFFFF2F
:10C12000FFFFFFFFFBFFC0919B3CFFFFFFFFFFFFF7
:10C13000FFFFFFFFFFFFFFFFFFFFFFFFFFFFFFFF0F
:10C14000FFFFFBFFC09100000000000000000000A6
:10C15000000000000000D201FFDFFFFFFFFF87DCCF
:10C1600000000000000000000000000000000000CF
:10C1700000000000D201FFDFFFFFFFFF87DC0000AF
:10C1800000000000000000000000000000000000AF
:10C190000000D201FFDFFFFFFFFF87DC000000008F
:10C1A000000000000000000000000000000000008F
:10C1B000D201FFDFFFFFFFFF87DC0000000000006F
:10C1C0000000B402FFE7FFFFFFFFF8FF0080000060
:10C1D0001000FFC7FFFFFFFFFFFFFFFF14FF00502E
:10C1E0001804FFFFF8FF00801804FFFFF8FF00802D
:10C1F00000000000000000003C55FFFF14FF00504D
:10C200000000000000003F86FFFFFCFFA0A200002E
:10C2100000000000000000001000FFC7FFFF00C486
:10C220003C55FFFFF8FF00801000FFC7FFFF2AE525
:10C230001000FFC7FFFFFFFFFFFFFFFFFCFFA0A2F3
:10C240000000B402FFE7FFFFFFFFFCFFA0A2000019
:10C250000000B402FFE7FFFFFFFFFCFFA0A2000009
:10C26000B402FFE7FFFFFFFFFFFFFFFFFCFFA0A2FD
:10C27000B402FFE7F8FF00801000FFC7FCFFA0A298
:10C280000A001FA7FFFFFFFFFFFFFFFF30FE0000B8
:10C290000A001FA7FFFFFFFFFFFFFFFF14FF005073
:10C2A0003C55FFFFF8FF00801000FFC7FFFF00C4F0
:10C2B0003C55FFFFF8FF00801000FFC7FFFF2AE595
:10C2C000B402FFE7FFFFFFFFFFFFFFFFFCFFA0A29D
:10C2D00000001804FFFFFFFFFFFFFFFF00C4000086
:10C2E0000000000000001804FFFFF8FF00800000BD
:10C2F000000000003F86FFFFFFFFF8FF0080000006
:10C300001000FFC7FFFFFFFFFFFFF8FF00800000E6
:10C310001000FFC700C43C55FFFFF8FF008000007D
:10C320000000000000003C55FFFFF8FF0080000007
:10C330000000000000003C55FFFFF8FF00800000F7
:10C340000000000000003C55FFFFF8FF00800000E7
:10C350000000000000003C55FFFFF8FF00800000D7
:10C360000000000000003C55FFFFF8FF00800000C7
:10C370000000000000000000D201FFDFFFFFFFFF10
:10C38000FFFFFBFFC0910000000000000000000064
:10C3900000000700DF96FFFFFFFFFFFFFFFFFFFF2B
:10C3A000FFFFFFFFACFD00000000000000000700E1
:10C3B000DF96FFFFFFFFFFFFFFFFFFFFFFFFFFFF16
:10C3C000FFFFFFFF87DC0000000000003603FFFFD7
:10C3D000FFFFFFFFD2FE003800000C00FFB7FFFF99
:10C3E000FFFFFBFFC09100000000BF65FFFFFFFFE4
:10C3F000F6FF00600000000000003603FFFFFFFFB3
:10C40000FFFF20B300000700DF96FFFFFFFFD2FE13
:10C410000038000000000000D201FFDFFFFFFFFF37
:10C4200087DC0000000000000000000000000000A9
:10C43000000000000000D201FFDFFFFFFFFF87DCEC
:10C4400000000000000000000000000000000000EC
:10C4500000000000BF65FFFFFFFFFBFFC091000071
:10C4600000000000000000000000000000000000CC
:10C47000D201FFDFFFFFFFFFD2FE00380000000007
:10C480000000000000000000000000000C00FFB7EA
:10C49000FFFFFFFFFFFF20B30000000000000000CF
:10C4A00000000000000000000700DF96FFFFFFFF14
:10C4B000FFFFD2FE00380000000000000000000076
:10C4C000000000000700DF96FFFFFFFFFFFFF6FF01
:10C4D00000600000000000000000000000000000FC
:10C4E0000700DF96FFFFFFFFFFFFFBFFC09100008B
:10C4F0000000000000000000000000000700DF96C0
:10C50000FFFFFFFFFFFFFFFF20B300000000000060
:10C5100000000000000000000000BF65FFFFFFFFFB
:10C52000FFFFFFFF20B3000000000000000000003C
:10C53000000000000000BF65FFFFFFFFFFFFFFFFDF
:10C5400020B3000000000000000000000000000018
:10C550000000BF65FFFFFFFFFFFFFFFFFFFFFFFFC3
:10C56000FFFFFFFFFFFFFFFFFFFFACFD00009B3C55
:10C57000FFFFFFFFFFFFFFFFFFFFFFFFFFFFFFFFCB
:10C58000FFFFFFFFFFFFFFFFACFD00009B3CFFFF35
:10C59000FFFFFFFFFFFFFFFFFFFFFFFFFFFFFFFFAB
:10C5A000FFFFFFFFFFFFACFD0000000000000000E8
:10C5B00000000000D201FFDFFFFFFFFFFFFFFBFFD6
:10C5C000C09100000000000000000000000000001A
:10C5D000BF65FFFFFFFFFFFFFFFFFFFFFFFFFFFF45
:10C5E000ACFD000000000000000000009B3CFFFFCD
:10C5F000FFFFFFFFFFFFFFFFFFFFFFFFFFFFFFFF4B
:10C6000087DC0000000000000C00FFB7FFFFFFFF09
:10C61000FBFFC0910000D201FFDFFFFFFFFFF6FF2D
:10C62000006000000000D201FFDFFFFFFFFF87DC9A
:10C630000000000000009B3CFFFFFFFFFBFFC091DC
:10C64000000000003603FFFFFFFFFFFF20B30000E4
:10C65000000000003603FFFFFFFFFFFF20B30000D4
:10C660000000D201FFDFFFFFFFFF87DC00000000BA
:10C6700000009B3CFFFFFFFFFBFFC091000000009C
:10C680000700DF96FFFFFFFFFBFFC0910000D20114
:10C69000FFDFFFFFFFFFD2FE0038000000000000B8
:10C6A000D201FFDFFFFFFFFFFFFFFFFFFFFFFFFFE5
:10C6B000FFFFFBFFC091000000000000000007002A
:10C6C000DF96FFFFFFFFFFFFFFFFFFFFFFFFFFFF03
:10C6D000D2FE00380000000000000C00FFB7FFFF92
:10C6E000FFFFFFFFFFFFFFFFFFFFFFFFFFFFFFFF5A
:10C6F000F6FF006000000000BF65FFFFFFFFFFFFC7
:10C70000ACFD000000000000BF65FFFFFFFFFFFF62
:10C71000ACFD00000C00FFB7FFFFFFFFACFD000009
:10C720000000000000000000BF65FFFFFFFFF6FFF4
:10C730000060D201FFDFFFFFFFFF87DC0000000089
:10C740000000000000009B3CFFFFFFFFFBFFC091CB
:10C75000D201FFDFFFFFFFFFACFD00000000000083
:10C7600000000000BF65FFFFFFFFFBFFC091070057
:10C77000DF96FFFFFFFFFFFFACFD000000000000A1
:10C780009B3CFFFFFFFFFFFFD2FE00380000360397
:10C79000FFFFFFFFFFFFFFFFFFFFFFFFFFFFFFFFA9
:10C7A000FFFFFFFFFFFF20B30000000000009B3CE5
:10C7B000FFFFFFFFFFFFFFFFFFFFFFFFFFFFFFFF89
:10C7C000FFFF87DC00000000000000000000070001
:10C7D000DF96FFFFFFFFFFFFFFFFFFFFD2FE0038E6
:10C7E000000000000000000000000A001FA7FFFF7B
:10C7F000FFFF14FF005000001000FFC7FFFFFFFF06
:10C80000FFFFFFFF14FF00501804FFFFFCFFA0A272
:10C81000B402FFE7FFFF00C43C55FFFF14FF0050C8
:10C820001000FFC7FFFF2AE53C55FFFF14FF005033
:10C830000A001FA7FFFF2AE53C55FFFFF8FF008015
:10C840000A001FA7FFFF2AE51804FFFFFCFFA0A2B4
:10C85000B402FFE7FFFF00C40A001FA7FFFFFFFFAE
:10C86000FFFFFFFF14FF005000000A001FA7FFFF9B
:10C87000FFFF14FF00500000000000000000000057
:10C8800000000000000000000000000000000000A8
:10C890000000000000000000000000000000000098
:10C8A00000000000000000000A001FA7FFFFFCFFBF
:10C8B000A0A20000180400C43C55FFFFFFFFFFFFCB
:10C8C000FFFFFFFFFFFF00C43855A0A20000B40225
:10C8D000FFE7FFFF30FE0000000000000000000046
:10C8E0000000000000000000000000000000000048
:10C8F0000000000000000000000000000000000038
:10C900000000000000000000000000000000000027
:10C910000C00FFB7FFFFFFFFFFFFFFFF20B300008A
:10C920000000000000000000000000009B3CFFFF32
:10C93000FFFFFFFFFFFFFFFFFFFFFFFFD2FE0038FB
:10C9400000000000000000003603FFFFFFFFFFFFB4
:10C95000FFFFFFFFFFFFFFFFFFFFFFFFACFD00003A
:10C96000000000000700DF96FFFFFFFFFFFF20B37E
:10C9700000000700DF96FFFFFFFFFBFFC0910000F4
:10C980000000D201FFDFFFFFFFFF87DC0000000097
:10C9900000003603FFFFFFFFFFFF20B30000000091
:10C9A0000000000000000000000000000000000087
:10C9B0009B3CFFFFFFFFFBFFC09100000000000059
:10C9C000000000000000000000000000BF65FFFF45
:10C9D000FFFFFFFFD2FE0038000000000000000053
:10C9E000000000000C00FFB7FFFFFFFFFFFFFFFF8D
:10C9F000D2FE00380000000000000000000000002F
:10CA000000000C00FFB7FFFFFFFFFFFFF6FF006015
:10CA10000000000000000000000000000000000016
:10CA20000C00FFB7FFFFFFFFFFFFFFFFFFFFACFDA5
:10CA300000000000000000000000000000000000F6
:10CA4000000000003603FFFFFFFFFFFFFFFF87DC52
:10CA500000000000000000000000000000000000D6
:10CA6000000000000C00FFB7FFFFFFFFF6FF0060B3
:10CA700000000000000000000000000000000000B6
:10CA8000000000009B3CFFFFFFFFFBFFC091D201B5
:10CA9000FFDFFFFFFFFF87DC000000000000000059
:10CAA00000009B3CFFFFFFFFFBFFC0910C00FFB7A6
:10CAB000FFFFFFFFD2FE003800000000000007006B
:10CAC000DF96FFFFFFFFF6FF00600000BF65FFFF7E
:10CAD000FFFFFFFFD2FE003800000000BF65FFFF30
:10CAE000FFFFFFFFACFD000000000C00FFB7FFFFE1
:10CAF000FFFFFFFFFFFFFFFFFFFFFFFFFFFFFFFF46
:10CB0000F6FF0060000000000000D201FFDFFFFF21
:10CB1000FFFFFFFFFFFFFFFFFFFFFFFFF6FF0060CC
:10CB20000000000000000000000000009B3CFFFF30
:10CB3000FFFFFFFFFFFFFFFF20B30000000000002A
:10CB400000000000010001000100010002000200DD
:10CB500003000300040004000500050006000600B1
:10CB60000700070008000800090009000A000A0879
:10CB70000B080B080C100D100D180E180E200F28A6
:10CB80000F28103010301138113812401240124066
:10CB9000134813481348134813501450145014509A
:10CBA00014581458145814581460156015603568DA
:10CBB000556875689570B570D5701579557975811A
:10CBC000B581D589158A35927592B592D49A149B00
:10CBD000349B54A394A3B4A3D4ABF4AB13AC33AC45
:10CBE00053B473B492B4B2B4B2B4D1BCF1BC10BDFE
:10CBF00030BD30BD4FBD6FBD6EBD8EBD8EC5AEC5E7
:10CC0000ADC5CDC5CDC5EDC5EDC5EDC50DC60DC6D2
:10CC10000DC62EC62EC62FC62FC630CE30CE51CE54
:10CC200051CE52CE53CE53CE54CE54CE55CE55CEF9
:10CC300056CE56CE56CE57CE57CE57CE58CE58CECD
:10CC400058CE58CE0000000000000000BF65FFFF76
:10CC5000FFFFFFFFFFFFFFFFFFFFFFFFFFFF87DC7F
:10CC600000000000000000000700DF96FFFFFFFF4C
:10CC7000FFFFFFFFFFFFFFFFFFFFFFFF87DC00005D
:10CC8000000000000000D201FFDFFFFFFFFFFFFFF9
:10CC9000FFFFFFFFFFFFFFFFFFFF87DC000000003B
:10CCA000000000003603FFFFFFFFF6FF00600000FA
:10CCB0000000000000000000000000000000000074
:10CCC0000000BF65FFFFFFFFD2FE0038000000003C
:10CCD000000000000000000000000000000007004D
:10CCE000DF96FFFFFFFFACFD00000000000000002A
:10CCF0000000000000000000000000000C00FFB772
:10CD0000FFFFFFFF87DC00000000000000000000C4
:10CD1000000000000000000000003603FFFFFFFFDE
:10CD2000FFFFFFFFFFFFFFFFFFFF20B3000000003A
:10CD300000000000000000009B3CFFFFFFFFFFFF22
:10CD4000FFFFFFFFFFFFFFFFFFFFD2FE00380000E5
:10CD5000000000000000BF65FFFFFFFFFFFFFFFFB7
:10CD6000FFFFFFFFFFFFFFFFFFFFACFD0000000024
:10CD700000000700DF96FFFFFFFFD2FE0038000033
:10CD80000C00FFB7FFFFFFFFFFFF20B30000000014
:10CD90000000000000000000000000000000000093
:10CDA000D201FFDFFFFFFFFFACFD0000000000002D
:10CDB00000000000000000000000000000000C0067
:10CDC000FFB7FFFFFFFFACFD000000000000000008
:10CDD0000000000000000000000000000C00FFB791
:10CDE000FFFFFFFFACFD00003603FFFFFFFFFFFF6B
:10CDF000ACFD00000000000000003603FFFFFFFF55
:10CE0000FFFF87DC00000C00FFB7FFFFFFFFFFFF05
:10CE1000ACFD00000000D201FFDFFFFFFFFFFBFFC2
:10CE2000C091000000003603FFFFFFFFFFFFFFFF80
:10CE3000FFFFFFFFFFFFFFFFFFFFFFFF87DC00009B
:10CE40000000000000003603FFFFFFFFFFFFFFFFB1
:10CE5000FFFFFFFFFFFFFFFF87DC00000000000077
:10CE60000000000000000000BF65FFFFFFFFFFFFA4
:10CE7000FFFFD2FE003800000000000000000000AC
:10CE80000000D201FFDFFFFF87DC00000000000090
:10CE9000000000000700DF96FFFFFFFFFFFFD2FE4C
:10CEA00000380000D201FFDFFFFFFFFFFFFFFFFFA1
:10CEB000FFFF87DC000000000000D201FFDFFFFF62
:10CEC00087DC00000000000000000700DF96FFFF85
:10CED000FFFFFFFFFFFFFFFFD2FE0038D201FFDFA1
:10CEE000FFFFFFFFFFFFFFFFFFFFFBFFC091000001
:10CEF0000000D201FFDFFFFF87DC00000000000020
:10CF00000000D201FFDFFFFF20B300009B3CFFFFCA
:10CF1000FBFFC091D201FFDFFFFF87DC00009B3CDD
:10CF2000FFFFFBFFC09100000000D201FFDFFFFF09
:10CF300087DC00000000000000000C00FFB7FFFFCE
:10CF4000FFFFFFFFD2FE003800000000D201FFDF2C
:10CF5000FFFFFFFFFFFFFFFFFFFF20B30000000008
:10CF60000000D201FFDFFFFF87DC000000000000AF
:10CF7000000000000C00FFB7FFFFFFFFFFFFFFFFF7
:10CF8000D2FE0038D201FFDFFFFFFFFFFFFFFFFFF0
:10CF9000FFFFF6FF006000000000D201FFDFFFFF8F
:10CFA00087DC00000000000000000000000000001E
:10CFB00000000700DF96FFFFFFFF87DCD201FFDFE5
:10CFC000FFFF87DC0000D201FFDFFFFF87DC0000EE
:10CFD0000000D201FFDFFFFF87DC0000000000003F
:10CFE00000009B3CFFFFFBFFC0910000D201FFDF70
:10CFF000FFFF87DCD201FFDFFFFF87DC0000360385
:10D00000FFFFFFFF87DC00000000D201FFDFFFFF12
:10D01000FFFFFFFFFFFFFFFFACFD0C00FFB7FFFFAF
:10D02000FFFFFFFFFFFFFFFFFBFFC091D201FFDF0C
:10D03000FFFFFFFFFFFFFFFFFFFFFFFF20B3000029
:10D040000000D201FFDFFFFFFFFFFFFFFFFFFFFF39
:10D05000ACFD0000D201FFDFFFFFFFFFFFFFF6FF87
:10D0600000600000D201FFDFFFFFFFFFFFFFFFFFB7
:10D07000FFFF87DC0000000000001804FFFFFFFF37
:10D08000FFFFFFFF00C40000B402FFE7FFFFFFFF48
:10D09000FFFFFFFFFCFFA0A23C55FFFFF8FF008051
:10D0A0001000FFC7FFFF2AE500000000000000009D
:10D0B000B402FFE7FFFF00C4000000000000B4025C
:10D0C000FFE7FFFF14FF0050000000003C55FFFF8A
:10D0D000FFFF30FE0000000000003C55FFFFFFFF97
:10D0E00000C4000000000000B402FFE7FFFFFFFFE4
:10D0F000FFFFFFFFFFFF2AE53F86FFFFFFFFFFFF68
:10D10000FFFFFFFFFFFF2AE5D201FFDFFFFF87DC04
:10D11000000000009B3CFFFFFBFFC09100000700E8
:10D12000DF96FFFFFFFFFFFFD2FE00380000D201B5
:10D13000FFDFFFFFFFFFFFFFFFFFFFFF87DC0000B8
:10D14000D201FFDFFFFF87DC000000009B3CFFFFF8
:10D15000FBFFC0910700DF96FFFFFFFFFFFFFFFF10
:10D16000FFFFD2FE0038D201FFDFFFFFFFFFFFFF0E
:10D17000FFFFFFFFFBFFC091D201FFDFFFFF87DC56
:10D18000000000009B3CFFFFFBFFC091D201FFDFCE
:10D19000FFFF20B300009B3CFFFFFBFFC091D201CB
:10D1A000FFDFFFFF87DC00009B3CFFFFFBFFC09120
:10D1B000D201FFDFFFFF87DC000000009B3CFFFF88
:10D1C000FBFFC0910C00FFB7FFFFFFFFFFFFD2FE88
:10D1D000003800000000D201FFDFFFFFFFFFFFFF6C
:10D1E000FFFFFFFF20B30000D201FFDFFFFF87DC5E
:10D1F000000000009B3CFFFFFBFFC09100000C0003
:10D20000FFB7FFFFFFFFFFFFFFFFD2FE0038D20195
:10D21000FFDFFFFFFFFFFFFFFFFFFFFFF6FF0060E5
:10D22000D201FFDFFFFF87DC000000009B3CFFFF17
:10D23000FBFFC09100000000000000000700DF9627
:10D24000FFFFFFFF87DCD201FFDFFFFF87DC00006D
:10D25000D201FFDFFFFF87DC0C00FFB7FFFFD2FE2C
:10D2600000380700DF96FFFFF6FF00609B3CFFFFE2
:10D27000FBFFC0910000D201FFDFFFFF87DCD2017E
:10D28000FFDFFFFF87DC00003603FFFFFFFF87DCC7
:10D2900000009B3CFFFFFFFFFFFFFFFFFFFFFFFFC3
:10D2A00087DC00000C00FFB7FFFFFFFFFFFFFFFF61
:10D2B000FFFFFBFFC091D201FFDFFFFFFFFFFFFF7A
:10D2C000FFFFFFFFFFFF20B3000000009B3CFFFFBC
:10D2D000FFFFFFFFFFFF87DC000000000000D2011E
:10D2E000FFDFFFFFFFFFFFFFF6FF00600000D2013E
:10D2F000FFDFFFFFFFFFFFFFFFFFFFFF87DC0000F7
:10D3000000003F86FFFFFFFFFFFFFFFFFCFFA0A223
:10D310000A001FA7FFFFFFFFFFFFFFFFFCFFA0A208
:10D320001000FFC7FCFFA0A20000000000000000EA
:10D330001000FFC7FCFF1FE7FFFFFFFF00C4000056
:10D34000B402FFE7FFFFFFFFFFFFFFFFFFFF00C487
:10D3500000000000000000001000FFC7FFFF2AE5EA
:10D360003C55FFFFF8FF00801000FFC7FFFF2AE5D4
:10D37000B402FFE7FFFFFFFFFFFFFFFFFCFFA0A2DC
:10D380000000B402FFE7FFFFFFFFFCFFA0A20000C8
:10D39000000000000000000000000000000000008D
:10D3A000FFFF00000000000000000000000000007F
:10D3B00000000000FFFF000000000000000000006F
:10D3C0000000000000000000FFFF0000000000005F
:10D3D000000000000000000000000000FFFF00004F
:10D3E000000000000000000000000000000000003D
:10D3F000FFFF00000000000000000000000000002F
:10D4000000000000FFFF000000000000000000001E
:10D410000000000000000000FFFF0000000000000E
:10D42000000000000000000000000000FFFF0000FE
:10D4300000000000000000000000000000000000EC
:10D44000FFFF0000000000000000000000000000DE
:10D450000000EF7BFFFFEF7B0000000000000000FA
:10D46000000000000000EF7BFFFFEF7B00000000EA
:10D4700000000000000000000000EF7BFFFFEF7BDA
:10D480000000000000000000000000000000EF7B32
:10D49000FFFFEF7B00000000000000000000000024
:10D4A0000000EF7BFFFFEF7B0000000000000000AA
:10D4B000000000000000EF7BFFFFEF7B000000009A
:10D4C000000000000000000000000000000000005C
:10D4D000000000000000FFFF00000000000000004E
:10D4E00000000000000000000000FFFF000000003E
:10D4F0000000000000000000000000000000FFFF2E
:10D50000000000000000000000000000000000001B
:10D510000000FFFF0000000000000000000000000D
:10D52000000000000000FFFF0000000000000000FD
:10D5300000000000000000000000FFFF00000000ED
:10D540000000000000000000000000000000FFFFDD
:10D5500000000000000000000000000000000000CB
:10D560000000FFFF000000000000000000000000BD
:10D57000000000000000FFFF0000000000000000AD
:10D580000000000000000000EF7BFFFFEF7B0000C9
:10D59000000000000000000000000000EF7BFFFF23
:10D5A000EF7B000000000000000000000000000011
:10D5B000EF7BFFFFEF7B0000000000000000000099
:10D5C00000000000EF7BFFFFEF7B00000000000089
:10D5D0000000000000000000EF7BFFFFEF7B000079
:10D5E000000000000000000000000000EF7BFFFFD3
:10D5F000EF7B0000000000000000000000000000C1
:10D60000000000000000000000000000FFFF00001C
:10D61000000000000000000000000000000000000A
:10D6200000000000000000000000000000000000FA
:10D6300000000000FFFF00000000000000000000EC
:10D6400000000000000000000000000000000000DA
:10D65000000000000000000000000000FFFF0000CC
:10D6600000000000000000000000000000000000BA
:10D6700000000000000000000000000000000000AA
:10D6800000000000FFFF000000000000000000009C
:10D69000000000000000000000000000000000008A
:10D6A000000000000000000000000000FFFF00007C
:10D6B000000000000000000000000000000000006A
:10D6C000000000000000000000000000000000005A
:10D6D0000000EF7BFFFFEF7B000000000000000078
:10D6E000000000000000000000000000000000003A
:10D6F00000000000000000000000EF7BFFFFEF7B58
:10D700000000000000000000000000000000000019
:10D710000000000000000000000000000000000009
:10D720000000EF7BFFFFEF7B000000000000000027
:10D7300000000000000000000000000000000000E9
:10D740000000FFFF000000000000000000000000DB
:10D7500000000000000000000000000000000000C9
:10D7600000000000000000000000FFFF00000000BB
:10D7700000000000000000000000000000000000A9
:10D780000000000000000000000000000000000099
:10D790000000FFFF0000000000000000000000008B
:10D7A0000000000000000000000000000000000079
:10D7B00000000000000000000000FFFF000000006B
:10D7C0000000000000000000000000000000000059
:10D7D0000000000000000000000000000000000049
:10D7E0000000FFFF0000000000000000000000003B
:10D7F0000000000000000000000000000000000029
:10D800000000000000000000EF7BFFFFEF7B000046
:10D810000000000000000000000000000000000008
:10D8200000000000000000000000000000000000F8
:10D83000EF7BFFFFEF7B0000000000000000000016
:10D8400000000000000000000000000000000000D8
:10D850000000000000000000EF7BFFFFEF7B0000F6
:10D8600000000000000000000000000000000000B8
:10D8700000000000000000000000000000000000A8
:10D880000000000000000000000000000000000098
:10D890000000000000000000000000000000000088
:10D8A0000000000000000000000000000000000078
:10D8B0000000000000000000000000000000000068
:10D8C0000000000000000000000000000000000058
:10D8D0000000000000000000000000000000000048
:10D8E0000000000000000000000000000000000038
:10D8F0000000000000000000000000000000000028
:10D900000000000000000000000000000000000017
:10D910000000000000000000000000000000000007
:10D9200000000000000000000000000000000000F7
:10D9300000000000000000000000000000000000E7
:10D9400000000000000000000000000000000000D7
:10D9500000000000000000000000000000000000C7
:10D9600000000000000000000000000000000000B7
:10D9700000000000000000000000000000000000A7
:10D980000000000000000000000000000000000097
:10D990000000000000000000000000000000EF7B1D
:10D9A000FFFFFFFFFFFFEF7B000000000000EF7BA9
:10D9B000FFFF000000000000000000000000000069
:10D9C0000000000000000000000000000000000057
:10D9D000000000000000FFFFFFFFEF7B00000000E1
:10D9E0000000000000000000000000000000000037
:10D9F0000000000000000000000000000000FFFF29
:10DA0000FFFFFFFF0000000000000000000000001A
:10DA10000000000000000000000000000000000006
:10DA2000000000000000FFFFFFFFFFFF00000000FC
:10DA300000000000000000000000000000000000E6
:10DA40000000000000000000000000000000EF7B6C
:10DA5000FFFFFFFF000000000000000000000000CA
:10DA600000000000000000000000000000000000B6
:10DA7000000000000000EF7BFFFFFFFF0000EF7BD6
:10DA8000FFFFFFFF0000000000000000000000009A
:10DA90000000000000000000000000000000EF7B1C
:10DAA0000000FFFF0000EF7BFFFFFFFF0000000012
:10DAB0000000000000000000000000000000000066
:10DAC000000000000000EF7BFFFF00000000EF7B84
:10DAD000FFFFFFFFFFFF000000000000000000004C
:10DAE00000000000FFFFFFFF00000000000000003A
:10DAF0000000000000000000000000000000000026
:10DB00000000000000000000000000000000000015
:10DB1000FFFF000000000000000000000000000007
:10DB200000000000000000000000000000000000F5
:10DB300000000000FFFF00000000000000000000E7
:10DB400000000000000000000000000000000000D5
:10DB500000000000000000000000000000000000C5
:10DB6000FFFF0000000000000000000000000000B7
:10DB700000000000000000000000000000000000A5
:10DB800000000000FFFF0000FFFF00000000000099
:10DB90000000000000000000000000000000000085
:10DBA000000000000000FFFF00000000FFFF000079
:10DBB000FFFF0000FFFF0000FFFF0000000000006B
:10DBC0000000000000000000000000000000FFFF57
:10DBD00000000000FFFF0000FFFF0000FFFF00004B
:10DBE000FFFF000000000000000000000000000037
:10DBF000000000000000FFFF00000000FFFF000029
:10DC000000000000FFFF0000FFFFEF7BFFFFFFFFB2
:10DC1000FFFFEF7B0000000000000000FFFF00009E
:10DC200000000000000000000000000000000000F4
:10DC300000000000000000000000000000000000E4
:10DC400000000000FFFFEF7B00000000000000006C
:10DC500000000000000000000000000000000000C4
:10DC6000000000000000000000000000FFFFFFFFB8
:10DC700000000000000000000000000000000000A4
:10DC80000000000000000000000000000000000094
:10DC900000000000FFFF0000000000000000000086
:10DCA0000000000000000000000000000000000074
:10DCB00000000000000000000000FFFFFFFFFFFF6A
:10DCC0000000000000000000000000000000000054
:10DCD00000000000000000000000FFFFFFFFFFFF4A
:10DCE00000000000FFFF00000000FFFF0000FFFF3A
:10DCF0000000000000000000000000000000000024
:10DD00000000FFFFFFFFFFFF0000FFFFFFFFFFFF1F
:10DD10000000FFFF0000FFFF000000000000000007
:10DD200000000000000000000000FFFFFFFFFFFFF9
:10DD30000000FFFFFFFFFFFF0000FFFF0000FFFFED
:10DD40000000000000000000FFFF000000000000D5
:10DD50000000FFFF000000000000000000000000C5
:10DD600000000000000000000000000000000000B3
:10DD7000000000000000000000000000FFFF0000A5
:10DD80000000000000000000000000000000000093
:10DD90000000000000000000000000000000000083
:10DDA00000000000FFFF0000000000000000000075
:10DDB0000000000000000000000000000000000063
:10DDC0000000000000000000EF7B000000000000E9
:10DDD0000000000000000000000000000000000043
:10DDE0000000000000000000000000000000000033
:10DDF00000000000FFFF0000000000000000000025
:10DE00000000000000000000000000000000000012
:10DE10000000FFFF00000000FFFF00000000000006
:10DE2000FFFF0000FFFF00000000000000000000F6
:10DE300000000000000000000000FFFF00000000E4
:10DE400000000000FFFF0000FFFF0000FFFF0000D8
:10DE500000000000000000000000000000000000C2
:10DE60000000FFFF00000000FFFF0000FFFF0000B8
:10DE7000FFFF0000FFFFEF7BFFFFFFFFFFFFEF7BD8
:10DE80000000000000000000FFFF00000000000094
:10DE90000000000000000000000000000000000082
:10DEA0000000000000000000000000000000FFFF74
:10DEB000FFFFEF7B000000000000000000000000FA
:10DEC0000000000000000000000000000000000052
:10DED000000000000000FFFFFFFFEF7B00000000DC
:10DEE0000000000000000000000000000000000032
:10DEF0000000000000000000000000000000FFFF24
:10DF00000000000000000000000000000000000011
:10DF10000000000000000000000000000000000001
:10DF200000000000000000000000FFFF00000000F3
:10DF300000000000000000000000000000000000E1
:10DF40000000000000000000000000000000FFFFD3
:10DF5000FFFFFFFF0000FFFFFFFFEF7B000000005F
:10DF600000000000000000000000000000000000B1
:10DF700000000000000000000000FFFF0000FFFFA5
:10DF8000FFFFEF7B00000000000000000000000029
:10DF90000000000000000000000000000000FFFF83
:10DFA000FFFFEF7B0000FFFFFFFFEF7B00000000A3
:10DFB00000000000D201FFDFFFFFFFFFFFFFFBFFBC
:10DFC000C091000000000000000000000000000000
:10DFD000BF65FFFFFFFFFFFFFFFFFFFFFFFFFFFF2B
:10DFE000ACFD00000000000000000000BF65FFFF66
:10DFF000FFFFFFFFFFFFFFFFFFFFFFFFFFFFFFFF31
:10E00000ACFD000000000000D201FFDFFFFFFFFFBA
:10E01000F6FF006000000C00FFB7FFFFFFFFFBFFF3
:10E02000C091000000009B3CFFFFFFFFFBFFC09181
:10E03000000000000000D201FFDFFFFFFFFFACFD8A
:10E0400000000700DF96FFFFFFFFD2FE0038000050
:10E05000000000000700DF96FFFFFFFFD2FE003840
:10E060000C00FFB7FFFFFFFFACFD00000000000049
:10E0700000000000BF65FFFFFFFFF6FF0060D20158
:10E08000FFDFFFFFFFFF87DC000000000000000053
:10E0900000009B3CFFFFFFFFFBFFC091D201FFDFB1
:10E0A000FFFFFFFF87DC0000000000000000000011
:10E0B0009B3CFFFFFFFFFBFFC091D201FFDFFFFF93
:10E0C000FFFF87DC000000000000000000009B3C18
:10E0D000FFFFFFFFFBFFC091D201FFDFFFFFFFFF4C
:10E0E00087DC000000000000000000009B3CFFFFF8
:10E0F000FFFFFBFFC091D201FFDFFFFFFFFF87DCC7
:10E10000000000000000000000009B3CFFFFFFFF3C
:10E11000FBFFC0910C00FFB7FFFFFFFFACFD00004D
:10E120000000000000000000BF65FFFFFFFFF6FFDA
:10E1300000600700DF96FFFFFFFFD2FE00380000FF
:10E14000000000000700DF96FFFFFFFFD2FE00384F
:10E150000000BF65FFFFFFFFFBFFC0910000000054
:10E1600000003603FFFFFFFFFFFFACFD00000000D3
:10E17000D201FFDFFFFFFFFFF6FF006000000C0091
:10E18000FFB7FFFFFFFFFBFFC09100000000000092
:10E19000BF65FFFFFFFFFFFFFFFFFFFFFFFFFFFF69
:10E1A000FFFFFFFFACFD00000000000000000700C3
:10E1B000DF96FFFFFFFFFFFFFFFFFFFFFFFFFFFFF8
:10E1C000D2FE003800000000000000000000000047
:10E1D000D201FFDFFFFFFFFFFFFFFFFF20B30000C3
:10E1E000000000000000000000001804FFFFFFFF17
:10E1F000FFFF14FF00500000B402FFE7FFFFFFFF26
:10E20000FFFFFFFF14FF00503C55FFFF14FF0050BD
:10E21000B402FFE7FFFF00C43C55FFFF14FF0050AE
:10E22000B402FFE7FFFF2AE5B402FFE7FFFFFFFFAD
:10E23000FFFFFFFFFFFF2AE500001804FFFFFFFFBD
:10E2400010C4FFC7FFFF2AE5000000000000000027
:10E250001804FFFFFFFF00C4B402FFE7FFFFFFFF4A
:10E26000FFFFFFFF14FF005000001804FFFFFFFF37
:10E27000FFFF14FF005000000000000000000A0033
:10E280001FA7FFFF30FE00000000000000003F86D7
:10E29000FFFFFFFF30FE0000000000003C55FFFFC5
:10E2A000FFFFFFFF30FE000000001804FFFFF8FF33
:10E2B0001884FFFF30FE00001804FFFFFCFFA0A23F
:10E2C0001804FFFF30FE00001FA7FFFFFFFFFFFF46
:10E2D000FFFFFFFFFFFF14FF1FA7FFFFFFFFFFFF71
:10E2E000FFFFFFFFFFFF14FF000000000000000021
:10E2F0001804FFFF30FE00000000000000000000D6
:10E300001804FFFF30FE00000000000000000C00B9
:10E31000FFB7FFFFFFFFFFFFFFFFD2FE0038000047
:10E32000000000000000000000000000BF65FFFFCB
:10E33000FFFFFFFFFFFFFFFFD2FE003800000000DD
:10E3400000000000000000003603FFFFFFFFFFFF9A
:10E35000FFFFFFFFFFFFD2FE0038000000000000BB
:10E36000000000000000C739000000000700DF9631
:10E37000FFFFFFFFD2FE0038000000000000000099
:10E38000000000000000000000000700DF96FFFF13
:10E39000FFFFD2FE00380000000000000000000077
:10E3A00000000000000000000700DF96FFFFFFFFF5
:10E3B000D2FE003800000000000000000000000055
:10E3C0000000000000000700DF96FFFFFFFFD2FE05
:10E3D0000038000000000000000000000000000005
:10E3E000000000000700DF96FFFFFFFFD2FE0038AD
:10E3F000000000000000000000000000000000001D
:10E4000000000700DF96FFFFFFFFD2FE003800008C
:10E4100000000000000000000000000000000000FC
:10E420000700DF96FFFFFFFFD2FE0038000000006C
:10E4300000000000000000000000000000000700D5
:10E44000DF96FFFFFFFFD2FE003800000000000053
:10E450000000000000000000000000000700DF9640
:10E46000FFFFFFFFD2FE00380000000000000000A8
:10E47000000000000000000000000700DF96FFFF22
:10E48000FFFFD2FE00380000000000000000000086
:10E4900000000000000000000700DF96FFFFFFFF04
:10E4A000D2FE003800000000000000000000000064
:10E4B0000000000000000700DF96FFFFFFFFD2FE14
:10E4C0000038000000000000000000000000000014
:10E4D000000000000700DF96FFFFFFFFD2FE0038BC
:10E4E000000000000000000000000000000000002C
:10E4F00000000700DF96FFFFFFFFD2FE003800009C
:10E50000000000000000000000000000000000000B
:10E510000700DF96FFFFFFFFD2FE0038000000007B
:10E5200000000000000000000000000000000700E4
:10E53000DF96FFFFFFFFD2FE003800000000000062
:10E5400000000000000000000000000000000000CB
:10E5500000009B3CD2FE00380000000000000000DC
:10E5600000000000000000000000000000000C009F
:10E57000FFB7FFFFFFFFD2FE0038000000000000E1
:10E580000000000000000000000000009B3CFFFFB6
:10E59000FFFFFFFF20B300000000000000000000AC
:10E5A0000000000000000000D201FFDFFFFFFFFFBE
:10E5B000D2FE003800000000000000000000000053
:10E5C000000000000000BF65FFFFFFFFFFFF20B35A
:10E5D000000000000000000000000000000000003B
:10E5E0000000D201FFDFFFFFFFFFD2FE0038000076
:10E5F000000000000000000000000000000000001B
:10E60000BF65FFFFFFFFFFFF20B300000000000019
:10E61000000000000000000000000000D201FFDF49
:10E62000FFFFFFFFACFD0000000000000000000045
:10E6300000000000000000000000BF65FFFFFFFFBA
:10E64000FFFFFFFFFFFFF6FF00600000000000007B
:10E650000000000000003603FFFFFFFFFFFFFFFF89
:10E66000FFFFFFFFFFFFFFFF87DC0000000000004F
:10E6700000000700DF96FFFFFFFFFFFFFFFFFFFF28
:10E68000FFFFFFFFFFFFFFFF87DC0000000000002F
:10E690003603FFFFFFFFFFFFD2FE00380000D2016C
:10E6A000FFDFFFFFFFFFF6FF006000000000BF6517
:10E6B000FFFFFFFFF6FF00600000000000003603D0
:10E6C000FFFFFFFFFFFF20B300000000BF65FFFF5B
:10E6D000FFFFD2FE0038000000000000D201FFDF83
:10E6E000FFFFFFFF20B300000000BF65FFFFFFFF3B
:10E6F000FBFFC0910000000000003603FFFFFFFF9A
:10E70000FFFF20B3000000003603FFFFFFFFFFFF05
:10E71000D2FE00380000D201FFDFFFFFFFFFF6FF4F
:10E720000060000000000000BF65FFFFFFFFFFFF6B
:10E73000FFFFFFFFFFFFFFFFFFFFFFFF87DC000082
:10E740000000000000000700DF96FFFFFFFFFFFF53
:10E75000FFFFFFFFFFFFFFFF87DC0000000000005E
:10E760000000000000000000D201FFDFFFFFFFFFFC
:10E77000FFFFF6FF00600000000000000000000046
:10E7800025396C640000000025346400252D3464B4
:10E7900000000000493243206469646E27742049F8
:10E7A0006E697420636F72726563746C7900000027
:10E7B00000040002000600010005000300078000BD
:10E7C000800480028006800180058003800740006D
:10E7D0004004400240064001400540034007C0009D
:10E7E000C004C002C006C001C005C003C0072000AD
:10E7F0002004200220062001200520032007A0007D
:10E80000A004A002A006A001A005A003A00760002C
:10E810006004600260066001600560036007E0005C
:10E82000E004E002E006E001E005E003E00710009C
:10E8300010041002100610011005100310079000BC
:10E84000900490029006900190059003900750006C
:10E850005004500250065001500550035007D0009C
:10E86000D004D002D006D001D005D003D0073000AC
:10E870003004300230063001300530033007B0007C
:10E88000B004B002B006B001B005B003B00770002C
:10E890007004700270067001700570037007F0005C
:10E8A000F004F002F006F001F005F003F0070800B4
:10E8B000080408020806080108050803080788007C
:10E8C000880488028806880188058803880748002C
:10E8D0004804480248064801480548034807C8005C
:10E8E000C804C802C806C801C805C803C80728006C
:10E8F0002804280228062801280528032807A8003C
:10E90000A804A802A806A801A805A803A8076800EB
:10E910006804680268066801680568036807E8001B
:10E92000E804E802E806E801E805E803E80718005B
:10E93000180418021806180118051803180798007B
:10E94000980498029806980198059803980758002B
:10E950005804580258065801580558035807D8005B
:10E96000D804D802D806D801D805D803D80738006B
:10E970003804380238063801380538033807B8003B
:10E98000B804B802B806B801B805B803B8077800EB
:10E990007804780278067801780578037807F8001B
:10E9A000F804F802F806F801F805F803F80704007F
:10E9B000040404020406040104050403040784009B
:10E9C000840484028406840184058403840744004B
:10E9D0004404440244064401440544034407C4007B
:10E9E000C404C402C406C401C405C403C40724008B
:10E9F0002404240224062401240524032407A4005B
:10EA0000A404A402A406A401A405A403A40764000A
:10EA10006404640264066401640564036407E4003A
:10EA2000E404E402E406E401E405E403E40714007A
:10EA3000140414021406140114051403140794009A
:10EA4000940494029406940194059403940754004A
:10EA50005404540254065401540554035407D4007A
:10EA6000D404D402D406D401D405D403D40734008A
:10EA70003404340234063401340534033407B4005A
:10EA8000B404B402B406B401B405B403B40774000A
:10EA90007404740274067401740574037407F4003A
:10EAA000F404F402F406F401F405F403F4070C0092
:10EAB0000C040C020C060C010C050C030C078C005A
:10EAC0008C048C028C068C018C058C038C074C000A
:10EAD0004C044C024C064C014C054C034C07CC003A
:10EAE000CC04CC02CC06CC01CC05CC03CC072C004A
:10EAF0002C042C022C062C012C052C032C07AC001A
:10EB0000AC04AC02AC06AC01AC05AC03AC076C00C9
:10EB10006C046C026C066C016C056C036C07EC00F9
:10EB2000EC04EC02EC06EC01EC05EC03EC071C0039
:10EB30001C041C021C061C011C051C031C079C0059
:10EB40009C049C029C069C019C059C039C075C0009
:10EB50005C045C025C065C015C055C035C07DC0039
:10EB6000DC04DC02DC06DC01DC05DC03DC073C0049
:10EB70003C043C023C063C013C053C033C07BC0019
:10EB8000BC04BC02BC06BC01BC05BC03BC077C00C9
:10EB90007C047C027C067C017C057C037C07FC00F9
:10EBA000FC04FC02FC06FC01FC05FC03FC07020063
:10EBB00002040202020602010205020302078200A9
:10EBC0008204820282068201820582038207420059
:10EBD0004204420242064201420542034207C20089
:10EBE000C204C202C206C201C205C203C207220099
:10EBF0002204220222062201220522032207A20069
:10EC0000A204A202A206A201A205A203A207620018
:10EC10006204620262066201620562036207E20048
:10EC2000E204E202E206E201E205E203E207120088
:10EC300012041202120612011205120312079200A8
:10EC40009204920292069201920592039207520058
:10EC50005204520252065201520552035207D20088
:10EC6000D204D202D206D201D205D203D207320098
:10EC70003204320232063201320532033207B20068
:10EC8000B204B202B206B201B205B203B207720018
:10EC90007204720272067201720572037207F20048
:10ECA000F204F202F206F201F205F203F2070A00A0
:10ECB0000A040A020A060A010A050A030A078A0068
:10ECC0008A048A028A068A018A058A038A074A0018
:10ECD0004A044A024A064A014A054A034A07CA0048
:10ECE000CA04CA02CA06CA01CA05CA03CA072A0058
:10ECF0002A042A022A062A012A052A032A07AA0028
:10ED0000AA04AA02AA06AA01AA05AA03AA076A00D7
:10ED10006A046A026A066A016A056A036A07EA0007
:10ED2000EA04EA02EA06EA01EA05EA03EA071A0047
:10ED30001A041A021A061A011A051A031A079A0067
:10ED40009A049A029A069A019A059A039A075A0017
:10ED50005A045A025A065A015A055A035A07DA0047
:10ED6000DA04DA02DA06DA01DA05DA03DA073A0057
:10ED70003A043A023A063A013A053A033A07BA0027
:10ED8000BA04BA02BA06BA01BA05BA03BA077A00D7
:10ED90007A047A027A067A017A057A037A07FA0007
:10EDA000FA04FA02FA06FA01FA05FA03FA0706006B
:10EDB0000604060206060601060506030607860087
:10EDC0008604860286068601860586038607460037
:10EDD0004604460246064601460546034607C60067
:10EDE000C604C602C606C601C605C603C607260077
:10EDF0002604260226062601260526032607A60047
:10EE0000A604A602A606A601A605A603A6076600F6
:10EE10006604660266066601660566036607E60026
:10EE2000E604E602E606E601E605E603E607160066
:10EE30001604160216061601160516031607960086
:10EE40009604960296069601960596039607560036
:10EE50005604560256065601560556035607D60066
:10EE6000D604D602D606D601D605D603D607360076
:10EE70003604360236063601360536033607B60046
:10EE8000B604B602B606B601B605B603B6077600F6
:10EE90007604760276067601760576037607F60026
:10EEA000F604F602F606F601F605F603F6070E007E
:10EEB0000E040E020E060E010E050E030E078E0046
:10EEC0008E048E028E068E018E058E038E074E00F6
:10EED0004E044E024E064E014E054E034E07CE0026
:10EEE000CE04CE02CE06CE01CE05CE03CE072E0036
:10EEF0002E042E022E062E012E052E032E07AE0006
:10EF0000AE04AE02AE06AE01AE05AE03AE076E00B5
:10EF10006E046E026E066E016E056E036E07EE00E5
:10EF2000EE04EE02EE06EE01EE05EE03EE071E0025
:10EF30001E041E021E061E011E051E031E079E0045
:10EF40009E049E029E069E019E059E039E075E00F5
:10EF50005E045E025E065E015E055E035E07DE0025
:10EF6000DE04DE02DE06DE01DE05DE03DE073E0035
:10EF70003E043E023E063E013E053E033E07BE0005
:10EF8000BE04BE02BE06BE01BE05BE03BE077E00B5
:10EF90007E047E027E067E017E057E037E07FE00E5
:10EFA000FE04FE02FE06FE01FE05FE03FE07010052
:10EFB0000000803F00000000ECFF7F3FD40FC93A03
:10EFC000B1FF7F3FC70F493B4EFF7F3FC1CB963B11
:10EFD000C4FE7F3F890FC93B13FE7F3F3053FB3B8D
:10EFE00039FD7F3F59CB163C39FC7F3F02ED2F3C6A
:10EFF00011FB7F3F900E493CC1F97F3F0030623CDE
:10F000004AF87F3F4B517B3CACF67F3F38398A3C16
:10F01000E6F47F3FB6C9963CF8F27F3F1C5AA33C0A
:10F02000E3F07F3F69EAAF3CA7EE7F3F9B7ABC3CB1
:10F0300043EC7F3FB00AC93CB8E97F3FA69AD53C74
:10F0400005E77F3F7B2AE23C2BE47F3F2DBAEE3C75
:10F0500029E17F3FB949FB3C00DE7F3F90EC033D57
:10F06000AFDA7F3F2F340A3D37D77F3FB87B103D63
:10F0700098D37F3F2CC3163DD1CF7F3F880A1D3DDB
:10F08000E2CB7F3FCC51233DCCC77F3FF698293D53
:10F090008FC37F3F07E02F3D2ABF7F3FFC26363DD1
:10F0A0009EBA7F3FD56D3C3DEAB57F3F91B4423D6E
:10F0B0000FB17F3F2FFB483D0DAC7F3FAF414F3D30
:10F0C000E3A67F3F0E88553D91A17F3F4CCE5B3D2F
:10F0D000189C7F3F6814623D78967F3F625A683D76
:10F0E000B1907F3F38A06E3DC28A7F3FE9E5743D15
:10F0F000AB847F3F742B7B3D6D7E7F3F6CB8803D42
:10F1000008787F3F0ADB833D7B717F3F94FD863D1E
:10F11000C76A7F3F0A208A3DEC637F3F6A428D3D8C
:10F12000E95C7F3FB464903DBF557F3FE786933DE8
:10F130006D4E7F3F05A9963DF4467F3F0ACB993D32
:10F14000543F7F3FF9EC9C3D8D377F3FCF0EA03D74
:10F150009D2F7F3F8C30A33D87277F3F3052A63DB8
:10F16000491F7F3FBA73A93DE4167F3F2B95AC3D05
:10F17000580E7F3F80B6AF3DA4057F3FBBD7B23D61
:10F18000C9FC7E3FDAF8B53DC7F37E3FDD19B93DD6
:10F190009DEA7E3FC33ABC3D4CE17E3F8D5BBF3D67
:10F1A000D4D77E3F397CC23D34CE7E3FC69CC53D20
:10F1B0006DC47E3F36BDC83D7FBA7E3F86DDCB3D08
:10F1C00069B07E3FB7FDCE3D2DA67E3FC81DD23D26
:10F1D000C99B7E3FB93DD53D3D917E3F895DD83D80
:10F1E0008B867E3F377DDB3DB17B7E3FC49CDE3D21
:10F1F000B0707E3F2EBCE13D88657E3F76DBE43D0E
:10F20000385A7E3F9AFAE73DC14E7E3F9A19EB3D50
:10F2100023437E3F7638EE3D5E377E3F2E57F13DED
:10F22000722B7E3FC075F43D5E1F7E3F2C94F73DF0
:10F2300024137E3F73B2FA3DC2067E3F92D0FD3D5D
:10F2400038FA7D3F4577003E88ED7D3F2E06023E31
:10F25000B1E07D3F0295033EB2D37D3FC223053E20
:10F260008CC67D3F6EB2063E40B97D3F0541083EEB
:10F27000CCAB7D3F86CF093E309E7D3FF35D0B3E9C
:10F280006E907D3F4AEC0C3E85827D3F8B7A0E3E30
:10F2900074747D3FB708103E3D667D3FCC96113EAD
:10F2A000DE577D3FCA24133E59497D3FB2B2143E1A
:10F2B000AC3A7D3F8340163ED82B7D3F3DCE173E76
:10F2C000DD1C7D3FE05B193EBC0D7D3F6BE91A3EC6
:10F2D00073FE7C3FDE761C3E03EF7C3F38041E3E0F
:10F2E0006CDF7C3F7B911F3EAECF7C3FA51E213E55
:10F2F000C9BF7C3FB6AB223EBDAF7C3FAD38243E9C
:10F300008A9F7C3F8CC5253E318F7C3F5152273EE2
:10F31000B07E7C3FFCDE283E086E7C3F8D6B2A3E33
:10F320003A5D7C3F04F82B3E444C7C3F61842D3E8B
:10F33000283B7C3FA2102F3EE5297C3FC99C303EF4
:10F340007A187C3FD428323EE9067C3FC4B4333E71
:10F3500031F57B3F9840353E53E37B3F50CC363E02
:10F360004DD17B3FEC57383E20BF7B3F6CE3393EAD
:10F37000CDAC7B3FCF6E3B3E539A7B3F15FA3C3E74
:10F38000B2877B3F3E853E3EEA747B3F4910403E5C
:10F39000FC617B3F379B413EE74E7B3F0726433E68
:10F3A000AB3B7B3FB9B0443E48287B3F4D3B463E9C
:10F3B000BE147B3FC2C5473E0E017B3F1850493EFD
:10F3C00037ED7A3F4FDA4A3E3AD97A3F67644C3E8E
:10F3D00016C57A3F60EE4D3ECBB07A3F38784F3E4F
:10F3E000599C7A3FF101513EC1877A3F898B523E49
:10F3F00002737A3F0115543E1C5E7A3F589E553E7B
:10F4000010497A3F8F27573EDD337A3FA4B0583EEC
:10F41000841E7A3F97395A3E04097A3F6AC25B3E9E
:10F420005EF3793F1A4B5D3E91DD793FA8D35E3E96
:10F430009DC7793F135C603E83B1793F5CE4613ED8
:10F44000439B793F836C633EDC84793F86F4643E62
:10F450004E6E793F667C663E9A57793F2204683E3D
:10F46000C040793FBA8B693EBF29793F2F136B3E6D
:10F470009812793F7F9A6C3E4AFB783FAB216E3EF3
:10F48000D6E3783FB2A86F3E3BCC783F942F713ED5
:10F490007BB4783F51B6723E939C783FE83C743E13
:10F4A0008684783F5AC3753E526C783FA649773EB2
:10F4B000F853783FCCCF783E773B783FCB557A3EB8
:10F4C000D122783FA4DB7B3E040A783F56617D3E23
:10F4D00010F1773FE1E67E3EF7D7773F2236803E58
:10F4E000B7BE773FC0F8803E51A5773F4ABB813E0B
:10F4F000C58B773FC07D823E1372773F2240833EAB
:10F500003A58773F7002843E3C3E773FAAC4843E1F
:10F510001724773FCE86853ECC09773FDF48863E6D
:10F520005BEF763FDA0A873EC4D4763FC1CC873E94
:10F5300007BA763F938E883E249F763F5050893E8F
:10F540001B84763FF8118A3EEC68763F8AD38A3E68
:10F55000974D763F07958B3E1B32763F6E568C3E1D
:10F560007A16763FC0178D3EB3FA753FFCD88D3EB4
:10F57000C6DE753F229A8E3EB3C2753F325B8F3E28
:10F580007BA6753F2C1C903E1C8A753F10DD903E7B
:10F59000976D753FDD9D913EED50753F945E923EB7
:10F5A0001D34753F351F933E2717753FBFDF933ED0
:10F5B0000BFA743F31A0943EC9DC743F8D60953ED8
:10F5C00062BF743FD220963ED5A1743F00E1963EC3
:10F5D0002284743F17A1973E4966743F1661983E96
:10F5E0004B48743FFE20993E272A743FCEE0993E57
:10F5F000DD0B743F86A09A3E6EED733F27609B3E05
:10F60000D9CE733FAF1F9C3E1FB0733F20DF9C3E9F
:10F610003F91733F789E9D3E3972733FB85D9E3E29
:10F620000E53733FDF1C9F3EBE33733FEEDB9F3EA6
:10F630004714733FE59AA03EACF4723FC259A13E15
:10F64000EBD4723F8718A23E04B5723F33D7A23E77
:10F65000F894723FC595A33EC774723F3F54A43ED1
:10F660007054723F9F12A53EF433723FE5D0A53E21
:10F670005213723F128FA63E8CF2713F254DA73E6A
:10F680009FD1713F1F0BA83E8EB0713FFEC8A83EB0
:10F69000578F713FC486A93EFB6D713F6F44AA3EF0
:10F6A0007A4C713F0102AB3ED42A713F77BFAB3E2B
:10F6B0000809713FD47CAC3E17E7703F153AAD3E68
:10F6C00002C5703F3CF7AD3EC6A2703F49B4AE3EA6
:10F6D0006680703F3A71AF3EE15D703F102EB03EE4
:10F6E000373B703FCBEAB03E6718703F6BA7B13E27
:10F6F00073F56F3FEF63B23E5AD26F3F5820B33E6F
:10F700001BAF6F3FA5DCB33EB88B6F3FD698B43EBE
:10F7100030686F3FEC54B53E83446F3FE610B63E11
:10F72000B0206F3FC3CCB63EBAFC6E3F8488B73E74
:10F730009ED86E3F2A44B83E5DB46E3FB2FFB83EDD
:10F74000F88F6E3F1EBBB93E6D6B6E3F6E76BA3E54
:10F75000BE466E3FA031BB3EEB216E3FB6ECBB3EDA
:10F76000F2FC6D3FAFA7BC3ED5D76D3F8B62BD3E6F
:10F7700093B26D3F4A1DBE3E2D8D6D3FEBD7BE3E11
:10F78000A1676D3F6F92BF3EF2416D3FD54CC03EC9
:10F790001D1C6D3F1E07C13E24F66C3F48C1C13E93
:10F7A00007D06C3F557BC23EC5A96C3F4435C33E74
:10F7B0005E836C3F15EFC33ED45C6C3FC8A8C43E6B
:10F7C00024366C3F5C62C53E500F6C3FD21BC63E78
:10F7D00058E86B3F29D5C63E3BC16B3F628EC73EA2
:10F7E000FB996B3F7C47C83E95726B3F7700C93EE3
:10F7F0000C4B6B3F53B9C93E5E236B3F1072CA3E40
:10F800008CFB6A3FAE2ACB3E95D36A3F2CE3CB3EBE
:10F810007BAB6A3F8B9BCC3E3C836A3FCA53CD3E59
:10F82000D95A6A3FEA0BCE3E52326A3FEAC3CE3E15
:10F83000A7096A3FCA7BCF3ED7E0693F8A33D03EF3
:10F84000E4B7693F2AEBD03ECC8E693FAAA2D13EF5
:10F850009165693F095AD23E323C693F4811D33E17
:10F86000AE12693F67C8D33E07E9683F647FD43E64
:10F870003CBF683F4136D53E4C95683FFDECD53ED8
:10F88000396B683F99A3D63E0341683F135AD73E70
:10F89000A816683F6B10D83E2AEC673FA3C6D83E37
:10F8A00087C1673FB97CD93EC196673FAD32DA3E2A
:10F8B000D86B673F80E8DA3ECA40673F319EDB3E47
:10F8C0009915673FC153DC3E45EA663F2E09DD3E90
:10F8D000CCBE663F79BEDD3E3093663FA273DE3E0E
:10F8E0007167663FA928DF3E8E3B663F8DDDDF3EB8
:10F8F000880F663F4F92E03E5EE3653FEE46E13E95
:10F9000010B7653F6AFBE13EA08A653FC4AFE23EA7
:10F910000B5E653FFA63E33E5431653F0E18E43EEB
:10F920007904653FFECBE43E7BD7643FCB7FE53E69
:10F9300059AA643F7533E63E147D643FFBE6E63E1C
:10F94000AC4F643F5D9AE73E2122643F9C4DE83E08
:10F9500073F4633FB700E93EA1C6633FAEB3E93E2F
:10F96000AC98633F8166EA3E956A633F3019EB3E8F
:10F970005A3C633FBBCBEB3EFC0D633F217EEC3E2C
:10F980007BDF623F6330ED3ED7B0623F80E2ED3E09
:10F990001082623F7994EE3E2653623F4C46EF3E22
:10F9A0001A24623FFBF7EF3EEAF4613F85A9F03E7F
:10F9B00098C5613FEA5AF13E2296613F290CF23E1A
:10F9C0008A66613F43BDF23ED036613F386EF33EFA
:10F9D000F206613F071FF43EF2D6603FB1CFF43E1E
:10F9E000CFA6603F3580F53E8976603F9330F63E86
:10F9F0002146603FCBE0F63E9615603FDC90F73E37
:10FA0000E9E45F3FC840F83E19B45F3F8EF0F83E2E
:10FA100027835F3F2DA0F93E12525F3FA54FFA3E6C
:10FA2000DB205F3FF7FEFA3E81EF5E3F22AEFB3EFA
:10FA300005BE5E3F275DFC3E678C5E3F040CFD3ECD
:10FA4000A65A5E3FBBBAFD3EC3285E3F4A69FE3EF2
:10FA5000BEF65D3FB217FF3E97C45D3FF3C5FF3E64
:10FA60004D925D3F063A003FE15F5D3FFF90003FF2
:10FA7000532D5D3FE4E7003FA3FA5C3FB53E013FF5
:10FA8000D1C75C3F7395013FDD945C3F1CEC013FA7
:10FA9000C7615C3FB142023F8E2E5C3F3299023F0C
:10FAA00034FB5B3F9FEF023FB8C75B3FF845033F26
:10FAB0001A945B3F3D9C033F5A605B3F6DF2033FEE
:10FAC000792C5B3F8948043F75F85A3F919E043F6B
:10FAD00050C45A3F84F4043F09905A3F624A053F9C
:10FAE000A05B5A3F2CA0053F16275A3FE2F5053F81
:10FAF0006AF2593F824B063F9CBD593F0EA1063F1B
:10FB0000AD88593F86F6063F9C53593FE84B073F67
:10FB10006A1E593F36A1073F17E9583F6FF6073F66
:10FB2000A1B3583F924B083F0B7E583FA1A0083F1E
:10FB30005348583F9BF5083F7912583F7F4A093F89
:10FB40007FDC573F4E9F093F63A6573F09F4093FAB
:10FB50002670573FAD480A3FC739573F3D9D0A3F82
:10FB60004803573FB7F10A3FA7CC563F1C460B3F0F
:10FB7000E595563F6B9A0B3F025F563FA5EE0B3F54
:10FB8000FE27563FC9420C3FD9F0553FD7960C3F50
:10FB900093B9553FD0EA0C3F2C82553FB33E0D3F01
:10FBA000A44A553F81920D3FFB12553F38E60D3F69
:10FBB00031DB543FDA390E3F47A3543F658D0E3F8A
:10FBC0003B6B543FDBE00E3F0F33543F3B340F3F62
:10FBD000C3FA533F84870F3F55C2533FB8DA0F3FF4
:10FBE000C789533FD52D103F1851533FDC80103F3C
:10FBF0004918533FCDD3103F59DF523FA726113F3D
:10FC000049A6523F6B79113F186D523F19CC113FF5
:10FC1000C633523FB01E123F54FA513F3071123F6B
:10FC2000C2C0513F9AC3123F1087513FEE15133F98
:10FC30003D4D513F2A68133F4A13513F50BA133F7D
:10FC400037D9503F5F0C143F039F503F585E143F1D
:10FC5000AF64503F39B0143F3B2A503F0402153F78
:10FC6000A8EF4F3FB753153FF4B44F3F54A5153F8E
:10FC70001F7A4F3FD9F6153F2B3F4F3F4748163F5E
:10FC800017044F3F9F99163FE4C84E3FDFEA163FE7
:10FC9000908D4E3F073C173F1C524E3F188D173F2B
:10FCA00089164E3F12DE173FD5DA4D3FF52E183F2D
:10FCB000029F4D3FC07F183F10634D3F73D0183FE8
:10FCC000FD264D3F0F21193FCBEA4C3F9471193F60
:10FCD00079AE4C3F00C2193F08724C3F55121A3F93
:10FCE00078354C3F93621A3FC7F84B3FB8B21A3F82
:10FCF000F8BB4B3FC6021B3F097F4B3FBB521B3F2C
:10FD0000FA414B3F99A21B3FCC044B3F5FF21B3F94
:10FD10007FC74A3F0C421C3F138A4A3FA2911C3FB7
:10FD2000874C4A3F1FE11C3FDC0E4A3F84301D3F99
:10FD300012D1493FD17F1D3F2993493F06CF1D3F37
:10FD40002155493F221E1E3FFA16493F266D1E3F90
:10FD5000B3D8483F12BC1E3F4E9A483FE50A1F3FAA
:10FD6000CA5B483F9F591F3F271D483F41A81F3F7F
:10FD700065DE473FCBF61F3F849F473F3B45203F13
:10FD80008560473F9393203F6721473FD2E1203F63
:10FD90002AE2463FF92F213FCEA2463F067E213F71
:10FDA0005463463FFBCB213FBB23463FD719223F3D
:10FDB00003E4453F9967223F2DA4453F43B5223FC9
:10FDC0003964453FD302233F2624453F4B50233F10
:10FDD000F5E3443FA99D233FA5A3443FEEEA233F1B
:10FDE0003763443F1A38243FAB22443F2C85243FDD
:10FDF00000E2433F25D2243F38A1433F041F253F63
:10FE00005160433FCB6B253F4C1F433F77B8253FA5
:10FE100029DE423F0A05263FE89C423F8451263FA7
:10FE2000895B423FE39D263F0B1A423F2AEA263F69
:10FE300070D8413F5636273FB796413F6882273FEB
:10FE4000E154413F61CE273FEC12413F401A283F29
:10FE5000DAD0403F0566283FA98E403FB0B1283F29
:10FE60005C4C403F41FD283FF009403FB848293FE6
:10FE700067C73F3F1594293FC0843F3F57DF293F65
:10FE8000FC413F3F802A2A3F1BFF3E3F8E752A3FA1
:10FE90001BBC3E3F82C02A3FFF783E3F5B0B2B3F9F
:10FEA000C5353E3F1B562B3F6EF23D3FBFA02B3F5B
:10FEB000F9AE3D3F4AEB2B3F676B3D3FB9352C3FD9
:10FEC000B8273D3F0F802C3FECE33C3F49CA2C3F15
:10FED00003A03C3F69142D3FFC5B3C3F6F5E2D3F10
:10FEE000D9173C3F59A82D3F98D33B3F29F22D3FCE
:10FEF0003B8F3B3FDE3B2E3FC14A3B3F78852E3F49
:10FF000029063B3FF7CE2E3F75C13A3F5B182F3F86
:10FF1000A47C3A3FA5612F3FB7373A3FD3AA2F3F82
:10FF2000ACF2393FE6F32F3F85AD393FDE3C303F41
:10FF30004268393FBB85303FE122393F7CCE303FBC
:10FF400065DD383F2217313FCB97383FAD5F313FFA
:10FF50001652383F1DA8313F430C383F71F0313FF6
:10FF600055C6373FAA38323F4A80373FC780323FB5
:10FF7000233A373FC9C8323FDFF3363FAF10333F34
:10FF80007FAD363F7A58333F0467363F29A0333F71
:10FF90006C20363FBCE7333FB8D9353F342F343F70
:10FFA000E792353F8F76343FFB4B353FCFBD343F33
:10FFB000F304353FF304353FCFBD343FFB4B353FB2
:10FFC0008F76343FE792353F342F343FB8D9353FF1
:10FFD000BCE7333F6C20363F29A0333F0467363FF0
:10FFE0007A58333F7FAD363FAF10333FDFF3363FB4
:10FFF000C9C8323F233A373FC780323F4A80373F34
:020000040801F1
:10000000AA38323F55C6373F71F0313F430C383F75
:100010001DA8313F1652383FAD5F313FCB97383F77
:100020002217313F65DD383F7CCE303FE122393F3A
:10003000BB85303F4268393FDE3C303F85AD393FBC
:10004000E6F32F3FACF2393FD3AA2F3FB7373A3F01
:10005000A5612F3FA47C3A3F5B182F3F75C13A3F03
:10006000F7CE2E3F29063B3F78852E3FC14A3B3FC6
:10007000DE3B2E3F3B8F3B3F29F22D3F98D33B3F4A
:1000800059A82D3FD9173C3F6F5E2D3FFC5B3C3F8D
:1000900069142D3F03A03C3F49CA2C3FECE33C3F91
:1000A0000F802C3FB8273D3FB9352C3F676B3D3F54
:1000B0004AEB2B3FF9AE3D3FBFA02B3F6EF23D3FD9
:1000C0001B562B3FC5353E3F5B0B2B3FFF783E3F1A
:1000D00082C02A3F1BBC3E3F8E752A3F1BFF3E3F1E
:1000E000802A2A3FFC413F3F57DF293FC0843F3FE2
:1000F0001594293F67C73F3FB848293FF009403F63
:1001000041FD283F5C4C403FB0B1283FA98E403FA5
:100110000566283FDAD0403F401A283FEC12413FA5
:1001200061CE273FE154413F6882273FB796413F68
:100130005636273F70D8413F2AEA263F0B1A423FE6
:10014000E39D263F895B423F8451263FE89C423F26
:100150000A05263F29DE423F77B8253F4C1F433F23
:10016000CB6B253F5160433F041F253F38A1433FE0
:1001700025D2243F00E2433F2C85243FAB22443F5D
:100180001A38243F3763443FEEEA233FA5A3443F98
:10019000A99D233FF5E3443F4B50233F2624453F91
:1001A000D302233F3964453F43B5223F2DA4453F49
:1001B0009967223F03E4453FD719223FBB23463FBF
:1001C000FBCB213F5463463F067E213FCEA2463FF4
:1001D000F92F213F2AE2463FD2E1203F6721473FE6
:1001E0009393203F8560473F3B45203F849F473F97
:1001F000CBF61F3F65DE473F41A81F3F271D483F05
:100200009F591F3FCA5B483FE50A1F3F4E9A483F30
:1002100012BC1E3FB3D8483F266D1E3FFA16493F19
:10022000221E1E3F2155493F06CF1D3F2993493FBE
:10023000D17F1D3F12D1493F84301D3FDC0E4A3F24
:100240001FE11C3F874C4A3FA2911C3F138A4A3F43
:100250000C421C3F7FC74A3F5FF21B3FCC044B3F21
:1002600099A21B3FFA414B3FBB521B3F097F4B3FBB
:10027000C6021B3FF8BB4B3FB8B21A3FC7F84B3F13
:1002800093621A3F78354C3F55121A3F08724C3F23
:1002900000C2193F79AE4C3F9471193FCBEA4C3FF5
:1002A0000F21193FFD264D3F73D0183F10634D3F7E
:1002B000C07F183F029F4D3FF52E183FD5DA4D3FC6
:1002C00012DE173F89164E3F188D173F1C524E3FC6
:1002D000073C173F908D4E3FDFEA163FE4C84E3F84
:1002E0009F99163F17044F3F4748163F2B3F4F3FFC
:1002F000D9F6153F1F7A4F3F54A5153FF4B44F3F31
:10030000B753153FA8EF4F3F0402153F3B2A503F1C
:1003100039B0143FAF64503F585E143F039F503FC5
:100320005F0C143F37D9503F50BA133F4A13513F27
:100330002A68133F3D4D513FEE15133F1087513F43
:100340009AC3123FC2C0513F3071123F54FA513F1D
:10035000B01E123FC633523F19CC113F186D523FA9
:100360006B79113F49A6523FA726113F59DF523FF3
:10037000CDD3103F4918533FDC80103F1851533FF5
:10038000D52D103FC789533FB8DA0F3F55C2533FB1
:1003900084870F3FC3FA533F3B340F3F0F33543F23
:1003A000DBE00E3F3B6B543F658D0E3F47A3543F50
:1003B000DA390E3F31DB543F38E60D3FFB12553F33
:1003C00081920D3FA44A553FB33E0D3F2C82553FCD
:1003D000D0EA0C3F93B9553FD7960C3FD9F0553F23
:1003E000C9420C3FFE27563FA5EE0B3F025F563F2A
:1003F0006B9A0B3FE595563F1C460B3FA7CC563FEB
:10040000B7F10A3F4803573F3D9D0A3FC739573F61
:10041000AD480A3F2670573F09F4093F63A6573F8E
:100420004E9F093F7FDC573F7F4A093F7912583F73
:100430009BF5083F5348583FA1A0083F0B7E583F0B
:10044000924B083FA1B3583F6FF6073F17E9583F5B
:1004500036A1073F6A1E593FE84B073F9C53593F5F
:1004600086F6063FAD88593F0EA1063F9CBD593F19
:10047000824B063F6AF2593FE2F5053F16275A3F85
:100480002CA0053FA05B5A3F624A053F09905A3FA6
:1004900084F4043F50C45A3F919E043F75F85A3F7C
:1004A0008948043F792C5B3F6DF2033F5A605B3F04
:1004B0003D9C033F1A945B3FF845033FB8C75B3F41
:1004C0009FEF023F34FB5B3F3299023F8E2E5C3F31
:1004D000B142023FC7615C3F1CEC013FDD945C3FD1
:1004E0007395013FD1C75C3FB53E013FA3FA5C3F26
:1004F000E4E7003F532D5D3FFF90003FE15F5D3F2C
:10050000063A003F4D925D3FF3C5FF3E97C45D3F05
:10051000B217FF3EBEF65D3F4A69FE3EC3285E3F0E
:10052000BBBAFD3EA65A5E3F040CFD3E678C5E3FA3
:10053000275DFC3E05BE5E3F22AEFB3E81EF5E3F87
:10054000F7FEFA3EDB205F3FA54FFA3E12525F3FB7
:100550002DA0F93E27835F3F8EF0F83E19B45F3F30
:10056000C840F83EE9E45F3FDC90F73E9615603FF7
:10057000CBE0F63E2146603F9330F63E8976603F01
:100580003580F53ECFA6603FB1CFF43EF2D6603F56
:10059000071FF43EF206613F386EF33ED036613FEE
:1005A00043BDF23E8A66613F290CF23E2296613FCE
:1005B000EA5AF13E98C5613F85A9F03EEAF4613FF1
:1005C000FBF7EF3E1A24623F4C46EF3E2653623F54
:1005D0007994EE3E1082623F80E2ED3ED7B0623FFA
:1005E0006330ED3E7BDF623F217EEC3EFC0D633FDE
:1005F000BBCBEB3E5A3C633F3019EB3E956A633F01
:100600008166EA3EAC98633FAEB3E93EA1C6633F64
:10061000B700E93E73F4633F9C4DE83E2122643FFE
:100620005D9AE73EAC4F643FFBE6E63E147D643FD7
:100630007533E63E59AA643FCB7FE53E7BD7643FE6
:10064000FECBE43E7904653F0E18E43E5431653F2D
:10065000FA63E33E0B5E653FC4AFE23EA08A653FAE
:100660006AFBE13E10B7653FEE46E13E5EE3653F63
:100670004F92E03E880F663F8DDDDF3E8E3B663F4A
:10068000A928DF3E7167663FA273DE3E3093663F66
:1006900079BEDD3ECCBE663F2E09DD3E45EA663FB3
:1006A000C153DC3E9915673F319EDB3ECA40673F30
:1006B00080E8DA3ED86B673FAD32DA3EC196673FDD
:1006C000B97CD93E87C1673FA3C6D83E2AEC673FB5
:1006D0006B10D83EA816683F135AD73E0341683FB7
:1006E00099A3D63E396B683FFDECD53E4C95683FEB
:1006F0004136D53E3CBF683F647FD43E07E9683F42
:1007000067C8D33EAE12693F4811D33E323C693FC1
:10071000095AD23E9165693FAAA2D13ECC8E693F6B
:100720002AEBD03EE4B7693F8A33D03ED7E0693F39
:10073000CA7BCF3EA7096A3FEAC3CE3E52326A3F28
:10074000EA0BCE3ED95A6A3FCA53CD3E3C836A3F3C
:100750008B9BCC3E7BAB6A3F2CE3CB3E95D36A3F71
:10076000AE2ACB3E8CFB6A3F1072CA3E5E236B3FC3
:1007700053B9C93E0C4B6B3F7700C93E95726B3F36
:100780007C47C83EFB996B3F628EC73E3BC16B3FC7
:1007900029D5C63E58E86B3FD21BC63E500F6C3F72
:1007A0005C62C53E24366C3FC8A8C43ED45C6C3F36
:1007B00015EFC33E5E836C3F4435C33EC5A96C3F15
:1007C000557BC23E07D06C3F48C1C13E24F66C3F0A
:1007D0001E07C13E1D1C6D3FD54CC03EF2416D3F12
:1007E0006F92BF3EA1676D3FEBD7BE3E2D8D6D3F33
:1007F0004A1DBE3E93B26D3F8B62BD3ED5D76D3F65
:10080000AFA7BC3EF2FC6D3FB6ECBB3EEB216E3FAA
:10081000A031BB3EBE466E3F6E76BA3E6D6B6E3FFC
:100820001EBBB93EF88F6E3FB2FFB83E5DB46E3F5F
:100830002A44B83E9ED86E3F8488B73EBAFC6E3FCD
:10084000C3CCB63EB0206F3FE610B63E83446F3F48
:10085000EC54B53E30686F3FD698B43EB88B6F3FCE
:10086000A5DCB33E1BAF6F3F5820B33E5AD26F3F5B
:10087000EF63B23E73F56F3F6BA7B13E6718703FF1
:10088000CBEAB03E373B703F102EB03EE15D703F8B
:100890003A71AF3E6680703F49B4AE3EC6A2703F2B
:1008A0003CF7AD3E02C5703F153AAD3E17E7703FCD
:1008B000D47CAC3E0809713F77BFAB3ED42A713F70
:1008C0000102AB3E7A4C713F6F44AA3EFB6D713F13
:1008D000C486A93E578F713FFEC8A83E8EB0713FB7
:1008E0001F0BA83E9FD1713F254DA73E8CF2713F53
:1008F000128FA63E5213723FE5D0A53EF433723FED
:100900009F12A53E7054723F3F54A43EC774723F7D
:10091000C595A33EF894723F33D7A23E04B5723F0B
:100920008718A23EEBD4723FC259A13EACF4723F8D
:10093000E59AA03E4714733FEEDB9F3EBE33733F04
:10094000DF1C9F3E0E53733FB85D9E3E3972733F6E
:10095000789E9D3E3F91733F20DF9C3E1FB0733FCA
:10096000AF1F9C3ED9CE733F27609B3E6EED733F19
:1009700086A09A3EDD0B743FCEE0993E272A743F55
:10098000FE20993E4B48743F1661983E4966743F7D
:1009900017A1973E2284743F00E1963ED5A1743F93
:1009A000D220963E62BF743F8D60953EC9DC743F95
:1009B00031A0943E0BFA743FBFDF933E2717753F7B
:1009C000351F933E1D34753F945E923EED50753F4A
:1009D000DD9D913E976D753F10DD903E1C8A753F01
:1009E0002C1C903E7BA6753F325B8F3EB3C2753F99
:1009F000229A8E3EC6DE753FFCD88D3EB3FA753F17
:100A0000C0178D3E7A16763F6E568C3E1B32763F6F
:100A100007958B3E974D763F8AD38A3EEC68763FAA
:100A2000F8118A3E1B84763F5050893E249F763FC2
:100A3000938E883E07BA763FC1CC873EC4D4763FBA
:100A4000DA0A873E5BEF763FDF48863ECC09773F88
:100A5000CE86853E1724773FAAC4843E3C3E773F2E
:100A60007002843E3A58773F2240833E1372773FAC
:100A7000C07D823EC58B773F4ABB813E51A5773F03
:100A8000C0F8803EB7BE773F2236803EF7D7773F2B
:100A9000E1E67E3E10F1773F56617D3E040A783FE5
:100AA000A4DB7B3ED122783FCB557A3E773B783F23
:100AB000CCCF783EF853783FA649773E526C783FCA
:100AC0005AC3753E8684783FE83C743E939C783FD9
:100AD00051B6723E7BB4783F942F713E3BCC783F49
:100AE000B2A86F3ED6E3783FAB216E3E4AFB783F1B
:100AF0007F9A6C3E9812793F2F136B3EBF29793F46
:100B0000BA8B693EC040793F2204683E9A57793FCC
:100B1000667C663E4E6E793F86F4643EDC84793FA7
:100B2000836C633E439B793F5CE4613E83B1793FD4
:100B3000135C603E9DC7793FA8D35E3E91DD793F4F
:100B40001A4B5D3E5EF3793F6AC25B3E04097A3F11
:100B500097395A3E841E7A3FA4B0583EDD337A3F1F
:100B60008F27573E10497A3F589E553E1C5E7A3F6C
:100B70000115543E02737A3F898B523EC1877A3FFA
:100B8000F101513E599C7A3F38784F3ECBB07A3FC5
:100B900060EE4D3E16C57A3F67644C3E3AD97A3FC7
:100BA0004FDA4A3E37ED7A3F1850493E0E017B3FFF
:100BB000C2C5473EBE147B3F4D3B463E48287B3F67
:100BC000B9B0443EAB3B7B3F0726433EE74E7B3FFD
:100BD000379B413EFC617B3F4910403EEA747B3FBE
:100BE0003E853E3EB2877B3F15FA3C3E539A7B3FA3
:100BF000CF6E3B3ECDAC7B3F6CE3393E20BF7B3FAD
:100C0000EC57383E4DD17B3F50CC363E53E37B3FD3
:100C10009840353E31F57B3FC4B4333EE9067C3F16
:100C2000D428323E7A187C3FC99C303EE5297C3F6F
:100C3000A2102F3E283B7C3F61842D3E444C7C3FDC
:100C400004F82B3E3A5D7C3F8D6B2A3E086E7C3F5C
:100C5000FCDE283EB07E7C3F5152273E318F7C3FE8
:100C60008CC5253E8A9F7C3FAD38243EBDAF7C3F7E
:100C7000B6AB223EC9BF7C3FA51E213EAECF7C3F16
:100C80007B911F3E6CDF7C3F38041E3E03EF7C3FB0
:100C9000DE761C3E73FE7C3F6BE91A3EBC0D7D3F49
:100CA000E05B193EDD1C7D3F3DCE173ED82B7D3FDE
:100CB0008340163EAC3A7D3FB2B2143E59497D3F67
:100CC000CA24133EDE577D3FCC96113E3D667D3FE4
:100CD000B708103E74747D3F8B7A0E3E85827D3F4F
:100CE0004AEC0C3E6E907D3FF35D0B3E309E7D3FA7
:100CF00086CF093ECCAB7D3F0541083E40B97D3FE4
:100D00006EB2063E8CC67D3FC223053EB2D37D3F08
:100D10000295033EB1E07D3F2E06023E88ED7D3F09
:100D20004577003E38FA7D3F92D0FD3DC2067E3FBA
:100D300073B2FA3D24137E3F2C94F73D5E1F7E3F35
:100D4000C075F43D722B7E3F2E57F13D5E377E3FDE
:100D50007638EE3D23437E3F9A19EB3DC14E7E3FF0
:100D60009AFAE73D385A7E3F76DBE43D88657E3F60
:100D70002EBCE13DB0707E3FC49CDE3DB17B7E3F2A
:100D8000377DDB3D8B867E3F895DD83D3D917E3F43
:100D9000B93DD53DC99B7E3FC81DD23D2DA67E3FA6
:100DA000B7FDCE3D69B07E3F86DDCB3D7FBA7E3F4D
:100DB00036BDC83D6DC47E3FC69CC53D34CE7E3F2A
:100DC000397CC23DD4D77E3F8D5BBF3D4CE17E3F39
:100DD000C33ABC3D9DEA7E3FDD19B93DC7F37E3F76
:100DE000DAF8B53DC9FC7E3FBBD7B23DA4057F3FD5
:100DF00080B6AF3D580E7F3F2B95AC3DE4167F3F4C
:100E0000BA73A93D491F7F3F3052A63D87277F3FD8
:100E10008C30A33D9D2F7F3FCF0EA03D8D377F3F70
:100E2000F9EC9C3D543F7F3F0ACB993DF4467F3F10
:100E300005A9963D6D4E7F3FE786933DBF557F3FA9
:100E4000B464903DE95C7F3F6A428D3DEC637F3F37
:100E50000A208A3DC76A7F3F94FD863D7B717F3FB4
:100E60000ADB833D08787F3F6CB8803D6D7E7F3F15
:100E7000742B7B3DAB847F3FE9E5743DC28A7F3FA5
:100E800038A06E3DB1907F3F625A683D78967F3FB3
:100E90006814623D189C7F3F4CCE5B3D91A17F3F23
:100EA0000E88553DE3A67F3FAF414F3D0DAC7F3FE0
:100EB0002FFB483D0FB17F3F91B4423DEAB57F3FE4
:100EC000D56D3C3D9EBA7F3FFC26363D2ABF7F3F15
:100ED00007E02F3D8FC37F3FF698293DCCC77F3F6A
:100EE000CC51233DE2CB7F3F880A1D3DD1CF7F3FD0
:100EF0002CC3163D98D37F3FB87B103D37D77F3F3B
:100F00002F340A3DAFDA7F3F90EC033D00DE7F3F98
:100F1000B949FB3C29E17F3F2DBAEE3C2BE47F3FF2
:100F20007B2AE23C05E77F3FA69AD53CB8E97F3FA4
:100F3000B00AC93C43EC7F3F9B7ABC3CA7EE7F3FA5
:100F400069EAAF3CE3F07F3F1C5AA33CF8F27F3FD5
:100F5000B6C9963CE6F47F3F38398A3CACF67F3F11
:100F60004B517B3C4AF87F3F0030623CC1F97F3FE8
:100F7000900E493C11FB7F3F02ED2F3C39FC7F3F37
:100F800059CB163C39FD7F3F3053FB3B13FE7F3F6F
:100F9000890FC93BC4FE7F3FC1CB963B4EFF7F3FCD
:100FA000C70F493BB1FF7F3FD40FC93AECFF7F3FEA
:100FB000000000000000803FD40FC9BAECFF7F3F63
:100FC000C70F49BBB1FF7F3FC1CB96BB4EFF7F3FF1
:100FD000890FC9BBC4FE7F3F3053FBBB13FE7F3F6D
:100FE00059CB16BC39FD7F3F02ED2FBC39FC7F3F4A
:100FF000900E49BC11FB7F3F003062BCC1F97F3FBE
:101000004B517BBC4AF87F3F38398ABCACF67F3FF6
:10101000B6C996BCE6F47F3F1C5AA3BCF8F27F3FEA
:1010200069EAAFBCE3F07F3F9B7ABCBCA7EE7F3F91
:10103000B00AC9BC43EC7F3FA69AD5BCB8E97F3F54
:101040007B2AE2BC05E77F3F2DBAEEBC2BE47F3F55
:10105000B949FBBC29E17F3F90EC03BD00DE7F3F37
:101060002F340ABDAFDA7F3FB87B10BD37D77F3F43
:101070002CC316BD98D37F3F880A1DBDD1CF7F3FBB
:10108000CC5123BDE2CB7F3FF69829BDCCC77F3F33
:1010900007E02FBD8FC37F3FFC2636BD2ABF7F3FB1
:1010A000D56D3CBD9EBA7F3F91B442BDEAB57F3F4E
:1010B0002FFB48BD0FB17F3FAF414FBD0DAC7F3F10
:1010C0000E8855BDE3A67F3F4CCE5BBD91A17F3F0F
:1010D000681462BD189C7F3F625A68BD78967F3F56
:1010E00038A06EBDB1907F3FE9E574BDC28A7F3FF5
:1010F000742B7BBDAB847F3F6CB880BD6D7E7F3F22
:101100000ADB83BD08787F3F94FD86BD7B717F3FFE
:101110000A208ABDC76A7F3F6A428DBDEC637F3F6C
:10112000B46490BDE95C7F3FE78693BDBF557F3FC8
:1011300005A996BD6D4E7F3F0ACB99BDF4467F3F12
:10114000F9EC9CBD543F7F3FCF0EA0BD8D377F3F54
:101150008C30A3BD9D2F7F3F3052A6BD87277F3F98
:10116000BA73A9BD491F7F3F2B95ACBDE4167F3FE5
:1011700080B6AFBD580E7F3FBBD7B2BDA4057F3F41
:10118000DAF8B5BDC9FC7E3FDD19B9BDC7F37E3FB6
:10119000C33ABCBD9DEA7E3F8D5BBFBD4CE17E3F47
:1011A000397CC2BDD4D77E3FC69CC5BD34CE7E3F00
:1011B00036BDC8BD6DC47E3F86DDCBBD7FBA7E3FE8
:1011C000B7FDCEBD69B07E3FC81DD2BD2DA67E3F06
:1011D000B93DD5BDC99B7E3F895DD8BD3D917E3F60
:1011E000377DDBBD8B867E3FC49CDEBDB17B7E3F01
:1011F0002EBCE1BDB0707E3F76DBE4BD88657E3FEE
:101200009AFAE7BD385A7E3F9A19EBBDC14E7E3F30
:101210007638EEBD23437E3F2E57F1BD5E377E3FCD
:10122000C075F4BD722B7E3F2C94F7BD5E1F7E3FD0
:1012300073B2FABD24137E3F92D0FDBDC2067E3F3D
:10124000457700BE38FA7D3F2E0602BE88ED7D3F11
:10125000029503BEB1E07D3FC22305BEB2D37D3F00
:101260006EB206BE8CC67D3F054108BE40B97D3FCB
:1012700086CF09BECCAB7D3FF35D0BBE309E7D3F7C
:101280004AEC0CBE6E907D3F8B7A0EBE85827D3F10
:10129000B70810BE74747D3FCC9611BE3D667D3F8D
:1012A000CA2413BEDE577D3FB2B214BE59497D3FFA
:1012B000834016BEAC3A7D3F3DCE17BED82B7D3F56
:1012C000E05B19BEDD1C7D3F6BE91ABEBC0D7D3FA6
:1012D000DE761CBE73FE7C3F38041EBE03EF7C3FEF
:1012E0007B911FBE6CDF7C3FA51E21BEAECF7C3F35
:1012F000B6AB22BEC9BF7C3FAD3824BEBDAF7C3F7C
:101300008CC525BE8A9F7C3F515227BE318F7C3FC2
:10131000FCDE28BEB07E7C3F8D6B2ABE086E7C3F13
:1013200004F82BBE3A5D7C3F61842DBE444C7C3F6B
:10133000A2102FBE283B7C3FC99C30BEE5297C3FD4
:10134000D42832BE7A187C3FC4B433BEE9067C3F51
:10135000984035BE31F57B3F50CC36BE53E37B3FE2
:10136000EC5738BE4DD17B3F6CE339BE20BF7B3F8D
:10137000CF6E3BBECDAC7B3F15FA3CBE539A7B3F54
:101380003E853EBEB2877B3F491040BEEA747B3F3C
:10139000379B41BEFC617B3F072643BEE74E7B3F48
:1013A000B9B044BEAB3B7B3F4D3B46BE48287B3F7C
:1013B000C2C547BEBE147B3F185049BE0E017B3FDD
:1013C0004FDA4ABE37ED7A3F67644CBE3AD97A3F6E
:1013D00060EE4DBE16C57A3F38784FBECBB07A3F2F
:1013E000F10151BE599C7A3F898B52BEC1877A3F29
:1013F000011554BE02737A3F589E55BE1C5E7A3F5B
:101400008F2757BE10497A3FA4B058BEDD337A3FCC
:1014100097395ABE841E7A3F6AC25BBE04097A3F7E
:101420001A4B5DBE5EF3793FA8D35EBE91DD793F76
:10143000135C60BE9DC7793F5CE461BE83B1793FB8
:10144000836C63BE439B793F86F464BEDC84793F42
:10145000667C66BE4E6E793F220468BE9A57793F1D
:10146000BA8B69BEC040793F2F136BBEBF29793F4D
:101470007F9A6CBE9812793FAB216EBE4AFB783FD3
:10148000B2A86FBED6E3783F942F71BE3BCC783FB5
:1014900051B672BE7BB4783FE83C74BE939C783FF3
:1014A0005AC375BE8684783FA64977BE526C783F92
:1014B000CCCF78BEF853783FCB557ABE773B783F98
:1014C000A4DB7BBED122783F56617DBE040A783F03
:1014D000E1E67EBE10F1773F223680BEF7D7773F38
:1014E000C0F880BEB7BE773F4ABB81BE51A5773FEB
:1014F000C07D82BEC58B773F224083BE1372773F8B
:10150000700284BE3A58773FAAC484BE3C3E773FFF
:10151000CE8685BE1724773FDF4886BECC09773F4D
:10152000DA0A87BE5BEF763FC1CC87BEC4D4763F74
:10153000938E88BE07BA763F505089BE249F763F6F
:10154000F8118ABE1B84763F8AD38ABEEC68763F48
:1015500007958BBE974D763F6E568CBE1B32763FFD
:10156000C0178DBE7A16763FFCD88DBEB3FA753F94
:10157000229A8EBEC6DE753F325B8FBEB3C2753F08
:101580002C1C90BE7BA6753F10DD90BE1C8A753F5B
:10159000DD9D91BE976D753F945E92BEED50753F97
:1015A000351F93BE1D34753FBFDF93BE2717753FB0
:1015B00031A094BE0BFA743F8D6095BEC9DC743FB8
:1015C000D22096BE62BF743F00E196BED5A1743FA3
:1015D00017A197BE2284743F166198BE4966743F76
:1015E000FE2099BE4B48743FCEE099BE272A743F37
:1015F00086A09ABEDD0B743F27609BBE6EED733FE5
:10160000AF1F9CBED9CE733F20DF9CBE1FB0733F7F
:10161000789E9DBE3F91733FB85D9EBE3972733F09
:10162000DF1C9FBE0E53733FEEDB9FBEBE33733F86
:10163000E59AA0BE4714733FC259A1BEACF4723FF5
:101640008718A2BEEBD4723F33D7A2BE04B5723F57
:10165000C595A3BEF894723F3F54A4BEC774723FB1
:101660009F12A5BE7054723FE5D0A5BEF433723F01
:10167000128FA6BE5213723F254DA7BE8CF2713F4A
:101680001F0BA8BE9FD1713FFEC8A8BE8EB0713F90
:10169000C486A9BE578F713F6F44AABEFB6D713FD0
:1016A0000102ABBE7A4C713F77BFABBED42A713F0B
:1016B000D47CACBE0809713F153AADBE17E7703F48
:1016C0003CF7ADBE02C5703F49B4AEBEC6A2703F86
:1016D0003A71AFBE6680703F102EB0BEE15D703FC4
:1016E000CBEAB0BE373B703F6BA7B1BE6718703F07
:1016F000EF63B2BE73F56F3F5820B3BE5AD26F3F4F
:10170000A5DCB3BE1BAF6F3FD698B4BEB88B6F3F9E
:10171000EC54B5BE30686F3FE610B6BE83446F3FF1
:10172000C3CCB6BEB0206F3F8488B7BEBAFC6E3F54
:101730002A44B8BE9ED86E3FB2FFB8BE5DB46E3FBD
:101740001EBBB9BEF88F6E3F6E76BABE6D6B6E3F34
:10175000A031BBBEBE466E3FB6ECBBBEEB216E3FBA
:10176000AFA7BCBEF2FC6D3F8B62BDBED5D76D3F4F
:101770004A1DBEBE93B26D3FEBD7BEBE2D8D6D3FF1
:101780006F92BFBEA1676D3FD54CC0BEF2416D3FA9
:101790001E07C1BE1D1C6D3F48C1C1BE24F66C3F73
:1017A000557BC2BE07D06C3F4435C3BEC5A96C3F54
:1017B00015EFC3BE5E836C3FC8A8C4BED45C6C3F4B
:1017C0005C62C5BE24366C3FD21BC6BE500F6C3F58
:1017D00029D5C6BE58E86B3F628EC7BE3BC16B3F82
:1017E0007C47C8BEFB996B3F7700C9BE95726B3FC3
:1017F00053B9C9BE0C4B6B3F1072CABE5E236B3F20
:10180000AE2ACBBE8CFB6A3F2CE3CBBE95D36A3F9E
:101810008B9BCCBE7BAB6A3FCA53CDBE3C836A3F39
:10182000EA0BCEBED95A6A3FEAC3CEBE52326A3FF5
:10183000CA7BCFBEA7096A3F8A33D0BED7E0693FD3
:101840002AEBD0BEE4B7693FAAA2D1BECC8E693FD5
:10185000095AD2BE9165693F4811D3BE323C693FF7
:1018600067C8D3BEAE12693F647FD4BE07E9683F44
:101870004136D5BE3CBF683FFDECD5BE4C95683FB8
:1018800099A3D6BE396B683F135AD7BE0341683F50
:101890006B10D8BEA816683FA3C6D8BE2AEC673F17
:1018A000B97CD9BE87C1673FAD32DABEC196673F0A
:1018B00080E8DABED86B673F319EDBBECA40673F27
:1018C000C153DCBE9915673F2E09DDBE45EA663F70
:1018D00079BEDDBECCBE663FA273DEBE3093663FEE
:1018E000A928DFBE7167663F8DDDDFBE8E3B663F98
:1018F0004F92E0BE880F663FEE46E1BE5EE3653F75
:101900006AFBE1BE10B7653FC4AFE2BEA08A653F87
:10191000FA63E3BE0B5E653F0E18E4BE5431653FCB
:10192000FECBE4BE7904653FCB7FE5BE7BD7643F49
:101930007533E6BE59AA643FFBE6E6BE147D643FFC
:101940005D9AE7BEAC4F643F9C4DE8BE2122643FE8
:10195000B700E9BE73F4633FAEB3E9BEA1C6633F0F
:101960008166EABEAC98633F3019EBBE956A633F6F
:10197000BBCBEBBE5A3C633F217EECBEFC0D633F0C
:101980006330EDBE7BDF623F80E2EDBED7B0623FE9
:101990007994EEBE1082623F4C46EFBE2653623F02
:1019A000FBF7EFBE1A24623F85A9F0BEEAF4613F5F
:1019B000EA5AF1BE98C5613F290CF2BE2296613FFA
:1019C00043BDF2BE8A66613F386EF3BED036613FDA
:1019D000071FF4BEF206613FB1CFF4BEF2D6603FFE
:1019E0003580F5BECFA6603F9330F6BE8976603F66
:1019F000CBE0F6BE2146603FDC90F7BE9615603F17
:101A0000C840F8BEE9E45F3F8EF0F8BE19B45F3F0E
:101A10002DA0F9BE27835F3FA54FFABE12525F3F4C
:101A2000F7FEFABEDB205F3F22AEFBBE81EF5E3FDA
:101A3000275DFCBE05BE5E3F040CFDBE678C5E3FAD
:101A4000BBBAFDBEA65A5E3F4A69FEBEC3285E3FD2
:101A5000B217FFBEBEF65D3FF3C5FFBE97C45D3F44
:101A6000063A00BF4D925D3FFF9000BFE15F5D3FD2
:101A7000E4E700BF532D5D3FB53E01BFA3FA5C3FD5
:101A8000739501BFD1C75C3F1CEC01BFDD945C3F87
:101A9000B14202BFC7615C3F329902BF8E2E5C3FEC
:101AA0009FEF02BF34FB5B3FF84503BFB8C75B3F06
:101AB0003D9C03BF1A945B3F6DF203BF5A605B3FCE
:101AC000894804BF792C5B3F919E04BF75F85A3F4B
:101AD00084F404BF50C45A3F624A05BF09905A3F7C
:101AE0002CA005BFA05B5A3FE2F505BF16275A3F61
:101AF000824B06BF6AF2593F0EA106BF9CBD593FFB
:101B000086F606BFAD88593FE84B07BF9C53593F47
:101B100036A107BF6A1E593F6FF607BF17E9583F46
:101B2000924B08BFA1B3583FA1A008BF0B7E583FFE
:101B30009BF508BF5348583F7F4A09BF7912583F69
:101B40004E9F09BF7FDC573F09F409BF63A6573F8B
:101B5000AD480ABF2670573F3D9D0ABFC739573F62
:101B6000B7F10ABF4803573F1C460BBFA7CC563FEF
:101B70006B9A0BBFE595563FA5EE0BBF025F563F34
:101B8000C9420CBFFE27563FD7960CBFD9F0553F30
:101B9000D0EA0CBF93B9553FB33E0DBF2C82553FE1
:101BA00081920DBFA44A553F38E60DBFFB12553F49
:101BB000DA390EBF31DB543F658D0EBF47A3543F6A
:101BC000DBE00EBF3B6B543F3B340FBF0F33543F42
:101BD00084870FBFC3FA533FB8DA0FBF55C2533FD4
:101BE000D52D10BFC789533FDC8010BF1851533F1C
:101BF000CDD310BF4918533FA72611BF59DF523F1D
:101C00006B7911BF49A6523F19CC11BF186D523FD5
:101C1000B01E12BFC633523F307112BF54FA513F4B
:101C20009AC312BFC2C0513FEE1513BF1087513F78
